:020000040000FA
:040000006FD00400B9
:101000006F00907E00000000000000009020002093
:10101000AA220020A9BDF9F56C23002000000000E1
:10102000000000006C230020902000200000000041
:101030000000000090200020000000009020002010
:101040000000000090200020902000209020002030
:101050009020002090200020582F00209424002071
:101060000000000090200020902000201E2400207E
:1010700090200020D22300209020002090200020EB
:101080009020002090200020902000209020002020
:101090009020002001A04111B7170040985F3AC688
:1010A000945F3247E39CE6FE3245410182800111A4
:1010B00013078008F337078093F787083EC20100C3
:1010C0000100B7170040930570052380B70413068D
:1010D00080FA2380C7040100010083C6B70493F699
:1010E000F60DA385D704238007049246F3A6068055
:1010F0000100010093760502D5CEF336078093F602
:10110000860836C4010001002380B7042380C70489
:1011100001000100B70614007D89558D88C70100C4
:1011200001000100010023800704A246F3A6068007
:101130000100010073370780137787083AC6010062
:1011400001002380B7042380C704010001000100CF
:1011500001003727004093061005A303D7802380A2
:101160000704B247F3A70780010001009307800836
:10117000F3B7078093F787083ECE01000100B71749
:101180000040130770052380E704130780FA2380CB
:10119000E7040100010003C7B70413670708A3852C
:1011A000E70423800704F247F3A70780010001004A
:1011B0000561828093760504BDC6F336078093F6F9
:1011C000860836C8010001002380B7042380C704C5
:1011D00001000100B7061400938606047D89558D31
:1011E00088C7010001000100010023800704C246F6
:1011F000F3A6068001000100733707801377870884
:101200003ACA010001002380B7042380C70401000B
:1012100001003727004093062005A303D7802380D1
:101220000704D24781B773370780137787083ACC12
:10123000010001002380B7042380C70401000100DE
:1012400098471367070C98C723800704E24719BF24
:101250000111814601468145114506CE97000000E7
:10126000E780605893078008F3B7078093F78708F3
:101270003EC601000100B717004013077005238028
:10128000E704130780FA2380E7040100010003C785
:101290006704136717002383E70423800704B2471A
:1012A000F3A7078001000100F2400561828041112F
:1012B000814601468145114597000000E780A05214
:1012C00013078008F337078093F787083EC40100AF
:1012D0000100B7170040130670052380C70493066A
:1012E00080FA2380D70401000100FD552396B70240
:1012F00023800704A245F3A5058001000100733790
:101300000780137787083AC6010001002380C704CD
:101310002380D7040100010003C767041367170087
:101320002383E70423800704B247F3A70780010063
:10133000010001A0BD473305F50201007D1575FDD3
:101340008280411122C426C206C6AA8401446317C2
:101350009400B24022449244410182800504130566
:10136000803E420497000000E78000FD4180C5B741
:101370009305000273A04580824573901534924016
:101380002242B2424243D2436244F2440255925551
:101390002256B2564257D2576258F25806499649D9
:1013A000264AB64A464BD64B664CF64C065D965DD1
:1013B000265EB65E465FD65F09617300203041113C
:1013C000B7170040985F3AC6945F3247E39CE6FE49
:1013D000324541018280B71700401307000323887C
:1013E000E702854717170000232EF74673002030C9
:1013F000411122C42D6426C24AC006C637190040D6
:101400001304A4AAB704002023208900977000E0E9
:10141000E780A09B9C408297977000E0E780E09A6D
:10142000E5B737370040834747009146BD8B639E41
:10143000D702B73600401306F00F973500009385AA
:10144000651E9737000083D7E72D03C7A6001377E3
:10145000F70F1DE3B7E70400BC4F09468945171590
:1014600000000345A5F7829731A099466394D70001
:10147000834757007300203003C786001377F70FA8
:10148000E365F6FC13851700AE9717380000231BA1
:10149000A8282380E70075B7B787004003C7670017
:1014A000098B6309071003C77700930600031377BE
:1014B0000703630DD708173800000348F87717367D
:1014C0000000130666740547B30606012380E60094
:1014D00083C577001737000013070775429793F508
:1014E000F50F2300B70003C58700973500009385EB
:1014F000A572C2951375F50F2380A5000347070059
:1015000089451377F703630CB70C63E7E50A6306B5
:10151000071A8545630CB7129737000083C7D77148
:101520003307F600034707001377F70F19CB85073A
:1015300093F7F70F3D476363F71A17370000A30DC2
:10154000F76EB787004009472383E700B78700405D
:1015500083C77700E207E18763DE0704973700005F
:1015600083C7976D173700001307076A3E978546B4
:101570002300D700173700001307076B3E97930629
:1015800000032300D700173700001307E7683E97D2
:10159000A14685072300D70093F7F70F3D47636403
:1015A000F71417370000A309F768B7870040094709
:1015B0002383E70073002030930610026300D70EE8
:1015C000930620026305D70693060002E316D7F4BC
:1015D00003C727021377C70F13672700D5A803C7D0
:1015E00067001377070465CB03C7A702173800000D
:1015F00013080843173500001305453A1347070839
:101600002385E70203C7A7021377370F1367870005
:101610002385E702814713070004B305F5008C41D9
:10162000B306F80091078CC2E399E7FEF5B503C74E
:10163000A702134707042385E70203C7A70213770E
:10164000C70F136727002385E702F9B503C76700B3
:101650001377070449C303C767021738000013084C
:10166000E82F1735000013052527134707082383A4
:10167000E70203C767021377370F136787002383D7
:10168000E702814713070004B305F5008C41B30658
:10169000F80091078CC2E399E7FEBDBD03C767025E
:1016A000134707042383E70203C767021377C70FB3
:1016B000136727002383E70285B503C76700137705
:1016C000070411CB03C727021377370F136787006F
:1016D0002381E70291B5238006003DBD97370000C6
:1016E000A38C0754B9BD97370000A387075475BD75
:1016F0002303048015472303E48001002302A48010
:10170000828083076480E3CE07FE23030480828007
:1017100083076480E3CE07FE03454480828083070D
:101720006480E3CE07FE2302A4808280411126C498
:101730004AC24EC006C61377F50BAD47AA892E895B
:101740009544630CF700194597000000E78080FA84
:1017500097000000E78020FB8D444E859700000035
:10176000E78040F9FD59FD1463983401B240A2446A
:101770001249824941018280135509011375F50F01
:1017800097000000E780E0F92209F1BF011126CCA3
:1017900006CEB704080097000000E780C0F61545A4
:1017A00097000000E78000F597000000E78080F6D2
:1017B00097000000E78000F62AC697000000E78047
:1017C00080F432459377150089EB13651500137586
:1017D000F50FF240E24405618280FD14E9F0014515
:1017E000CDBF397126DC4ADA4ED852D656D45AD2F9
:1017F0005ED006DE62CE66CCB7E700E07D5783AAF6
:10180000070022C603AA470023A0E71823A2E7186F
:10181000B7170040130770052380E704130780FA09
:101820002380E70483C74704930B75FFB684E20760
:1018300093FBFB0F8546AA892E8B32893724004003
:10184000E187015763FA76016308D50089461307DB
:1018500000026313D5000157D98F93F7F70FB71C18
:1018600000402382FC0411472303E4801305F00F9A
:1018700097000000E78000E8094C97000000E7802F
:1018800080E863657C15B7050700DA9537870700A0
:10189000795563FEE504B3879500636AF704370B57
:1018A0000800A94733EB65016395F90881E8814495
:1018B00097000000E78020E5268515A8DA85094510
:1018C00097000000E780C0E605090345F9FFFD1415
:1018D000050B97000000E780C0E481C49377FB0FFD
:1018E000E5F797000000E780A0EA69F17D55B7179A
:1018F0000040130770052380E704130780FA238054
:10190000E70403C74704418B2382E704F250B7E79B
:1019100000E023A0571123A24711E2543244525948
:10192000C259325AA25A125B825B724CE24C21615C
:101930008280A547639BF90685691309F00FB306FA
:101940009900B3742B01B6941349F9FFB37499004D
:10195000856B33796901416B9387F9FFB3F72701F1
:1019600099E363FC340193D94900C147E3E637FFAB
:101970003DBF0569C1697D19D9B71305800D63881D
:101980006901130500026384790113051008CA85F3
:1019900097000000E780C0D997000000E78040DF93
:1019A00031D54E99B38434416DBFDA852D4597000A
:1019B0000000E780E0D7CA94E30B99EE0509970091
:1019C0000000E78020D5A30FA9FEFDB79387F9FF9C
:1019D00093F7F70F636DFC0C83C71C0413073008E3
:1019E0006315F706370708006361EB06B3079B0032
:1019F000B706100063FBD704334BEB0089476399AC
:101A0000F9068980D549E38404EADA850945970017
:101A10000000E780E0D111090327C9FF9147232087
:101A2000E48003076480E34E07FE23033481FD173F
:101A3000EDFBFD14110B81C49377FB0FE9FF9700B9
:101A40000000E780E0D461F155B5B717004003C747
:101A50005704B70708001377070219E3B787070091
:101A60007955E376FBE833079B00E3F9E7F841B5E6
:101A70008547E380F9F0DA852D4597000000E7807F
:101A800020CB9389F4FFE38404E297000000E78011
:101A900060C893F7390091EB83260480032709007F
:101AA00093074900E396E6E03E89CE84D9BFB54767
:101AB0006399F9001305900B97000000E78080C33D
:101AC000FDB3B1471305B00AE388F9FE9947639760
:101AD000F904B7050800B365BB002D459700000069
:101AE000E78000C581448D4BA14997000000E78045
:101AF00060C263967401832704802320F900850463
:101B0000E39534FF8327048013172B0163550700E7
:101B10002312F90069BB2322F90051BB9D47639F43
:101B2000F90281451305B00497000000E78040C02A
:101B3000BD442320090023220900FD59970000001D
:101B4000E78040BD93F77400CA9703C70700FD14F0
:101B5000398D2380A700E39334FF91BBA14763979E
:101B6000F90697000000E780A0C28144630D0B00D6
:101B70008D479304C0036308FB00930400056304CE
:101B80008B01930440041375C507E30295D21945F0
:101B900097000000E78000B697000000E780A0B63D
:101BA000054597000000E780E0B426859700000017
:101BB000E78020B7094597000000E78080B69700CE
:101BC0000000E780E0BCE31405CE0DB39147639FAE
:101BD000F9001305600697000000E780A0B19700A8
:101BE0000000E78040B213059009F9B5E38109CC04
:101BF000F1547DB9BD660147173600001306063063
:101C0000938606A685458347060093F7F70F91C391
:101C100082800507E3F9E6FE973700002380B72EA0
:101C2000DDB77D166206618693178601E18763D46E
:101C3000070001458280931726003307F500AE9711
:101C400018439C4363E7E7007D16E37FF7FC7D556F
:101C5000828005458280FD15E205E18513978501A7
:101C6000618793F7F50F63480700FD15139725006B
:101C70002A97584365D713851700620561858280CE
:101C80003308B5021C4283A80600B335B502C297DB
:101C900033B50701AE98469585486367B5006394F0
:101CA000A50063E3070181480C43C6950CC388C2B5
:101CB0001CC2828081471397870161876343B70005
:101CC0008280139727002A97232007008507E5B70E
:101CD0008147014793968701E18663C5B6001335B6
:101CE0001700828093962700AA9694428507558F05
:101CF000D5B793D755408A07AA979C430545331516
:101D0000B5007D8D828017F3FFDFE702833D2A84D3
:101D100097000000E78060F405C5931725003E9406
:101D20000327C4FF814711EB7D1516053E9542053B
:101D3000418517F3FFDF6700033D05838507E5B79E
:101D40000145C5BF81471397870161876343C7007A
:101D5000828013972700B386E50094422A9785076F
:101D600014C3D5B77D1662066186014793178601B5
:101D7000E18763D50700133517008280931726008B
:101D8000B306F500AE9794429C437D16B58F5D8FE8
:101D9000F1BF8A05AA9501476363B500828083A6D7
:101DA000C5FFF11593D71600D98F9CC11397F60183
:101DB000E5B72A830148014701456343D700828084
:101DC000B387050183A80700B30706019C43C697A4
:101DD000AA976384F80033B517010507B308030118
:101DE000620723A0F80061871108C1BF2A83014759
:101DF0008147014563C3D70082803388E50083288B
:101E00000800330EE600032E0E003388A840330886
:101E1000C8416384080133B508018507B308E300AE
:101E2000E20723A00801E1871107E9B717F3FFDFF5
:101E3000E702232B0111B286B2842E86AA850A8579
:101E400097000000E780C0FA2A84A6850A859700DB
:101E50000000E78020E833348000060413351500C5
:101E6000018D056117F3FFDF6700E32917F3FFDF3B
:101E7000E702A3244111AA89AE8A328BB68402C23A
:101E800002C402C60144131C8401135C8C416349E3
:101E90009C02939B1400FD1B0549138CF4FFF15C1D
:101EA00033048901620461846340740792478E049D
:101EB000CE9423AEF4FE410117F3FFDF67006323E6
:101EC00013192400B30B2B01014A93172A00D6974C
:101ED00083A50B0088437800340050009700000071
:101EE000E78040DA050A93178A01E187F11BE35E78
:101EF000FCFC92474E9905042320F900A2473EC2FC
:101F0000B24702C63EC441B7131A8901135A8A4127
:101F1000131D240093178A01E18763CF970092472E
:101F20000A044E941CC0A24705091379F90F3EC25A
:101F3000B24702C63EC4ADB7B3079A0313152A00D1
:101F400056950841780034005000050AEA97DA9760
:101F50008C4397000000E780E0D26DBF197106C284
:101F600012C416C61AC81ECA22CC26CE2AD02ED219
:101F700032D436D63AD83EDA42DC46DECAC0CEC2C9
:101F8000D2C4D6C6DAC8DECAE2CCE6CEEAD0EED2F9
:101F9000F2D4F6D6FAD8FEDA971500009385058CB0
:101FA0008841E700050092402242B2424243D243B8
:101FB0006244F244025592552256B2564257D257C5
:101FC0006258F25806499649264AB64A464BD64BBD
:101FD000664CF64C065D965D265EB65E465FD65F45
:101FE0000961730020300000972100209381810156
:101FF000175100201301018117F5FFFF1305C500DC
:102000009705002093850500171600201306C6FDCE
:1020100063FAC5008322050023A055001105910530
:10202000E3EAC5FE170502001305855B971500203E
:102030009385C5FB171600201306C66563FAC50015
:102040008322050023A0550011059105E3EAC5FE92
:102050001715002013050564974500209385053664
:102060006377B500232005001105E36DB5FEFD4241
:10207000739002BC8D4273904280B722000093821D
:10208000828873900230970200209382A2F793E235
:1020900032007390523097520000938242AD739099
:1020A00012346FB0F47573002030397101436EC67D
:1020B00019A0397141536AC866CA62CC5ECE19A0B4
:1020C000397101535AD056D252D44ED64AD826DA54
:1020D00022DC06DE33016140828241114AC026C201
:1020E00022C406C68282B24D4101024D924C224C5E
:1020F000B24B4101024B924A224AB2494101024984
:1021000092442244B240410182803D432A87637356
:10211000C3029377F700BDEFADE5937606FF3D8AE6
:10212000BA960CC34CC30CC74CC74107E36BD7FE30
:1021300011E28280B306C3408A0697020000969699
:102140006780A6002307B700A306B7002306B700E1
:10215000A305B7002305B700A304B7002304B70005
:10216000A303B7002303B700A302B7002302B700FD
:10217000A301B7002301B700A300B7002300B700F5
:10218000828093F5F50F93968500D58D9396050182
:10219000D58D61B7939627009702000096968682A8
:1021A000E78086FA9680C1171D8F3E96E374C3F8C8
:1021B000A5B73367B500FD530D8B79E7B7877F7FF0
:1021C0009387F7F710419441B372F6003363F6003A
:1021D000BE92B3E262006397720C6318D606504158
:1021E000D441B372F6003363F600BE92B3E26200EC
:1021F0006398720A631BD60410459445B372F600C7
:102200003363F600BE92B3E262006391720A631E0A
:10221000D6025045D445B372F6003363F600BE9241
:10222000B3E26200639A72086311D60210499449BE
:10223000B372F6003363F600BE92B3E262006393BA
:1022400072085105D105E30FD6F6131706019397CF
:102250000601631CF7001357060193D706013305E7
:10226000F7409375F50F91E982804183C18333056F
:10227000F7409375F50F91E182801377F70F93F78D
:10228000F70F3305F74082800346050083C605003B
:10229000050585056313D60065FA3305D6408280AF
:1022A00011059105E312D6FE014582802105A105A5
:1022B000E31CD6FC014582803105B105E316D6FC4E
:1022C000014582804105C105E310D6FC01458280AD
:1022D000B717004003C777051377E70FA38BE70411
:1022E000130700F8A38DE7043D47238CE704130789
:1022F0005003A38CE70403C7A7051377D70F238DDB
:10230000E7048280B717004003C7E7020D89411137
:102310001377C70F498F93068008F3B6068093F6AC
:10232000860836C601000100930670052380D70495
:10233000930680FA2380D704010001002387E70277
:1023400023800704B247F3A7078001000100410181
:10235000828041112A83014E930E407E130F001993
:10236000930F400663E56E129308001913034006AD
:10237000B3781503854E0D4FA14F337365020D8958
:102380001335150063EFBE121308F6FF79467298F5
:102390004208135808013307C70213D61700BE07B7
:1023A00032976146B3F6C60213068070B386C60242
:1023B0003697A166F58F42075D8FB716004083C739
:1023C000F60293F70708A303F1000346710083C7E1
:1023D000F60293F70708E394C7FE83477100B71628
:1023E000004093F7F70F6388071293078008F3B74D
:1023F000078093F787083EC401000100B71700402B
:10240000930670052380D704930680FA2380D704AF
:102410000100010023AA070383C6170393E60608F9
:10242000A388D70223800704A247F3A707800100EF
:1024300001001166B71700407D16D45BC85F938515
:102440004703A98EF18EF5FA93068008F3B606804D
:1024500093F6860836C601000100930670052380B6
:10246000D704930680FA2380D7040100010098C1A5
:1024700003C7170313670704A388E7022380070431
:10248000B247F3A7078001000100410182807D135C
:102490003368E3039308E016630E08003368F30320
:1024A0009308D016630808009378330093B8180097
:1024B0009388D81633081E01131E0801135E0E01FF
:1024C00055B56393E5030548638608000148630337
:1024D00003002A8871087298FD15131E0801C205B1
:1024E000135E0E01C18179BD13F8150063F4BF00BE
:1024F0007908D5B713381800E5BF83C7F60293F7FC
:102500000708A303F1000346710083C7F60293F79F
:102510000708E394C7FE8347710093F7F70FF1DFD5
:10252000E9B531714AD966CB06DF22DD26DB4ED70D
:1025300052D556D35AD15ECF62CD6AC96EC7AA8C26
:1025400002D897100000E78020B12A8993078008FD
:10255000F3B7078093F787083EDA01000100B71749
:102560000040130770052380E704130780FA2380D7
:10257000E7040100010003C7F7021377770FA38771
:10258000E70203C7F70213678700A387E7022380E8
:102590000704D257F3A70780010001000545970003
:1025A0000000E78060D6130780C13347E902116A53
:1025B00093070AE893065002BD69930BA004814A71
:1025C000014B13048008930470057D1AB347F90288
:1025D0003307D7023EC0FD873ECC938709A69309F7
:1025E000803E3347F7023AC27D873AC43347390306
:1025F0008549B399990193D93940B306D702B30BF2
:102600007703B3C6F602B3CBFB0236C6FD8636C8E7
:1026100093D6FB4136CEB7460F0093860624334946
:10262000D9028566938606FAB3969601B389E902C4
:10263000130760553309D90293060010B389E902E4
:102640003349D902B3C9F9029316390036CA37198A
:102650000040FD8636D0930D090493D7F9413ED250
:10266000F336048093F6860836DC010001009307F8
:1026700070052380FD00930680FA2380DD000100B1
:1026800001008346390593F6860FA309D9048346D2
:10269000390593E61600A309D90423800D00E256FC
:1026A000F3A6068001000100130C80FA116DF336C9
:1026B000048093F6860836DE01000100930770055A
:1026C0002380FD0023808D01010001008346390530
:1026D000216693E60602A309D90483560905B3E6E9
:1026E000A6012318D90483560905D18E2318D904CD
:1026F00023800D00F256F3A60680010001008346F8
:10270000390593F606026381061A03463905218AC4
:102710006DDE081897100000E7800098733604807B
:1027200013768608B2C20100010023809D00238039
:102730008D0101000100B717004003C6370513766D
:10274000F60DA389C70403C6370513660602A389DD
:10275000C704835609052166B3E6A6012318D904E8
:1027600083560905D18E2318D90423800D0096467F
:10277000F3A60680010001008346390593F60602A0
:10278000638B061483463905A18AEDFE970000206D
:10279000E7806090AA8636D497000020E780A08F5B
:1027A000A256E30AD5FE835609054255B3E6A601B3
:1027B0002318D90497100000E780C08F834639059D
:1027C000A18AEDDE03560905834629058247337643
:1027D000CA00B306DA0293D5F641B296B388F64042
:1027E000E24733B8C6002E983308F840A247B3B684
:1027F00016013308D84063C70701631DF8009247EC
:1028000063FA1701C247634FF80E63950701B24799
:1028100063EAF80E894663E9660FF24693151800DD
:1028200013D3F8015E8613951800B365B30042D642
:1028300046D497C00100E780003B3258050B137B5C
:10284000FB0F63470001631A0838A25863870838F2
:1028500013081500B336A800B69513D6F5013298C3
:10286000B336C800AE9613581800FE06B3E606014C
:102870007336048013768608B2C6010001002380F7
:102880009D0023808D01010001000356C902B2960C
:10289000C206C1822316D90223800D00B646F3A6D4
:1028A00006800100010021B5F336048093F6860806
:1028B000B6C00100010023809D0023808D0101002E
:1028C00001008346390593E60602A309D904238053
:1028D0000D0086460DB5F336048093F68608B6C41F
:1028E0000100010023809D0023808D010100010073
:1028F0008346390593E60602A309D90423800D0017
:10290000A646BDB5E30B0BF0F336048093F68608BC
:10291000B6C801000100930680FA23809D00238041
:10292000DD00010001008346390593F5FC0F93F6A5
:10293000860FA309D90483463905CD8EA309D9048E
:1029400023800D00C646F3A6068001000100130592
:1029500080FA03463905930639051D8A631C9629BA
:102960007336048013768608B2CC0100010013068A
:1029700080FA23809D002380CD000100010003C662
:1029800006001376F60D2380C60003C60600136604
:1029900006022380C600835609051166D18E2318CE
:1029A000D904835609052166D18E2318D9042380C2
:1029B0000D00E646F3A6068001000100130680FA2A
:1029C0008346390593F60602638006268346390559
:1029D000130C3905A18AFDDA081897000000E7807A
:1029E000A06BF336048093F68608B6D00100010090
:1029F000930680FA23809D002380DD000100010002
:102A000083460C00116693F6F60D2300DC00834626
:102A10000C0093E606022300DC0083560905D18EE4
:102A20002318D904835609052166D18E2318D904A9
:102A300023800D008656F3A60680010001001306D0
:102A400080FA8346390593F60602638A0620834698
:102A50003905A18AEDFE97F0FF1FE780C0632A8C3D
:102A600097F0FF1FE7802063E30C85FF835609057D
:102A700011664255D18E2318D90497000000E780D3
:102A800060638346390513063905A18AFDDAF336FA
:102A9000048093F68608B6D401000100930680FAFC
:102AA00023809D002380DD00010001008346060095
:102AB00093F6F60D2300D60023800D00A656F3A64C
:102AC0000680010001008356090503462905D24707
:102AD000B376DA003306CA021305800C9355F6412B
:102AE0003696330DF6408257333CD6002E9C333653
:102AF000A601330CFC40330CCC40330885039256BE
:102B00004E86B335A5033305A503C29597C00100D2
:102B1000E780600D63468001631E0C16630C0D1682
:102B2000130615003335A6002E959356F5013696FB
:102B3000B335D600AA959396F50105828585D18E89
:102B40006346B000639D051A638B061A0356C902DB
:102B500015823305D6003336C500B2956348B00000
:102B6000639105241306F00F637DA622894663F363
:102B7000561593078008F3B7078093F78708BED6EA
:102B80000100010037170040930770052300F70488
:102B9000930780FA2300F704010001008356C7025F
:102BA00089678117D58FC207C1832316F7022300D7
:102BB0000704B657F3A7078001000100FA506A54D2
:102BC000DA544A59BA592A5A9A5A0A5BFA4B6A4C49
:102BD000DA4C4A4DBA4D296182801308F5FF33352E
:102BE000A800FD152E951356F5013298B336C8008E
:102BF000AA9695B9F336048093F68608B6CA010002
:102C0000010023809D002380AD0001000100834668
:102C10003905CD8EA309D90423800D00D646F3A62D
:102C200006800100010035B3F336048093F6860870
:102C3000B6CE0100010023809D002380CD0001005D
:102C400001008346390593E60602A309D9042380CF
:102C50000D00F646F3A606800100010095B3F33699
:102C6000048093F68608B6D20100010023809D00FF
:102C70002380CD00010001008346390593E606025A
:102C8000A309D90423800D009656F3A606800100FF
:102C9000010045BB9306F5FF33B5A600FD152E9543
:102CA0009355F501AE96B3B5B600AA951396F50106
:102CB000858269B5F336048093F68608B6D801009C
:102CC0000100930680FA23809D002380DD0001002F
:102CD00001008356C9020566011693F6F60FD18EE0
:102CE000C206C1822316D90223800D00C656F3A660
:102CF000068001000100850A93FAFA0F95B233E6C7
:102D0000B60045C20356C9023305D0403338A0008F
:102D1000B305B040B385054115826345B000D1E1EC
:102D20006371A608894663F0560593078008F3B7D8
:102D3000078093F78708BEDA01000100B71700404B
:102D4000130770052380E704130780FA2380E70444
:102D50000100010003D7C7027D8B2396E702238081
:102D60000704D65781BDF336048093F68608B6DC97
:102D700001000100930680FA23809D002380DD007E
:102D8000010001008356C9020566011693F6F60F8D
:102D9000D18EC206C1822316D90223800D00E656C9
:102DA000B9B793078008F3B7078093F78708BEDEAB
:102DB0000100010037170040930770052300F70456
:102DC000930780FA2300F704010001000356C702AD
:102DD00093975600B297C207C1832316F7022300C8
:102DE0000704F657C1BB914763EEB70217D701003E
:102DF0001307C77D8A05BA959C41BA978287B71792
:102E0000004003A7470B1345F5FF698F23AAE70A84
:102E100003A7070B698F23A8E70A03A7070A798D81
:102E200023A0A70A8280B717004083A6470B134749
:102E3000F5FFF98E23AAD70A83A6070B558D23A881
:102E4000A70A83A6070A758F23A0E70A8280B7170F
:102E5000004003A7470B498F23AAE70A03A7070BE4
:102E60001345F5FF45BFB717004083A6470B13472F
:102E7000F5FF758F23AAE70A03A7070A598D4DB7F7
:102E8000B717004003A7470B498FEDB7914763EE93
:102E9000B70217D701001307A7748A05BA959C419A
:102EA000BA978287B717004003A7470D1345F5FF70
:102EB000698F23AAE70C03A7070D698F23A8E70CE6
:102EC00003A7070C798D23A0A70C8280B7170040B9
:102ED00083A6470D1347F5FFF98E23AAD70C83A6C7
:102EE000070D558D23A8A70C83A6070C758F23A06B
:102EF000E70C8280B717004003A7470D498F23AA2C
:102F0000E70C03A7070D1345F5FF45BFB7170040B2
:102F100083A6470D1347F5FF758F23AAE70C03A778
:102F2000070C598D4DB7B717004003A7470D498FC0
:102F3000EDB7797122D43714004026D24AD0035914
:102F400024028354040206D64209C2044ECE52CC57
:102F500056CA13590901C1802DE11379F9F793F489
:102F6000F49F4209C20413590901C18093078008E4
:102F7000F3B7078093F787083EC401000100930769
:102F800070052300F404930780FA2300F404010081
:102F90000100231124032310940223000404A247F8
:102FA000F3A7078001000100B25022549254025945
:102FB000F249624AD24A45618280B7F507008146EC
:102FC0003000B105194597000020E7808081A247B5
:102FD00013972701E34A07FC1369090893E40440A7
:102FE00093098008F3B7098093F787083EC0010072
:102FF0000100930A700523005405130A80FA230088
:10300000440501000100231124032310940223002E
:1030100004048247F3A7078001000100294597F0C7
:10302000FF1FE7802031F3B9098093F989084EC268
:1030300001000100230054052300440501000100A4
:103040008357040293E707202310F40223000404AB
:103050009247B9B7B7170040884742054181937737
:10306000050491EB9377F5013755E80113050580C9
:103070003345F50282809377050C130700046397AC
:10308000E7009377F50137459C1CCDB72165130503
:1030900005D0828037E700E01C435443A183E20659
:1030A000D58F1CC1FD572320F7182322F7188280E3
:1030B00013178500B7E700E023A0E710618123A282
:1030C000A7108280B7F700E08847CC47828081470D
:1030D00037370040A14663C4C7003285828003456C
:1030E000B740E38EA6FE3385F5000345050085074E
:1030F0002304A740CDB797070020938727EF9C4371
:10310000173700201307872B3E95636EE5001737AE
:1031100000201307273F6368A70017070020232715
:10312000A7EC3E858280FD57EDBF8280411122C40D
:1031300006C62A8497000000E78000F22947B307FB
:10314000E502B2408D83B3D7870222449507B3D7F7
:10315000E70237370040C207C1832316F700410159
:103160008280411137150E0006C697000000E780E7
:1031700020FCB7370040130770F82381E7000D47A4
:10318000A381E70013070004A380E7000547238716
:10319000E700B24041018280373700408347270073
:1031A0001A0593F7F703C98F93F7F70F2301F70079
:1031B0008280B737004003C7170019C9D98DA38093
:1031C000B70003C70700136787002380E7008280EA
:1031D00093C5F5FFF98DA380B7008280AE872A875B
:1031E000B736004021463738004089E71703000012
:1031F0006700E3F383C8B600E30916FF05078348B9
:10320000F7FFFD17C20723041801C183F9BF41115D
:1032100022C406C62A8497000000E780E0E329471D
:10322000B307E502B2408D83B3D7870222449507E6
:10323000B3D7E70237370040C207C1832316F740F0
:1032400041018280716541111305052006C6970072
:103250000000E78000FCB7370040130770F82381B7
:10326000E7400D47A381E74013070004A380E74030
:1032700005472387E740B24041018280CC4141119C
:1032800006C6328503C6150083C5050022064D8E8D
:1032900042068D654186138875A2630C0611634B47
:1032A000C804138845A26300060D634AC8009385CD
:1032B00035A26301B6082390060029464DA0138865
:1032C00055A26305060D938565A2E316B6FE8D45EE
:1032D0001D4663E6E5081146198E63F3C7003E8676
:1032E000B7E704002390C600FC4797D501009385FB
:1032F00065319DA0138895A263030611634E060DE8
:103300001388A5A263000613938505A5E315B6FAF5
:1033100099451D4663E5E504198E63F3C7003E86B3
:10332000B7E704002390C600FC479705002093856B
:1033300025D61DA09D451D4663E3E5022146198E55
:1033400063F3C7003E86B7E70400FC472390C6003E
:103350009705002093858534BA9582970146B2403F
:10336000328541018280AD451D46E3EAE5FE3146E6
:10337000198E63F3C7003E86B7E704002390C600AA
:10338000FC4797D501009385652AF9B7B1451D46DD
:10339000E3E7E5FC3546198E63F3C7003E86B7E7E1
:1033A00004002390C600FC4797D5010093850529AA
:1033B00065B78D451D46E3E4E5FA1146198E63F3C2
:1033C000C7003E86B7E704002390C600FC4797D5A8
:1033D00001009385E52349B78D451D46E3E1E5F8F6
:1033E0001146198E63F3C7003E86B7E704002390A9
:1033F000C600FC4797D5010093850526B1BFA545BA
:103400001D46E3EEE5F42946198E63F3C7003E86B8
:10341000B7E704002390C600FC4797D501009385C9
:10342000E51F1DBFB5451D46E3EBE5F23946198E94
:1034300063F3C7003E86B7E704002390C600FC474D
:1034400097D501009385051B01BFB7E7040003A3CF
:103450000713970600209386A6C24146A545170587
:1034600000201305E5B802832D455DE703C505007F
:103470000947631FE50803A84500411106C6034735
:10348000180032850346080022074168518F9308CF
:1034900028FE6307170563E9E800051863030703BF
:1034A00023900600294591A8130648FE630AC70425
:1034B0001518E31707FF15463E87637BF60015478F
:1034C00001A8130600023E876374F600130700028A
:1034D000B7E704002390E600FC471316070111A884
:1034E0003E8691C30546B7E70400FC472390C6001B
:1034F0004206CC45418282970145B240410182801B
:10350000130600083E87E375F6FC13070008C9B7E9
:103510002390060005458280828041677917630405
:10352000E504411122C406C685472A84639FF5003D
:10353000B7E7040022852244B24003A3871397050E
:1035400000209385E52F4101028389476399F500A7
:10355000B7E7040083A7070B8545829771D9B2406E
:103560002244410182808280797126D252CCAE847D
:103570002A8A97D501009385251017D501001305D8
:10358000251206D63AC622D44AD0368432894ECE87
:1035900097C00100E78060B0A28517D50100130530
:1035A000251197C00100E78040AF294597C0010071
:1035B000E78080B383C7840093F70702F9E383C9E8
:1035C00004008947054532476396F908D44083C70C
:1035D000160083C60600A207D58FC166138616FEA5
:1035E000638CC7028D16638FD7068D6693862690EF
:1035F00029456391D706B7E70400A286225403A3A6
:103600004714B250F2494A86A6850259925452850F
:10361000624A8547456102832D450DEF93070002FD
:10362000354563E98702B7E70400FC47C844130641
:103630000002CA8582978149970700209387072156
:103640009C43014581CB9C4391C74E852286CA8508
:1036500082970145B250225492540259F249624A6B
:10366000456182802D457DF79307700F3545E3E373
:1036700087FEB7E70400FC47C8442286CA858297C4
:1036800065BF2145C1BF411122C437E4040083272F
:10369000841326C2AA84416506C697050020938537
:1036A000251A7D1582978327C40A17050000130584
:1036B00005E78588829795C0032304132244B2400E
:1036C000924497060020938626AE4146C5451705CD
:1036D00000201305659C41010283B24022449244BC
:1036E00001454101828019C59707002023A0A71634
:1036F00001458280454582801147636AA70A97D6B3
:103700000100938626F60A0536951841411106C632
:103710003697AE87B2850287130700026145639D25
:10372000E700B7E70400FC47130600021705002076
:10373000130545F782970145B24041018280054754
:103740006145E39BE7FEB7E70400FC470546170524
:103750000020130525F7F9BF1307700F6145E39D9E
:10376000E7FCB7E70400FC471306700F17050020BD
:10377000130585F5C1B7130700086145E39EE7FA15
:10378000B7E70400FC4713060008170500201305DF
:1037900025034DB715476145E390E7FAB7E7040005
:1037A000FC471546170500201305C50961B70945F3
:1037B0008280411126C2B7E4040083A7C41322C447
:1037C0004AC006C62E8497050020938565072A897E
:1037D0008297058905C5970700209387E78B83D7D4
:1037E000A70BA28503A3440D2310F4002244B2408A
:1037F00092444A850249014641010283B240224473
:103800009244024949454101828097070020238163
:1038100007049707002023AF0702B717004003A74C
:10382000070CB706C0FFFD16758F23A0E70C03A792
:10383000070DB7064000558F23A8E70C03A7070C18
:103840003D9B23A0E70C03A7070D1367070123A8DF
:10385000E70C8280B717004003A5470C83A7470CED
:10386000598113451500C18B058999E3136525001E
:103870009707002083C7C7FD6380A7029707002032
:103880002388A7FC11C9970700209387A7FC03A3EF
:1038900007006303030002838280114517F3FFFFD3
:1038A000670063C8011122CC06CE3714004026CA37
:1038B0004AC84EC652C483447405034AB4058349BA
:1038C00084050349940597F0FFFFE780A0A0834794
:1038D000A40593F4F40F137AFA0F93E71700230D5E
:1038E000F40493F9F90F1379F90FB717004003C7E0
:1038F000A705058B6DFF03D5C705A38D4705238C51
:103900003705A38C2705A38B9704F2406244D24469
:103910004249B249224A05618280411193970501CB
:1039200022C406C626C2C1872E8463DC0700B7E422
:103930000400FC54829719C1BC5482972165218DE3
:1039400015A893F7150013C515008DE793F725000B
:103950009DC797000000E78020F0B7E70400BC4F48
:103960001306000A894517050020034525EF8297B5
:1039700013452400B240224492444101828093972F
:10398000250163D80702B7E4040083A7C41E829709
:1039900097000000E780A0F0BC4C375607001306E4
:1039A0000630896517050020034545EB82970965B8
:1039B00079B7939715010145E3DE07FA17D50100A2
:1039C000130505D797C00100E7800085B7E704001D
:1039D000BC4F13060064916517050020034505E8F8
:1039E00082971165A9BF1D71A2CC37E404005C5C0D
:1039F000485886CE494697D501009385E5CE8297F3
:103A000011E917D50100130565CF97C00100E780C4
:103A1000A08001A0B7F600E0795798CAFD57DCCA2C
:103A20000567B7E700E023A0E7101306F00290C295
:103A300023A0E718010001003707002018471306EC
:103A4000000481459706002023A8E6E04157A38A99
:103A5000E7403C4408088297970700209387077C3B
:103A60003EC8856713870740938757D1231AE10023
:103A70002312F1021307B00F97F7FFFF9387C76474
:103A80002310E1023ED81547970700009387C7E14E
:103A9000B7F50700A30FE1003EDC054797070000DC
:103AA0009387E7DF81463000E10519452301E102F4
:103AB0003EDE97F0FF1FE780C0D218088147994685
:103AC00030003E960346060085070507A30BC70096
:103AD000E398D7FEC24791C70357410185676373D7
:103AE000F70001A0B7E7040083A7470A08088297F8
:103AF000AA8511C917D50100130585C197B001002A
:103B0000E780A05901A0F6406644256182804111FA
:103B100026C2B7E4040083A7040806C622C417051A
:103B200000001305C5DF829717040020130404D397
:103B30002300A40097000000E780800297000000A7
:103B4000E780E0CC03450400224403A38405B2408F
:103B5000924413060032896541010283797106D6C9
:103B600022D413078008F337078093F787083EC2F3
:103B700001000100B7170040930570052380B704CA
:103B8000130680FA2380C7040100010083C6F702F0
:103B900093F6A60FA387D702238007049246F3A6C5
:103BA00006800100010073370780137787083AC445
:103BB000010001002380B7042380C7040100010035
:103BC00003C7F70213672700A387E70223800704D0
:103BD000A247F3A7078001000100054597E0FFFF1A
:103BE000E780807297000000E78060CB0147814644
:103BF0008147054685451305407E97E0FFFFE78036
:103C0000807537E404003C44680051468145829742
:103C1000B707C0A83EC8B787E803938707D03ECA56
:103C200097E7FF1F9387A7793EC67C586800829765
:103C3000B250225445618280411197D5010093858D
:103C4000651117D501001305A5A506C697B001009B
:103C5000E780A04417D501001305852797B0010020
:103C6000E780A043B2402945410117B30100670036
:103C7000A347411197D501009385050F17D5010082
:103C8000130505A206C697B00100E780004117D5CD
:103C900001001305A52297B00100E7800040B24063
:103CA0002945410117B3010067000344411122C4B3
:103CB00006C6834705002A849DC797D501009385D2
:103CC000651017D501001305A59D97B00100E78089
:103CD000C03C4C4017D501001305453897B0010092
:103CE000E780A03B3DA058410DEF97D5010093859B
:103CF000650D17D501001305A59A97B00100E7805F
:103D0000C03917D501001305E53697B00100E780EB
:103D1000C0382244B2402945410117B30100670071
:103D2000A33CA1679386D7036313D70297D50100FD
:103D30009385450917D501001305859697B00100B5
:103D4000E780A03517D501001305C5337DBFED070A
:103D500097D501009385050717D5010013054594F4
:103D6000631BF70097B00100E780203317D50100EF
:103D70001305853259BF97B00100E78000324C40EF
:103D800017D501001305453391BF411197D50100A7
:103D90009385C5FE17D501001305859006C697B01B
:103DA0000100E780802FB2402945410117B301008F
:103DB00067008333397122DC26DA4AD82E842A89B7
:103DC0008145B2844808714636C606DE97E0FFFF9B
:103DD000E780E03397F7FF1F9387075EDC4783D7C1
:103DE0000700231C2101231BF10097500000E780EE
:103DF000E046B246230DA10091E2854693070019E3
:103E00003ECE2686FD57A2854808A30DD100230289
:103E1000F10297500000E7804047F2506254D254BC
:103E20004259216182808546170300006700C3F86C
:103E30004111814617F6FF1F1306465585451705A4
:103E400000200355252306C697D00000E780A096E2
:103E500015C997D501009385A5F517D50100130560
:103E6000258497B00100E780402317D50100130592
:103E7000E51A97B00100E7804022294597B001007C
:103E8000E780802697D50100938585F217D501003C
:103E90001305058197B00100E780202017D50100A8
:103EA0001305051997B00100E780201F294597B039
:103EB0000100E780602397F7FF1F9387E74FDC47F8
:103EC000054797D501009385A5EE2390E70017C518
:103ED00001001305E57C97B00100E780001C17D5B1
:103EE00001001305251697B00100E780001BB240C2
:103EF0002945410117B301006700031F011122CCBE
:103F000006CE26CA4AC84EC693F715002E84B5CBF6
:103F100097000000E78000F2930710F817070020D1
:103F20002302F7209707002083D787141707002064
:103F3000A30AF71E9145A183170500201305851ECE
:103F4000170700202301F71E97070020A38D071CE9
:103F500097600000E780C0F1B7E70400BC4F13068C
:103F6000001493050010170500200345A58F8297C4
:103F700013451400F2406244D2444249B2490561FB
:103F8000828093F70510B1C3054597600000E78074
:103F900020F7171500200355C57897600000E780CB
:103FA000A0C297200000E780205E9707002083C70B
:103FB000B72689E797600000E780C0189760000087
:103FC000E780001A1345041075B793F72500E9CF71
:103FD000170700200357871369C7AD64B71900405E
:103FE0009384A4AA23A099009706002093864612E2
:103FF000944297D7010093872714170600200346A1
:104000000611814517D5010013050514978000009E
:10401000E780E09623A0990097F7FF1F2392A72A35
:104020002A8941C197D50100938545DF17C5010055
:104030001305056797B00100E7802006CA8517C5FC
:1040400001001305A57D97B00100E7800005294513
:1040500097B00100E7804009970700202398070ADE
:10406000930710F817070020230EF70A9707002080
:1040700083D7070017070020A306F70AA1831707B5
:1040800000202302F70A91458D47170500201305EC
:10409000650917070020A308F70897600000E7806C
:1040A00020DD13452400F9B593F74500D1C397D51A
:1040B00001009385A5D617C501001305655E97B06D
:1040C0000100E78080FD17C501001305E57697B074
:1040D0000100E78080FC294597B00100E780C0001F
:1040E000930720F817070020230EF70297070020F8
:1040F00083D747FA17070020A306F702A183170703
:1041000000202302F702854717070020A30DF700C0
:1041100097500000E780802B1705002013058500CD
:10412000914597600000E780A0D41345440099B5FD
:1041300093F78500A9C797D50100938525CE17C5AC
:1041400001001305E55597B00100E78000F517C59C
:1041500001001305A56F97B00100E78000F4294521
:1041600097B00100E78040F897070020239007FAF6
:1041700097800000E780809013458400E5BB93F7AB
:104180000501D1C38545170500200355A5F09760AB
:104190000100E780804597D50100938525C817C5A4
:1041A00001001305E54F97B00100E78000EF17C548
:1041B00001001305E56A97B00100E78000EE29458C
:1041C00097B00100E78040F2930730F8170700200E
:1041D000230AF7F49707002083D7C7EB17070020BF
:1041E000A302F7F4170500201305C5F3A1838D453D
:1041F000170700202309F7F297600000E78040C707
:104200001345040185BB93F70502D1C797D501007B
:104210009385C5C017C501001305854897B00100F7
:10422000E780A0E717C501001305C56597B0010039
:10423000E780A0E6294597B00100E780E0EA930710
:1042400040F817070020230FF7EC9707002083D7CB
:10425000A7E217070020A307F7ECA18317070020A8
:104260002303F7EC854717070020A30EF7EA97070B
:104270000020239307E097500000E78020151705E2
:104280000020130525EA914597600000E78040BEB5
:1042900013450402C5B193F70504FDC397D501008A
:1042A0009385C5B717C501001305853F97B0010079
:1042B000E780A0DE17C501001305455E97B0010039
:1042C000E780A0DD294597B00100E780E0E197078E
:1042D000002083C727E51307700A6386E7061307E4
:1042E000800A638CE7081307600A6393E704930767
:1042F00060F8170700202307F7E29707002083D70D
:10430000C7E017070020A30FF7E0A18317070020DD
:10431000230BF7E0854717070020A30AF7E0B14514
:1043200017050020130505E097600000E78040B402
:1043300097500000E7808009134504049707002088
:10434000239507DC05B9930770F817070020230BA6
:10435000F7DC9707002083D747DB17070020A3036C
:10436000F7DCA18317070020230FF7DA854717072B
:104370000020A30BF7DA994565B7930780F8F1B7EA
:1043800093F705080145E38707BE97D5010093859C
:10439000E5A817C501001305A53097B00100E78017
:1043A000C0CF17C501001305E55097B00100E780A5
:1043B000C0CE294597B00100E78000D39307A0F84D
:1043C000170700202300F7D69707002083D787D44C
:1043D00017070020A308F7D4A183170700202304A0
:1043E000F7D4854717070020A30FF7D297070020BF
:1043F000239207D297500000E78040FD1705002068
:10440000130545D2914597600000E78060A61345EB
:1044100004088DB6411122C497D501009385C59B30
:104420002A8417C501001305A52706C697B0010009
:10443000E780A0C64C4017D501001305A5BB97B077
:104440000100E78080C5294597B00100E780C0C919
:10445000034704009307F00F631FF70297D501008D
:104460009385859717C501001305852397B0010033
:10447000E780A0C24C4017D501001305A5B897B03E
:104480000100E78080C12244B2402945410117B3B1
:104490000100670063C5B24022444101828041119E
:1044A00022C426C22A84AE8417C501001305451F05
:1044B00097D501009385058E06C697B00100E78069
:1044C000C0BD17D501001305E5C397B00100E78013
:1044D000C0BC294597B00100E78000C197D5010015
:1044E0009385458B97070020239687B817C5010051
:1044F0001305051B054497070020239B97B69707D4
:104500000020239887B697170020239C972097B008
:104510000100E78080B89715002083D5852017D546
:1045200001001305A5BE97B00100E78000B729453B
:1045300097B00100E78040BB971700202380870ECB
:1045400097F7FF1F938747E7DC4717F5FF1F0345E2
:10455000653103D70700C167FD17631EF700B7E792
:10456000040003A387051306000A85452244B240D0
:10457000924441010283B7E7040003A387051306B1
:10458000001493050010DDB7B1C1411122C417C555
:1045900001001305E5102E8497C501009385C57EA3
:1045A00006C697B00100E78040AFA28517D501008D
:1045B000130585B497B00100E78020AE2244B240D5
:1045C0002945410117B30100670003B2828097F7C4
:1045D000FF1F83C7972917F5FF1F034525293D8D29
:1045E000220597F7FF1F83C777283D8D4605458134
:1045F00011C5D1476315F500554582800545828078
:10460000411197170020239E07109717002023873A
:10461000070006C6170700200347C7B09307F00A34
:104620006315F7029307F0F8894517050020130575
:1046300065AF170700202307F7AE97070020A38375
:1046400007AE97600000E780A08297600000E780D7
:1046500060AF97600000E780A0B081453705040097
:104660009707002023A607AA97070020238107AAFF
:1046700097070020239007A297070020239E079EFC
:1046800097070020239307A897070020239407A8E3
:1046900097300000E7806014014597600000E780D4
:1046A000208697000000E780C0F297070020239F34
:1046B000A7A4B7E70400BC4F13060014894517F5FB
:1046C000FF1F0345251A829797C501009385856DC5
:1046D00017C501001305C5FC97B00100E780E09BFA
:1046E0009705002083D585A217D50100130505A3E2
:1046F00097B00100E780609AB2402945410117B3A5
:1047000001006700639E797122D437E404005C5C89
:1047100006D626D2354697C501009385A57C17D5C8
:1047200001001305A551829711E917C50100130572
:10473000E5FC97B00100E78020AE01A097F7FF1FCE
:10474000938707133ECCB7F50700856793870780EB
:10475000814617F6FF1F13062611E10519453ECEC7
:1047600097E0FF1FE780E0077C44194697F5FF1F9D
:104770009385850F1705002013050592829734084D
:1047800017F6FF1F1306460E97D501009385C5C186
:1047900017D501001305C5C297700000E78020F30C
:1047A000AA8421C197C501009385456617C50100FC
:1047B000130505EF97B00100E780208EA68517C589
:1047C00001001305257397B00100E780008D29458E
:1047D00097B00100E7804091B25022549254456155
:1047E000828097E00000E780405817C5010013055C
:1047F000656797600000E78040E797600100E78009
:10480000801117F5FF1F1305A5B797600100E7801A
:1048100020FA17C501001305E56597600100E780E0
:104820000012AA8497600000E780004E97100100F4
:10483000E78060E997900100E78080829780000020
:10484000E780E0A997700000E78000C4974001006E
:10485000E780C0AA97C501009385455B17C5010095
:10486000130505E499C897B00100E7800083A68589
:1048700017C501001305456AB9B797B00100E78075
:10488000C08117C501001305656B97B00100E78073
:10489000C080294597B00100E7800085974001005E
:1048A000E780A08697000100E78060A563080514F3
:1048B00097000000E780E0D197F7FF1F83D7479F5D
:1048C00017170020231FF7E42A8699C36302F5080F
:1048D00097C501009385855317C50100130545DC75
:1048E00032C697A00100E780407B32469715002032
:1048F00083D525E317C501001305C56597A0010001
:10490000E780A079294597A00100E780E07D97170F
:104910000020238507D097170020239407E0977085
:104920000000E780A01597C501009385254E17C5A7
:1049300001001305E5D697A00100E780007617C5B2
:1049400001001305E56997A00100E780007541B5F6
:1049500085453705040097300000E78000E897C5DB
:1049600001009385A54A17C50100130565D397A0DB
:104970000100E780807217C501001305E56097A06C
:104980000100E7808071294597A00100E780C0758C
:104990008547171700202303F7C897F7FF1F938752
:1049A000A7A1DC4703D70700C167FD176316F7000F
:1049B00097F0FFFFE780004897700000E780401CF9
:1049C0008567938707E33E9597700000E780001C9A
:1049D00097200000E78040BB17150020035565D4E1
:1049E00097500000E780401E054597500000E78083
:1049F000205197500000E780A07635B7970000005F
:104A0000E78020BD97F7FF1F2392A77097C501008D
:104A10009385C53F17C50100130585C897A0010000
:104A2000E780A06717C601001306465897F5FF1FD9
:104A300083D5C56D17C501001305C55797A00100A3
:104A4000E780A065294597A00100E780E0693C4C1C
:104A50001306000A894517F5FF1F0345A5E0829755
:104A6000014597500000E780A04975BD411122C45F
:104A700037E404008327041A06C682979750000083
:104A8000E78040188327040817F5FFFF1305454703
:104A9000829797F7FF1F2387A7DC17F5FF1F1305E2
:104AA000A59197500000E78020C92244B2404101FF
:104AB00017030000670063C5B7E70400FC471171E6
:104AC000A2DDCAD986DFA6DBCED72E8432892E8618
:104AD000AA8517F5FF1F1305E564829717F7FF1FD7
:104AE0001307476483470700930680029387E7070D
:104AF00093F7F70FE3ECF610BA898A0717C701009E
:104B0000130747C3BA979C43BA9782878D4797C5C7
:104B100001009385E53117C50100130565B8630FE2
:104B2000F40097A00100E780405717C50100130566
:104B3000E5EE97A00100E7804056BDA497A00100D4
:104B4000E780A05517C501001305C5EE97A0010029
:104B5000E780A054294597A00100E780E05893071B
:104B600020F8114697F5FF1F9385C55B4A8517F717
:104B7000FF1F2309F75A97F7FF1FA386075A97F0DD
:104B8000FFFFE780802A2A841DC997C5010093850D
:104B9000252A17C501001305A5B097A00100E780DD
:104BA000C04FA28517C50100130585EC97A0010031
:104BB000E780A04E294597A00100E780E05297C505
:104BC00001009385E52617C50100130565AD97A083
:104BD0000100E780804C17C501001305A5EA97A0E6
:104BE0000100E780804B294597A00100E780C04F76
:104BF0004165930730FA054697F5FF1F9385855267
:104C00007D1517F7FF1F230FF75097F0FFFFE78081
:104C1000C0212A841DC997C501009385652117C548
:104C200001001305E5A797A00100E7800047A285D2
:104C300017C501001305C5E397A00100E780E04513
:104C4000294597A00100E780204AB7E70400BC4F40
:104C50000566130606C8A14517F5FF1F034585C065
:104C60008297FE506E54DE544E59BE5911618280B7
:104C700091476303F40297C501009385651B17C52F
:104C800001001305E5A197A00100E780004117C5C9
:104C90000100130565E271BDB7E70400FC4F9145C3
:104CA00017F5FF1F034505BC829797C50100938543
:104CB000251817C501001305A59E97A00100E780E0
:104CC000C03D17C501001305E5E097A00100E7808E
:104CD000C03C294597A00100E780004197400000B3
:104CE000E780C06E914535A485476303F40297C5FC
:104CF00001009385E51317C501001305659A97A078
:104D00000100E780803917C50100130525DE15B5C0
:104D100097F7FF1F23902739B7E704000566BC4FBC
:104D2000130606C8C1450DBF8D476303F40297C53E
:104D300001009385E50F17C501001305659697A03F
:104D40000100E780803517C501001305E5DBD5B309
:104D5000930740F8114697F5FF1F9385A53C4A85B8
:104D600017F7FF1F2300F73C97F7FF1FA38D073AA4
:104D700097F0FFFFE780600B2A84E30405EE97C5F8
:104D800001009385E50A17C501001305659197A0F9
:104D90000100E7808030A28517C50100130545CDCD
:104DA00097A00100E780602F294597A00100E780C8
:104DB000A03345BD9147E31CF4F6B7E70400FC4F70
:104DC0009305000217F5FF1F0345C5A9829797C5F4
:104DD00001009385E50517C501001305658C97A0B3
:104DE0000100E780802B17C50100130565D3F1BDD5
:104DF000894763E3870297C501009385650317C55B
:104E000001001305E58997A00100E780002917C577
:104E10000100130525D231BB97F4FF1F83C4A430D2
:104E200097F7FF1F83C7173097C50100938545008B
:104E3000A20417C501001305A586DD8C97A001000B
:104E4000E780A025A28517C501001305E5CF97A02F
:104E50000100E7808024C204294597A00100E78073
:104E6000A028C1849305D4FF93960401C1824A8689
:104E700093F5F50F17F5FF1F1305F52A973000007E
:104E8000E7806099E35F90DC930750F817F7FF1F06
:104E9000230AF72883C73900228697F5FF1F9385D9
:104EA000652885074A8517F7FF1FA30EF72697F099
:104EB000FFFFE78080F72A84E30505DA97C5010044
:104EC000938505F717B501001305857D97A00100AF
:104ED000E780A01CA28517C501001305E520C9B510
:104EE000894763E3870297C50100938565F417B589
:104EF00001001305E57A97A00100E780001A17C5A5
:104F00000100130525C635B197400000E780004C2D
:104F1000A28517F5FF1F1305E52097500000E780D5
:104F200020F581B38D476303F40297C50100938593
:104F300025F017B501001305A57697A00100E780BD
:104F4000C01517C501001305A5C3E5B6B766020075
:104F50000146B7750200054597E0FF1FE7806088AE
:104F6000930760F817F7FF1F230EF71A97F7FF1F35
:104F7000A38B071A9307000617F7FF1F2306F71ADC
:104F8000894717F7FF1FA301F71A97F7FF1F238E13
:104F9000071897F7FF1FA38A0718C14717F7FF1FC6
:104FA0002306F718930720F917F7FF1FA300F71838
:104FB000314697F7FF1FA38CA71697F5FF1F938520
:104FC00065164A8597F7FF1F2383071697F0FFFFA3
:104FD000E780A0E52A84E30605C897C5010093850C
:104FE00025E517B501001305A56B97A00100E78023
:104FF000C00AA28517C50100130505BA55B3B1470C
:105000006303F40297C50100938585E217B501009B
:105010001305056997A00100E780200817C5010066
:10502000130545B939B6B7E70400FC4F93050004F2
:1050300017F5FF1F03450583829797400000E7801F
:10504000E038B145F9B5914763E3870297C50100A0
:10505000938505DE17B501001305856497A001004F
:10506000E780A00317C50100130585B6D9B497F4EE
:10507000FF1F83C4640B97F7FF1F83C7D70AA204DF
:10508000DD8C8E04B77702006D14BE942286A6854F
:1050900017C50100130505B597A00100E780E0FFE3
:1050A000B7E70400FC47228697F5FF1F9385D507D5
:1050B0002800829793160401C1823000A685094515
:1050C00097D0FF1FE780E0712A8409C917C5010046
:1050D000130505B397A00100E7800014930770F84B
:1050E000194697F5FF1F9385E5034A8517F7FF1FBC
:1050F000230AF70297F7FF1FA388870297F0FFFFA5
:10510000E780A0D22A84E30E05B497C501009385F9
:1051100025D217B501001305A55897A00100E78017
:10512000C0F7A28517C50100130585AE95B999474B
:10513000630BF41297C50100938585CF17B5010065
:105140001305055697A00100E78020F517C501005B
:10515000130585ADF9BA914763E3870297C501004E
:10516000938505CD17B501001305855397A0010060
:10517000E780A0F217C50100130585AC5DBA97F46E
:10518000FF1F83C464FA97F7FF1F83C7D7F9A204F0
:10519000DD8C8E04B77702006D14BE942286A6853E
:1051A00017C50100130505AB97A00100E780E0EEED
:1051B000B7E70400FC47228697F5FF1F9385D5F6D5
:1051C0002800829793160401C1823000A6850D4500
:1051D00097D0FF1FE780E0602A8409C917C5010046
:1051E000130505A997A00100E7800003930780F845
:1051F000194697F5FF1F9385E5F24A8517F7FF1FBC
:105200002302F7F297F7FF1FA38087F297F0FFFFC3
:10521000E780A0C12A84E30605A497C50100938511
:1052200025C117B501001305A54797A00100E78028
:10523000C0E6A28517C501001305C5A495B6994718
:105240006303F40297C50100938585BE17B501007D
:105250001305054597A00100E78020E417C501006C
:105260001305C5A3F9B0B7E70400FC4F930500048C
:1052700017E5FF1F0345055F829797400000E78011
:10528000E014994579B18D476303F40297C5010095
:10529000938505BA17B501001305854097A0010055
:1052A000E780A0DF17C501001305C5A059B017C5D9
:1052B0000100130525A197A00100E780E0F5130583
:1052C000C01297D0FF1FE780C007014597E0FFFF9E
:1052D000E78080DC0D4597100000E78060A4294539
:1052E00097D0FF1FE780E00597D0FF1FE78040F6CB
:1052F0008DBA99476303F40297C50100938545B3BE
:1053000017B501001305C53997A00100E780E0D863
:1053100017C501001305C59B29B817F7FF1F0347E1
:10532000B7E097F7FF1F83C727E022075D8F9166DD
:10533000BA96C2061166C1821306F6EF8D47636501
:10534000D60297E7FF1F938727079C4B17F6FF1F8F
:10535000034676DD9386C7002DC203D6070069CACF
:105360008907E39CD7FE89471307A0F8114697F5F4
:10537000FF1F938525DB4A8597F6FF1F2384E6DA16
:1053800017F7FF1FA301F7DA97F0FFFFE780E0A907
:105390002A84E308058C97C50100938565A917B594
:1053A00001001305E52F97A00100E78000CFA2853B
:1053B00017C5010013050593E5B203D60700630E78
:1053C000E60A8907E39BF6FE8D4779BF91476304A0
:1053D000F40297C501009385A5A517B50100130533
:1053E000252C97A00100E78040CB17C501001305CD
:1053F000E5906FF00FF4B7E70400FC4F9305000849
:1054000017E5FF1F034505468297C9B897C50100F8
:10541000938505A217B501001305852897A0010003
:10542000E780A0C717C501001305C58E6FF06FF0A8
:105430002390E70017E5FF1F130505F897300100DB
:10544000E78020F297C501009385859E17B501007E
:105450001305052597A00100E78020C417C50100AA
:105460001305458C97A00100E78020C3294597A02C
:105470000100E78060C78147C5BD2390070017E59D
:10548000FF1F130565F397300100E78080ED97C596
:1054900001009385E59917B501001305652097A0D4
:1054A0000100E78080BF17C50100130525895DBF96
:1054B000011122CC06CE26CA4AC8834705002A8499
:1054C0009DC797C501009385659217B50100130527
:1054D000251D97A00100E78040BC4C4017C5010086
:1054E000130585C797A00100E78020BBE1A05841C4
:1054F000B707CF009387777D631DF7060359C50073
:10550000854704450356E5009706002083D66621AB
:1055100063FC270383C7040003C71400A207D98FC5
:10552000C2077177C1871307C755639FE7006305FB
:10553000D60C6244F240CA8526854249D2440561B0
:1055400017E3FFFF6700C3C9630AD600CA85268533
:1055500032C697E0FFFFE780A0C832466244F240BF
:10556000CA8526854249D244056117F3FFFF6700CB
:10557000E354B707CC009387777D6317F70497C58B
:1055800001009385A58617B501001305651197A045
:105590000100E78080B01C448356E4008355C400BA
:1055A00003C6070017C50100130585BC97A00100BD
:1055B000E780A0AE6244F240D244424929450561E9
:1055C00017A30100670043B2B707CE009387777D2A
:1055D0006304F70297C501009385458117B5010063
:1055E0001305050C97A00100E78020AB4C4017C5C0
:1055F0000100130565ACFDB5F2406244D244424956
:1056000005618280B7E70400FC4741112E8606C67B
:1056100022C426C24AC02E842A89AA8517F5FF1FF4
:10562000130545B0829797C501009385258217B56C
:1056300001001305E50697A00100E78000A697F595
:10564000FF1F83C525AE17B501001305252897A0B8
:105650000100E78080A4294597A00100E780C0A849
:1056600097F4FF1F938404AC83C7040041479387DA
:10567000070693F7F70F636FF75A17B70100130781
:10568000A7158A07BA979C43BA9782879D476307F5
:10569000F40297B501009385657B17B501001305EA
:1056A000250097A00100E780409F17B50100130572
:1056B000652297A00100E780409E95A497F7FF1F01
:1056C00083C757A6DDCB17F7FF1F0347D7A597F76B
:1056D000FF1F83C747A522075D8F97F7FF1F83C76B
:1056E000A7A4C2075D8F97F7FF1F83C7F7A3E20741
:1056F000D98F17F7FF1F232DF7A083C7640097B535
:1057000001009385A57417B50100130565F917F716
:10571000FF1F230EF79E97A00100E780009897F7E0
:10572000FF1F9387E79E8C4317F6FF1F0346269EB5
:1057300017B501001305C51B97A00100E780E09590
:10574000294597A00100E780209A97F7FF1FA38BB8
:10575000079C2244B24092440249930700F817F78D
:10576000FF1F2301F79C9D4517F5FF1F1305859B20
:105770004101174300006700A36F97600000E780B6
:10578000603F97F7FF1F2380A79A9357850017F76D
:10579000FF1FA30AF798935705012A8417F7FF1FE5
:1057A0002304F79893578501014517F7FF1FA30DB1
:1057B000F79697600000E780404097F7FF1F238629
:1057C000A79697B501009385656817B50100130585
:1057D00025ED97A00100E780408C17F6FF1F0346D8
:1057E000C694A28517B5010013050512B1B7CD47C0
:1057F0006303F40297B501009385456517B5010071
:10580000130505EA97A00100E780208917B501007C
:105810001305051179BD97F7FF1F83C7C79117F7C8
:10582000FF1F03473791A207D98FC207C18717F718
:10583000FF1F231DF78C634AF00097F0FFFFE780FE
:1058400040D997F7FF1F2393A78CB7E7040003A362
:1058500087051306000A89452244B2409244024952
:1058600017E5FF1F03450500410102838D476303D0
:10587000F40297B501009385655D17B50100130526
:1058800025E297A00100E780408117B501001305CC
:10589000E51805B517F4FF1F0344E48897F7FF1FC9
:1058A00083C7578897B501009385455A220417B5D9
:1058B00001001305E5DE5D8C97900100E780E07D37
:1058C000A28517B501001305250797900100E78011
:1058D000C07C294597A00100E78000810D4697F51F
:1058E000FF1F93852584228597E0FFFFE780E05323
:1058F000AA8421C197B501009385455517B50100CC
:10590000130505DA97900100E7802079A68517B581
:1059100001001305A50397900100E7800078224459
:10592000B2409244024929454101179301006700A2
:10593000A37B97E7FF1F239F8774B7E704001166D7
:1059400003A38705130606E8914539B78D4763031E
:10595000F40297B501009385654F17B50100130553
:1059600025D497900100E780407317B50100130517
:10597000A51981B317E4FF1F0344E47A97E7FF1FDB
:1059800083C7577A97B501009385454C220417B514
:1059900001001305E5D05D8C97900100E780E06F72
:1059A000A28517B501001305A5FB97900100E780BC
:1059B000C06E294597900100E78000730D4697E57A
:1059C000FF1F93852576228597E0FFFFE780E0455E
:1059D000AA841DC197B501009385454717B50100FD
:1059E000130505CC97900100E780206BA68517B5BD
:1059F0000100130525F805B797E7FF1F239E87666B
:105A0000B7E70400116603A38705130606E89305AC
:105A1000000299B5894763E3870297B50100938532
:105A2000E54217B501001305A5C797900100E7806F
:105A3000C06617B501001305E50FA5B997E4FF1F70
:105A400083C4646E97E7FF1F83C7D76D97B50100C6
:105A50009385C53FA20417B50100130565C4DD8C0D
:105A600097900100E7806063A68517B501001305D4
:105A7000E5F197900100E780406229459790010089
:105A8000E7808066228697E5FF1F9385A5692685B6
:105A900097E0FFFFE78060392A84630E051A97B507
:105AA00001009385A53A17B50100130565BF9790CE
:105AB0000100E780805EA28517B50100130545EE61
:105AC00099BD854763F98718834519002244B24080
:105AD00092440249B335B00097E7FF1F2386B75CB5
:105AE00017B50100130505ED41011793010067008B
:105AF000C35AA2852244B24092444A8502494101D8
:105B0000170300006700032899476303F40297B561
:105B100001009385A53317B50100130565B897906B
:105B20000100E780805717B501001305651A51B6CB
:105B300017E4FF1F0344245F97E7FF1F83C7975EA7
:105B400097B5010093858530220417B50100130530
:105B500025B55D8C97900100E7802054A28517B58C
:105B600001001305A5E697900100E7800053294541
:105B700097900100E7804057194697E5FF1F9385EE
:105B8000655A228597E0FFFFE780202AAA841DC17D
:105B900097B501009385852B17B50100130545B016
:105BA00097900100E780604FA68517B501001305A7
:105BB000E5E295B397E7FF1F239E8754B7E70400FC
:105BC000116603A38705130606E89305000869B16B
:105BD000854797B501009385652717B50100130523
:105BE00025AC630BF40097900100E780004B17B5DC
:105BF00001001305E5DF75BC97900100E780E049DF
:105C000017B50100130545E097900100E780E048D3
:105C1000294597900100E780204D2244B2409244EC
:105C2000024997E7FF1F2393074E410117630000C6
:105C30006700C3E497B501009385452117B50100BE
:105C4000130505A697900100E780204517B50100D0
:105C50001305450CB9BCB2402244924402494101AB
:105C60008280411106C622C426C239C12A8497E027
:105C70000000E780C068AA8411EDB7E70400BC47C4
:105C80004146814522858297B2402244268592442E
:105C90004101828041657D1597E00000E780006743
:105CA000B7E7040001E9BC47414681452285829758
:105CB0008144D9BF0347E501FC479305900819E3E8
:105CC00093050003AA9541462285829785446DBFBE
:105CD000411106C697E0FFFFE780000E0DC197E770
:105CE000FF1F83D7873C850717E7FF1F231FF73A5E
:105CF00097E7FF1F239CA73AB2404101828097E7B4
:105D0000FF1F83D7C73A850717E7FF1F2311F73A0D
:105D1000E5B78546170300006700C3FB411122C4A5
:105D200091462A8417E6FF1F1306C64D9D652D4533
:105D300006C697D0FF1FE780C0AAB7F7070003C7C2
:105D40000701A5476313F70001A093060010014661
:105D50009D65254597D0FF1FE780A0A897E7FF1F07
:105D60002382874A2244B240914617E6FF1F13065A
:105D700066499D652945410117D3FF1F670063A64A
:105D80001171CED7B7E9040083A7C904CAD917E9AE
:105D9000FF1F13092939A2DD2E8686DFA6DB2E849C
:105DA000AA854A85829797E7FF1F83C7A7371307FE
:105DB000700A6385E710636DF7001307600A638557
:105DC000E704FE506E54DE544E59BE591161828074
:105DD0001307800A6385E7161307900AE393E7FE2B
:105DE0008D476306F41C97B501009385E54317B50D
:105DF00001001305E58A97900100E780002A17B596
:105E000001001305A53F25A08D47630CF40297B54B
:105E100001009385654117B50100130565889790CA
:105E20000100E780802717B50100130565369790BC
:105E30000100E7808026294597900100E780C02A6D
:105E400049B7854717B501001305453617E7FF1F0A
:105E5000230CF72497900100E780003CB7750200FF
:105E6000B76602000146054597D0FF1FE78060979F
:105E7000930760F817E7FF1F2306F72A97E7FF1F2E
:105E8000A383072A9307002617E7FF1F232EF7286F
:105E9000E5779387072117E7FF1F2319F728B145F7
:105EA00097E7FF1F2385072897E7FF1FA381A728F0
:105EB0004A8597000000E780E01621B7914763E329
:105EC000870297B501009385253617A501001305B4
:105ED000257D97900100E780401C17B50100130550
:105EE000E52EB1B797E4FF1F83C4042497E7FF1F93
:105EF00083C77723A204DD8C83A7C9046D1422868F
:105F000097E5FF1F93855522280082978E049316EC
:105F10000401B7750200C1823000A695094597D0EB
:105F2000FF1FE780008C930770F817E7FF1F230B14
:105F3000F71E994597E7FF1FA388A71E95BF9147B6
:105F400063E3870297B501009385052E17A501002D
:105F50001305057597900100E780201417B501001F
:105F600013054528E9B597E4FF1F83C4E41B97E7B1
:105F7000FF1F83C7571BA204DD8C83A7C9046D14C0
:105F8000228697E5FF1F9385351A280082978E0495
:105F900093160401B7750200C1823000A6950D4525
:105FA00097D0FF1FE780E083930780F8BDBF17B548
:105FB00001001305E52597900100E780E025930790
:105FC00090F82304F100834719008D452800A304AD
:105FD000F100834729002305F10097000000E780C6
:105FE00060041305C01297C0FF1FE780803501458C
:105FF00097D0FFFFE780400A0D4597000000E7803B
:1060000020D2294597C0FF1FE780A03397C0FF1F0C
:10601000E78000247DB397E7FF1F23ADA71E828092
:1060200097E7FF1F9387071F03A30700630303007E
:106030000283174300006700A3E341114AC097F6AB
:10604000FF1F83D6066E328917D6FF1F0356E63828
:1060500022C426C206C62A84AE8497000000E780C8
:10606000E06729C921C8994763F69704834714005C
:1060700003470400A207D98F13978700A183D98F04
:10608000C2073167C1831307C7556395E70297D7E6
:10609000FF1F83D78734A301F400A1832302F400F8
:1060A00097F7FF1F83D7E76791C7A302F400A18387
:1060B0002303F40097F7FF1F83C74756A1CB26861B
:1060C000A28517D5FF1F0355453197000000E780D3
:1060D00080C4630F090297F7FF1F83C727548DEB16
:1060E00097E7FF1F83C7471385C79DC097E7FF1F2B
:1060F00083C787FB91EF22852244B2400249A685DF
:106100009244410117430000670083D6E31A09FC5B
:10611000B24022449244024941018280014582807A
:1061200097A70100938747489C4301116800914558
:1061300006CE3EC697000000E780C0EEF240056143
:1061400082808D4763F6B708011126CA06CE22CC9D
:106150000344350097E4FF1F83C4140C97B5010076
:106160009385450EB337800017E7FF1FA306F70A94
:1061700009C497B501009385A50D17B50100130556
:10618000A50D97900100E78040F197E7FF1F83C7B7
:10619000B7086386970097000000E78000439740A8
:1061A0000000E780E0FB9967938757EE2316F10024
:1061B000680085479145A30781002307F1009700F8
:1061C0000000E78020E6F2406244D244056182800C
:1061D0008280894763F7B708011122CC06CE26CA10
:1061E0008344250085472A84639DF404914763F521
:1061F000B704034545008347340022055D8D97D7DA
:10620000FF1F239CA71C97000000E780005699679A
:10621000938767EE2314F100834734002305910030
:10622000A305F10083474400954528002306F100AB
:1062300097000000E78000DFF2406244D24405612D
:106240008280FDF89967938767EE2314F10097D752
:10625000FF1F83D78718A305F10023050100A18341
:10626000E1B782800111996722CCD51717F4FF1F7F
:106270001304C43A2314F1008347040026CA97F498
:10628000FF1F9384044A2305F10083D704002800EC
:106290009545A305F100A18306CE2306F1009700E2
:1062A0000000E78020D803D604008345040017B51A
:1062B0000100130565FB97900100E78000DEF240C6
:1062C0006244D244056182809D677971D917231693
:1062D000F10097F7FF1F9387673483C70700130503
:1062E000F10006D62307F10097000000E780A09791
:1062F00009E9B7E70400BC47414681451305F100B1
:1063000082976800CD4597000000E780A0D197F5FF
:10631000FF1F83C5A53017B501001305E5F797905A
:106320000100E78080D7B25045618280630805167E
:10633000411126C206C622C44AC097E7FF1F83C781
:10634000B7ED97F4FF1F83C4642D99C393E4240031
:106350002A8497100000E78080F719C193E40401B4
:1063600037E9040083278904228513062003814529
:106370008297930750FA2300F4009307A005A30027
:10638000F4008D472301F4009147A301F400930723
:106390005005A302F40097F7FF1F83D78738230423
:1063A000F400A183A304F40097D7FF1F83D7E7026B
:1063B000230394002305F4009304C400A183230263
:1063C0000400A305F400268597000000E780A0895B
:1063D00019E583278904414681452685829797D709
:1063E000FF1F83D727FD230EF400A183A30EF40023
:1063F00093070002230FF400930710FAA30FF40091
:106400009D472300F402A3000402B7E70400FC4701
:1064100013052402194697D5FF1F9385E5448297FB
:1064200097E7FF1F83D7A7C82304F402A183A3041F
:10643000F40297E7FF1F83D747C72305F402A18320
:10644000A305F40297E7FF1F938747C683970700CA
:106450002285930500032306F402C207C183A183AA
:10646000A306F40297D7FF1F938787E5839707005A
:106470002307F402C207C183A183A307F402970094
:106480000000E780A0212308A4022181A308A40220
:10649000B2402244924402494101828082805D716F
:1064A000E17793C777FF1305E10086C62316F10055
:1064B00097000000E780C0E768009305400397005D
:1064C0000000E78020B6B640616182805DC941115D
:1064D00022C426C206C6930750FA2300F50093078C
:1064E000A005A300F50089472301F5009147A3010A
:1064F000F50093075005A302F50097F7FF1F938758
:10650000E71183C707009304C5002A842303F5001D
:1065100097E7FF1F938757D083C707002302050023
:10652000A303F50097F7FF1F83D7A71F2304F500E8
:10653000A183A304F50097D7FF1F83D707EA23059C
:10654000F500A183A305F500268597F0FFFFE780FE
:10655000807101E9B7E70400BC47414681452685C3
:1065600082972285F14597000000E7802013230ED3
:10657000A4002181A30EA400B24022449244410110
:10658000828082805D710A8586C6A2C49700000061
:10659000E78000F437E404007C448A8508107946DB
:1065A00082973C441305E103094681458297101008
:1065B00093050002014597D0FFFFE7802014B64005
:1065C0002644616182800111B7C7A55A22CC938706
:1065D000C73317E4FF1F130434C43EC483470400C9
:1065E000856601469965254506CE3EC697C0FF1FC4
:1065F000E780201F3000A1469965294597C0FF1FFD
:10660000E780201E8345040017B50100130545D31C
:1066100097900100E78060A8F240624405618280A3
:106620000111A146300099652D4522CC06CE97C0B8
:10663000FF1FE780001BA24737C4A55A1304C433C9
:1066400063958702B24517B50100130525C7B33519
:10665000B00097E7FF1FA381B7BC97900100E780C8
:10666000C0A3F2406244056182809165A14630007A
:10667000938505F02D4597C0FF1FE7808016A24740
:10668000E38287FC97E7FF1FA38807B8814517B50A
:1066900001001305E5C4D1B7C16769768146FD17CE
:1066A00005061397060141836364B7003E85828027
:1066B0003307D50003470700B98F214713F81700A8
:1066C000858363050800B18FC207C1837D171377E7
:1066D000F70F6DF78506F1B741C5A547054763F28A
:1066E000B70883471500034705003168A207D98F13
:1066F00013978700A183D98FC207C1831308C85598
:10670000054763900707411106C622C426C2034409
:106710002500914763F087049307540063ECF5026A
:10672000A301C50021822302C5009304340091C651
:10673000A302D500A1822303D5002A84A685970051
:106740000000E780A0F526942300A4002181A30087
:10675000A4000147B240224492443A85410182801C
:1067600005473A8582800111B7C7A55A22CC938785
:10677000E7342A842AC6856601469565254506CEF6
:106780003EC497C0FF1FE780C0053000A146956555
:10679000294597C0FF1FE780C004A28517B50100F7
:1067A000130505BC97900100E780208F970000003B
:1067B000E78080DDF2406244056182800111A146DC
:1067C000300095652D4522CC06CE97C0FF1FE7808F
:1067D0004001A24737C4A55A1304E43463958702E5
:1067E000B24517B501001305A5B197D7FF1F239632
:1067F000B7BEC205C18197900100E780008AF240D0
:106800006244056182809165A1463000938505EE62
:106810002D4597C0FF1FE780C0FCA247E38287FC9D
:10682000D14717D7FF1F231AF7BAD14517B5010073
:10683000130505AFC9B74DC5411126C206C622C40E
:10684000AE84D1C92A8497100000E780E0A897E7BA
:10685000FF1F83C7679C99C7A685228597300000D4
:10686000E780006197F7FF1F83C747DBADC79547F8
:1068700063F397068347040013073005639DE7041D
:1068800083461400130750046397E60483462400EC
:10689000130710046391E60403473400631DF702F5
:1068A000034744009307B0046317F70203475400FB
:1068B000930790056311F702A2852244B240268611
:1068C000924417D5FF1F035545B18D46410117F37B
:1068D000FFFF67002340B24022449244410182807E
:1068E000828001114EC606CE22CC26CA4AC893F732
:1068F0001500AE899DCBAD67371700409387A7AAD7
:106900001CC3B7E70400BC4F13060019854517D513
:10691000FF1F034565AC829713C51900F24062441E
:10692000D2444249B2490561828093F7250001456E
:10693000F5D717F7FF1F0357A7DE954763F9E70C55
:10694000014417F6FF1F1306A6CD93063005130565
:106950005004130810049308B00413039005930720
:1069600064006374F7043A847D5997F4FF1F83C46D
:1069700024CB97F7FF1F83C7B7CAA204DD8CAD678E
:106980009387B755638BF41463E3970AA9679387DA
:10699000A755638EF414A28517F5FF1F130545C88C
:1069A00097000000E78060E9E9A0B307860083C58F
:1069B0000700639AD50483C517006396A50483C5B1
:1069C00027006392050583C53700639ED50283C502
:1069D0004700639A150383C75700639667022289AD
:1069E0000DE897F5FF1F83D5A5D3B3852541C205D3
:1069F00017F5FF1F1305C5C2C1814A959700000016
:106A0000E780A0E3E1A005044204418089BF3A8405
:106A10007D598547E3EB87F45DC4854517F5FF1F76
:106A2000130505C097000000E78020E169A8B16761
:106A30009387C7556389F404B5679387D755E39C5B
:106A4000F4F4A28517F5FF1F130585BD97300000EC
:106A5000E78000428947630EF4009305E4FFC20516
:106A6000C18117F5FF1F1305C5BB97100000E78014
:106A7000A086A68517B501001305459097800100F3
:106A8000E780A06189A097200000E780C0339710BD
:106A90000000E780C08311C9A28517F5FF1F130509
:106AA00025B897100000E78020830546A28517F5DA
:106AB000FF1F1305E5B697F0FFFFE78040589720CA
:106AC0000000E7804030FD57E31DF9F097F7FF1F06
:106AD000239807C413C5290091B5A28517F5FF1F98
:106AE000130505B497F0FFFFE780806359B7A285CF
:106AF00017F5FF1F1305C5B297F0FFFFE78080620F
:106B00008DBF411122C437E404005C5C06C63546E3
:106B100097A501009385053D17B5010013050512E2
:106B2000829711E917B5010013058586978001004A
:106B3000E780806E01A08327041C82972A84054584
:106B400097C00000E780C02197700100E780E0A6B1
:106B500097600100E780E07B97B00000E78040335A
:106B60002285B2402244410182804111054506C67A
:106B700022C426C297C0FFFFE780E03B1305A004B4
:106B800097B0FF1FE780A052757585457D1597C0AA
:106B9000FFFFE78080257D7585451305F53697C095
:106BA000FFFFE780E02E371400408327840A8D45DD
:106BB0001305002093E707202324F40A97C0FFFF62
:106BC000E780A022B7E4040097C0FFFFE780C0671A
:106BD000C85897800100E780206417B501001305AD
:106BE000E50597800100E78020638327840C8545B5
:106BF000414593E707082324F40C97C0FFFFE78083
:106C000020298D451305000897C0FFFFE780402825
:106C100097C0FFFFE780205537A507001305051231
:106C200097C0FFFFE780C050014597C0FFFFE78096
:106C3000E05695450545894717F7FF1F2304F7AE32
:106C400097C0FFFFE7802057B7E700E01307000673
:106C5000238DE7403707000423A0E71097D0FFFFFC
:106C6000E780A0D897D0FFFFE780A0EA9700000058
:106C7000E78060E997000000E780C09A9700000075
:106C8000E78000B497E0FFFFE78080DE9700000018
:106C9000E780C06597000000E780801083A70408A4
:106CA00017050000130525C4829797C7FF1F23858A
:106CB000A772BC4C130600648545829797B0FF1FEE
:106CC000E780007301458280AD67371700409387E6
:106CD000A7AA1CC3B7E700E03707400023A0E718C6
:106CE00001000100B7F7070003C70701A5476316B6
:106CF000F7009397450191C301A04111AE8601466B
:106D0000AA85254506C697C0FF1FE78080ADB24023
:106D1000B7E700E03707400023A0E7104101828079
:106D20004111B2862E86AA852D4506C697C0FF1F43
:106D3000E78020ABB2400145410182809307000407
:106D400063ECC7041D71A2CC2A840808A6CACAC86D
:106D500086CE32C697800100E780C028AD6737171E
:106D600000409387A7AA1CC3B7E400E0370940009E
:106D700023A0241901000100B2461008A28529456C
:106D800097C0FF1FE780E0A5F640664423A02411CA
:106D9000D6444649256182803955828041110D656E
:106DA0008D4506C697C0FFFFE7802004B717004057
:106DB0008D6623A6D70A17F5FF1F1305E5961387DF
:106DC000C70A9387870A1CC15CC5856689675CC949
:106DD00058C114C518C9B7E70400B24003A3871E01
:106DE000410102838145B307B5008387070089E726
:106DF000172300006700C3038505C205C181E5B7FD
:106E0000411106C6B94763EEB70017A50100130587
:106E1000656F97000000E78020FDB2400545410105
:106E200082808347E500130710036390E7028547DC
:106E300017F7FF1F230CF79E17A501001305C56E5A
:106E400097F7FF1F2393079EE9B713070003E39EFD
:106E5000E7FA97F7FF1F238B079C97F7FF1F2396EF
:106E6000079C17A501001305A56D65B7411126C242
:106E7000E97797F4FF1F9384A49B22C49387A755B7
:106E80002E842381B4002E86AA8517F5FF1F1305D3
:106E9000659A06C62390F400A38104009780010040
:106EA000E780401493052400C205C18117F5FF1F38
:106EB0001305259897F0FFFFE780407EB387840095
:106EC0002382A7002181A382A700930564002244A6
:106ED000B24026859244C205C181410117230000BA
:106EE000670003F509C99307000463E6B7001703B9
:106EF00000006700E3F782809306F00F03070600A7
:106F000019E79307F00F63F0B7022E85828093870D
:106F10001500C207C183E3E6F6FEAA952380E500CB
:106F20000506BE85E1BF2E9523000500F9BF0111BE
:106F30001C08B69706CE238A07FE5C00BE9617A8EB
:106F400001001308686B1377F600429703470700A8
:106F5000FD1611822380E600E397D7FE3E86970058
:106F60000000E780A0F9F24005618280011158001D
:106F700006CE23070100A947BA8829482543B376DE
:106F80000603FD1793F7F70F93860603A304D700B4
:106F9000B35606036375C3007D173686EDF333865B
:106FA000F80097000000E78060F5F24005618280FC
:106FB000397117A601001306265D06DE22DC26DAEB
:106FC0002A844AD84ED697000000E78020F3AA858D
:106FD00017E6FF1F0356E6749146228597000000CE
:106FE000E78020F597E7FF1F83C74763AA8517A6A9
:106FF00001001306E65689C717A601001306C655F9
:10700000228597000000E78060EFAA8517A601009F
:107010001306C657228597000000E78020EEAA8558
:1070200017A6010013060657228597000000E78087
:10703000E0ECAA851146228597000000E78040F326
:10704000AA8517B60100130666B3228597000000D3
:10705000E780C0EAAA8517A60100130626542285F8
:1070600097000000E78080E9AA8517B601001306A3
:10707000E6B0228597000000E78040E8AA85130665
:107080005005228597000000E78080EE97D7FF1F0C
:1070900083C79718AA8517A601001306E64C89E74F
:1070A00017A601001306C64C228597000000E78052
:1070B000E0E4AA8517A601001306864E22859700F4
:1070C0000000E780A0E337A60700AA851306061292
:1070D000228597000000E780A0E9AA8517A6010095
:1070E0001306864C228597000000E78020E197E791
:1070F000FF1F83C7E764AA8517A601001306C647CA
:1071000089E717A601001306A6472285970000000D
:10711000E780C0DEAA8517A601001306A6492285CE
:1071200097000000E78080DDAA8517A601001306FE
:10713000E648228597000000E78040DCAA8517A674
:10714000010013062648228597000000E78000DB37
:107150009146AA8517C6FF1F0356C62522859700AC
:107160000000E78000DDAA8517A601001306C645CA
:10717000228597000000E78060D89146AA8517C64F
:10718000FF1F03568625228597000000E78060DAFE
:10719000AA8517A601001306A643228597000000C2
:1071A000E780C0D59146AA8517D6FF1F035626F063
:1071B000228597000000E780C0D7AA8517A60100A6
:1071C00013068641228597000000E78020D3914670
:1071D000AA8517D6FF1F035646ED228597000000AB
:1071E000E78020D5AA8517A601001306663F2285F1
:1071F00097000000E78080D09146AA8517D6FF1F30
:107200000356C6EA228597000000E78080D2AA854F
:1072100017A601001306063D228597000000E780AF
:10722000E0CDAA85914617C6FF1F03566609228541
:1072300097000000E780E0CFAA8517A6010013069B
:10724000E63A228597000000E78040CBAA8581447A
:1072500097C9FF1F938949611949B387340103C650
:1072600007008946228597000000E78080CC8504CE
:10727000AA85E39424FF17A601001306A6372285EA
:1072800097000000E78080C72AC6080897F0FFFF34
:10729000E780609DB24504081309010283C704001A
:1072A00003C614009146A2075D8E22859700000058
:1072B000E78020C88904AA85E31299FEF25062543F
:1072C000D2544259B2592161828017E5FF1F03450C
:1072D0002547828097E7FF1F83C7475589E7172314
:1072E00000006700E3B4828097E7FF1F83C7A758B9
:1072F00099EF411106C697200000E78040ABB240ED
:10730000854717E7FF1F2308F756410182808280D7
:107310006302054C6380054C2971B7064000232E9B
:107320001112232C8112232A9112232821132326A0
:107330003113232441132322511323206113232EBD
:107340007111232C8111232A91112328A1112326A5
:10735000B11101475948A5069319070193D90901AD
:1073600063F1B902B307E50083C70700D91793F7A4
:10737000F70F6368F800B3D7F600858B1306170084
:10738000A1E3B3893541C20993D90901B9472E89CF
:10739000AA8463F937033304E500394697A5010051
:1073A0009385C505228597800100E78040C119E9D2
:1073B000CE85228597000000E780C0A425E5F1A4D2
:1073C000328759BF97E7FF1F83C74746638F07245C
:1073D000BD6A396C014A17EBFF1F130BAB36938B59
:1073E000FA55938CFA66130DEC5505A8B387440142
:1073F00083C6070097E7FF1F83D72743A5E39307BB
:10740000A005639BF600854717E7FF1F231FF74082
:1074100097E7FF1F2388D732050A93170A01C18314
:10742000E3E627FD8320C113032481138324411342
:10743000032901138329C112032A8112832A4112CD
:10744000032B0112832BC111032C8111832C4111B9
:10745000032D0111832DC11031618280854D639B05
:10746000B7039307500A639EF600894717E7FF1F8B
:10747000231DF73A930750FA17E7FF1FA304F72CD1
:1074800061BF9307A005E389F6F897E7FF1F239EE6
:10749000073859B7138717004207DA9741832380CB
:1074A000D70017E6FF1F2312E6388D47E3F6E7F60D
:1074B00017E4FF1F0344342997E7FF1F83C7A7285A
:1074C00022045D8C9307F4FFC207C1839306F00D7D
:1074D000E3EDF6FA93076400C207C183E31EF7F2F7
:1074E00093052400C205C18117E5FF1F1305A525DB
:1074F00097F0FFFFE780801A33078B008347570020
:1075000003474700A207D98F17E7FF1F231F073044
:107510006312F5108149630DB40197E9FF1F83C918
:10752000A922A20997E7FF1F83C71722B3E9F90031
:10753000170500001305459B97F0FFFFE780E0ADBE
:107540006385790963EF3B036388A9059307EC65BD
:107550006383F90697E7FF1F83C7071F054763800B
:10756000E70881CB1387A7051377F70F8D4663F9DB
:10757000E6081307F0072300E100A300F1008945A6
:1075800095A8638999059387FA77E395F9FC97F0B5
:10759000FFFFE78000F111A8A28517E5FF1F130583
:1075A000A51A97F0FFFFE78000BA014597F0FFFFAB
:1075B000E780A0A695B5A28517E5FF1F1305C5189E
:1075C00097F0FFFFE78020C1CDB797F0FFFFE7807E
:1075D000A0C9E1BF97F0FFFFE78040CFF9B793075D
:1075E00010F8130511002300F10097F0FFFFE7806A
:1075F00020EEFD450A8597000000E780608775B79B
:10760000A28517E5FF1F1305251497E0FFFFE7800C
:10761000607761BF9307F00789450A852310F10061
:1076200097000000E780C084C5BB15476375270538
:1076300003C604009306500B0147631FD60203C61E
:1076400014009306B0053E876318D602CA852685C6
:1076500097F0FFFFE780C0AC11C917A50100130523
:10766000E5DA97F0FFFFE78020786DBB17A50100F2
:10767000130505DBFDB70147B70640005946A506CF
:1076800013140701418063692401CA85268597C0C8
:10769000FFFFE780E0B479B3B389E40083C7090052
:1076A000D91793F7F70F6367F600B3D7F600858B0A
:1076B0000507F9F73304894042044180BD4763FD63
:1076C0008706414697A50100938585D74E8597800B
:1076D0000100E780C08E17A601001306A6D705C1DA
:1076E0003D4697A50100938525D84E8597800100DA
:1076F000E780E08C39E517A601001306E6D781453F
:107700000A8597F0FFFFE780607FAA850A859700CA
:107710000000E780208AAA85179601001306065507
:107720000A8597F0FFFFE780607DAA850A8597109C
:107730000000E780E06FFDB1E304F4FAB947E31617
:10774000F4F4394697A50100938545CB4E85978083
:107750000100E780C08601E5A2854E85A1B93946C2
:1077600097A50100938585D24E8597800100E7801B
:10777000008501DDC147E3FA87F0414697A5010086
:107780009385C5D14E8597800100E7804083E31E35
:1077900005EE83C7090113071003639CE7008547C3
:1077A00017E7FF1F230EF7F817A50100130545D0B3
:1077B0004DBD1307000317A50100130565D2E39221
:1077C000E7EA97E7FF1F238D07F617A501001305CA
:1077D000A5CF41BD8280411126C2AE848D4522C411
:1077E00006C62A8497B0FFFFE780806AB71700407B
:1077F00099C803A5C70C418D23A6A70CB24022440B
:1078000092444101828003A5870C418D23A4A70CDB
:10781000F5B78347050003471500A207D98FC207B4
:107820006177C18713072720639AE7008345250006
:107830003705040017030000670023FA828017E66B
:10784000FF1F1306A6038147B2861303F00FA94852
:107850003308F6000348080013F7F70F6307A80C76
:10786000630668008507E39517FF2947B387E6009D
:107870002380A70097E7FF1F938707015DA84111A9
:1078800013D765001347170006C693F63500058B1E
:10789000954791CA054699476387C60009469D47A3
:1078A0006383C600A14713F645003336C00093F644
:1078B0008503050685C2A145638BB604E145638A4D
:1078C000B604930580026388B6049305800363932E
:1078D000B600914697E5FF1F238DF52097E5FF1F22
:1078E0002388C52097E5FF1FA384D520BE8517A553
:1078F0000100130565D497700100E780007AB2405B
:10790000854717E7FF1FA306F71E410182808546C2
:10791000D1B78946C1B78D4675BF17A501001305BC
:1079200025D4177301006700437717E7FF1F13077C
:10793000A7F5BA972380B700E147E302F5F4930770
:107940007002E30CF5FC82802A87238005008147C2
:1079500017E5FF1F130585F21308F00F2946B3063C
:10796000F50083C606006396E60297E6FF1F93863E
:10797000A6F1B69783C7070005452380F500994710
:10798000636EF7029D4763FDE700E147630DF70073
:107990008280638506018507E393C7FC0145C5B76F
:1079A000238005008280B737004003C7370083C7B4
:1079B000050093F70704D98F2380F50082805D715D
:1079C00052DC56DA5ED6716A97EBFF1F938B8B23DE
:1079D0008D6AA6C24EDE62D486C6A2C4CAC05AD878
:1079E00066D26AD06ECEC1495E8C97E4FF1F938445
:1079F00064EA130A0A20938A7ADC17E9FF1F034915
:107A00006923B3872B0183C7070093F7F70FC9EFEB
:107A1000B787004003C76700058BE310077C03C7E7
:107A20006700118BE30D077E83C75700918B99E3A5
:107A30006F10200317E7FF1F0347E71F8547630405
:107A4000F7006F10400197E7FF1FA384E70A97E74D
:107A5000FF1F238107F097E7FF1F238F07FA97E7A0
:107A6000FF1F238D070697E7FF1F238A070697E767
:107A7000FF1FA38107EE97E7FF1FA38F07F897E784
:107A8000FF1FA38D070497E7FF1FA38A070497E74B
:107A9000FF1FA381070697E7FF1FA38E0718B7876D
:107AA000004011476F0070779307190093F7F70FA5
:107AB0003D476364F70617E7FF1F230DF71697E7A7
:107AC000FF1F93872716CA9783C707001307100263
:107AD00093F7F703638EE71E6366F7040544638537
:107AE000871CE38C07620947638EE71013070002C7
:107AF000E384E74EB7E700E03707400023A0E7182C
:107B000001000100629923000900FD1923A0E7107C
:107B100093F9F90FE39309EEE5BD97E7FF1F238B78
:107B2000071071BF130730026388E70C63E8E7169C
:107B300013074002638CE70A13070003E39CE7FA8C
:107B400097E7FF1F9387070DCA9703C70700A14751
:107B50001377F70FE31BF71483C7640097E6FF1F43
:107B60002380F6F897E7FF1F83C737D391C7FD57E8
:107B700097E6FF1F2386F6F697E5FF1F83C595D18D
:107B800097E7FF1FA38EB7F497E7FF1F83C787D040
:107B900013FB07089306000493F70706639FD74C6F
:107BA0009307A009638DF51663EAB7129307F005F2
:107BB0006386F54A930750096384F52A014497E7E1
:107BC000FF1F83C7F7F11547E392E736B7E700E0F9
:107BD0003707400023A0E71801000100B7860040E6
:107BE00023808602130680FC6F00500EFD5717E7B6
:107BF000FF1F2306F7EEFDBDFD5717E7FF1F230FFD
:107C0000F7ECCDBD17A50100130505B7977001006E
:107C1000E780806097E7FF1F9387C7FFCA9703C479
:107C20000700014B97ECFF1F938C4CDF1374F40F8C
:107C300017AD0100130DCDB463478B042945977030
:107C40000100E780604A854717E7FF1FA306F7DCBE
:107C500017E7FF1F230387DC17E7FF1F230CF7E855
:107C600037E700E0B70640002320D71801000100E5
:107C7000378600408347A60293F7370F2305F602A5
:107C80002320D71085BDB3876C0183C507006A85A3
:107C9000050B97700100E780404079BF854717E7E3
:107CA000FF1F230BF7D6B9B517E7FF1F130787F69A
:107CB0004A970347070097E6FF1FA38DF6C897E68C
:107CC000FF1F238AE6C817E7FF1F2305F7E21DB54C
:107CD000854717E7FF1F230FF7C629BD9307400A03
:107CE0006389F5349307200B6384F5369307100AF4
:107CF000E396F5EC838724000144E3D207EC97E791
:107D0000FF1F83C757B993F63700638A061A0546E3
:107D1000638AC62209466395C61A1D4755A217E510
:107D2000FF1F034545B7C94797ECFF1F83CCBCB67F
:107D300097E5FF1F83C545B617E4FF1F0344D4B57D
:107D40006315F510CD476392FC1093077008639C90
:107D5000F5021307300FB7170E006308E40013078E
:107D6000900DB7B704006314E40817E7FF1F232F33
:107D7000F7D6BE8517A50100130505A19770010070
:107D8000E780A03125BD93078008639DF500B30708
:107D9000804013F4F70FB7774600938787CDB3D7AA
:107DA0008702E1B793079008639AF500B307804014
:107DB00013F4F70F91679387C766D5B79307A008A9
:107DC000639BF500B307804013F4F70FB7173D002E
:107DD00093870790E9B79307B008639AF500B30754
:107DE000804013F4F70F9167938797D04DBF93F5B9
:107DF000F5078D47639BF500B307804013F4F70F39
:107E0000B7975B00938707D859BF8947639BF500F5
:107E1000B307804013F4F70FB7770B009387071B66
:107E2000BDBF8547639AF500B307804013F4F70F91
:107E3000DD67938767E3A5B7D28785F9B3078040ED
:107E400093F7F70FB3D7FA020DB797000000E7805A
:107E5000409FA285668597000000E780809EB9BBA1
:107E60009305610017E5FF1F0345E5A217E4FF1F17
:107E7000034474A297000000E78040AD93057100B1
:107E8000228597000000E78060AC3C0017E7FF1FE9
:107E90002328F7D6834761002304F100834771004C
:107EA000A304F100894717E7FF1F230BF7C283578D
:107EB000810017E7FF1F231FF79C094409B31547EB
:107EC00093F64700B336D00093F78703850685C342
:107ED0002146638BC7066146638AC7061306800284
:107EE0006388C706130680036393C700914717E6AC
:107EF000FF1F230FD6BE97E6FF1FA38BF6BE97E7A3
:107F0000FF1F2388E7BE17E7FF1F0347E798937615
:107F1000070497E7FF1F83C737988DEE1377770C19
:107F200093067008630CD7021377F7078D46631228
:107F3000D70CB307F040B7955B0093F7F70F938525
:107F400005D849A81947ADBF854755B7894745B7F3
:107F50008D4771BF930670086311D7021307300F66
:107F6000B7150E006389E7021307900DB7B504003B
:107F70006383E7021307700845BF9306800C631103
:107F8000D702B307F040B775460013F7F70F938792
:107F900085CDB3D5E70297E7FF1F23A9B7B4D9BBB7
:107FA0009306900C631CD700B307F04093F5F70FCE
:107FB00091679387C766B3D5B702F1BF9306A00C4C
:107FC000631DD700B307F040B7153D0093F7F70FD7
:107FD00093850590B3D5F5027DBF9306B00CE315EC
:107FE000D7F4B307F04093F5F70F9167938797D0D5
:107FF000D9B78946631BD700B307F040B7750B00AC
:1080000093F7F70F9385051BF1B78546631AD700E1
:10801000B307F040DD6593F7F70F938565E35DBF28
:10802000D28535FBB305F04093F5F50FB3D5BA0211
:108030009DB783C72400C18B99C7854717E7FF1FEA
:108040002303F7AAA5BE97E7FF1F238E07A8BDB697
:10805000854717E7FF1FA30EF7A88DB63C0017E76B
:10806000FF1F232FF7B80947930700032314F100DC
:1080700097E6FF1F2386E6A62DBD63940756A94702
:1080800063E5B74217970100130747588A05BA9569
:108090009C41BA97828717D4FF1F0344D47F894C31
:1080A0006306940D63E68C0685476303F408930723
:1080B000F00F17E7FF1F0347A7A263F6E70017E7D4
:1080C000FF1F230FF7A097ECFF1F83CC6CA1930732
:1080D000000413F4FC0F63F497011304000497E702
:1080E000FF1F9387E7B103AD070022862685EA8547
:1080F000B38C8C40229D97700100E780A0EE97E73B
:10810000FF1F238F979D97E7FF1F23ABA7AF45BCAA
:108110008D47630CF40A9947E31BF4F89797010025
:108120009387475517E7FF1F232CF7ACA94751B793
:1081300017E7FF1F034727B097E7FF1F9387479C69
:108140004946979501009385E55B630687009795FF
:108150000100938525573E8597700100E78080E8F0
:1081600017E7FF1F232EA7A8C947A1B797E6FF1F50
:1081700083C666AC054797E7FF1F938767986394AC
:10818000E6023E851306700297950100938505551A
:1081900097700100E78000E517E7FF1F2322A7A6DD
:1081A0009307700239B73E85130630049795010096
:1081B0009385054D97700100E780C0E217E7FF1F28
:1081C0002320A7A493073004EDB597D5FF1F83C5DF
:1081D000856C179501001305655C97700100E780B9
:1081E000C0EB054D97EDFF1F83CDEDA497D5FF1F85
:1081F00083C5656A179501001305455A6398AD0B51
:1082000097700100E78060E997D7FF1F83C7A768D1
:10821000B5CBE36EF4E8179401001304E452638CC9
:10822000B701179401001304A452638697011794B1
:10823000010013046453228597700100E78000FF5A
:108240001375F50F93071500860717E7FF1F23091E
:10825000F78A8D4717E7FF1FA304F78A97E7FF1FE9
:108260009387078A0147BE861376F70F89076365F0
:10827000A60297E7FF1F23A5D79897E7FF1F83C79D
:10828000278805BD979701009387074517E7FF1FCC
:108290002328F796914731BD3306E40003460600D4
:1082A000A380070005072380C7007DBF97700100EA
:1082B000E780A0DE97D7FF1F83C7E75DE1D7E368BC
:1082C000F4DE1794010013042445638CA70117946E
:1082D00001001304E444638697011794010013041A
:1082E000A445228597700100E78040F41375F50FCF
:1082F00093071500860717E7FF1F2303F7808D47B5
:1083000017D7FF1FA30EF77E97D7FF1F9387477FCF
:108310000147BE861376F70F8907E37CA6F4330680
:10832000E40003460600A380070005072380C7007A
:10833000D5B797D5FF1F83C50556179501001305BF
:10834000A54697700100E78040D597D7FF1F83C7E8
:10835000F77A93E7470017D7FF1FA301F77A83C780
:10836000240017D7FF1FA309F77889B817950100D4
:108370001305C54497700100E78000EA97D7FF1FF7
:108380009387877783C7070017D7FF1F2304F7500A
:1083900017D4FF1F0344C474333480000DB0179505
:1083A00001001305E54297700100E780E0E697D7EA
:1083B000FF1F83C7B77493E7070117D7FF1FA30FEA
:1083C000F77283C7240017D7FF1F2307F7726FF0D8
:1083D000EFFE179501001305E54097700100E78057
:1083E000A0E303C704007D8B51EFB787004003C7AC
:1083F00067021377C70B136727002383E70203C7BE
:10840000A7021377C70B136727002385E70203C76B
:10841000E7021377C70B136727002387E70203C719
:1084200027031377C70B136727002389E7028547C4
:1084300017D7FF1F2300F75217D7FF1F230EF75C34
:1084400017D7FF1F230CF76817D7FF1F2309F768FB
:1084500097D7FF1FA380075097D7FF1FA38E075AF8
:1084600097D7FF1FA38C076697D7FF1FA3890766BF
:1084700097D7FF1FA380076897D7FF1FA38D077AA1
:108480006FF0CFF389476312F70297D7FF1F83C7B7
:10849000A7409146638CD70863E0F604638EE70C2F
:1084A0006369F70A05476380E70EFD5717D7FF1F7B
:1084B000A308F76237074000B7E700E023A0E718FA
:1084C00001000100B78600401306F0FC2381C602BC
:1084D00023A0E7106FF00FE2130720086382E7087C
:1084E0006362F70213071008E391E7FC3787004047
:1084F0008347670293F7C70B93E727002303F7022D
:108500006FF0CFEB130730086389E70213074008C9
:10851000E39DE7F8378700408347270393F7C70BAE
:1085200093E727002309F7026FF04FE937870040F0
:108530008347270393F73707F5B73787004083470B
:10854000E70293F7C70B93E727002307F7026FF0C3
:10855000EFE6378700408347E70293F73707F5B721
:10856000378700408347A70293F7C70B93E727009D
:108570002305F7026FF08FE4378700408347A70297
:1085800093F73707F5B7378700408347670293F7BC
:108590003707ADB7179501001305C5259770010082
:1085A000E78080C797D7FF1F2386072ED5B317957F
:1085B00001001305252597700100E780E0C597D7D6
:1085C000FF1F2399072C97D7FF1F9387675103C479
:1085D0000700894763F3870009441374F40F6FF0B1
:1085E0000FDE13070002E392E7EC631B0B0A638FB5
:1085F000F500930720026383F50817950100130522
:10860000E52397700100E78040A945B51795010063
:108610001305052097700100E78000C00144179DF5
:108620000100130D2D20A14CB387840083C50700E2
:108630006A85050497700100E78020A6E31694FF81
:10864000178501001305856897700100E780C0BC9D
:1086500017D4FF1F0344442401E897D7FF1F238D3D
:108660000720014B6FF0AFD58947E310F4E485474D
:1086700017D7FF1F2302F7206FF04FD417D6FF1F25
:108680000346762197D5FF1F83C5E5201795010086
:108690001305C51997700100E78020A06FF00FD275
:1086A0006380F50693071002E399F5F497D5FF1F51
:1086B00083C5851E179501001305451997700100A4
:1086C000E780A09D97D7FF1F23AC975297D7FF1F36
:1086D0009387C741944383D7470017D7FF1F0347AA
:1086E000474117D6FF1F2327D61A1D4497D6FF1FD1
:1086F0002394F61A97D7FF1F2381E71A6FF02FCC28
:1087000097D5FF1F83C545191795010013058515DA
:1087100097700100E780609897D7FF1F238E07149A
:1087200097D7FF1F239807166FF02FF92547638F00
:10873000E7C89946378700406394D7022300870231
:10874000B7E700E0B706400023A0D71801000100FA
:10875000130600FC2301C70223A0D7106FF08FB9C6
:108760009306100A639FD70023008702B7E700E053
:10877000B706400023A0D71801000100130680FCB3
:10878000D1BF9306A009E381D7FE9306400AE38D8B
:10879000D7FC93062002639DD700B7E700E0B70639
:1087A000400023A0D7180100010023008702F9B779
:1087B0008546E384D7FE93070008E300FBFEB7E796
:1087C00000E0B706400023A0D718010001001306FF
:1087D00020FC23008702BDBF17D7FF1F0347573078
:1087E0006302F71E63E7E70295476300F7109947B6
:1087F000630AF704B786004023800602B7E700E06B
:108800003707400023A0E718010001001306A0FC71
:1088100075B99307F005630AF700930750096306DB
:10882000F70093071002E317F7FCB7E700E03707FC
:10883000400023A0E71801000100B786004013069E
:1088400020FC69B117DBFF1F034B8B299307000442
:108850005A8D63F46701130D000497D7FF1F9387A8
:10886000273A83AC07001374FD0F2286E685268520
:1088700097600100E7800077B3078B40669417D7B5
:10888000FF1F230FF72497D7FF1F23AB8736B78728
:108890000040630C0B022380A703B7E600E0370615
:1088A000400023A0C6180100010003C72702134798
:1088B00007042381E70203C727021377C70F238129
:1088C000E70223A0C6106FF0EFA22380070237E76C
:1088D00000E0B70640002320D7180100010013066E
:1088E00020FC2381C7026FF0AFB937870040834770
:1088F000370097D6FF1F83C6362093F70708D58F1A
:10890000A301F700B7064000B7E700E023A0D7189F
:10891000010001001306A0FC35BD97D7FF1F938708
:10892000672FCA9783C7070093F7F70FC1CF97D771
:10893000FF1F83C74730D9E717D7FF1F0347571AD1
:10894000930700026310F70883AD040017DDFF1FD3
:10895000034D8DF497DCFF1F83CC1CF417DBFF1F46
:10896000034BABF3E6876A87DA866E8697D5FF1FDF
:1089700083C585F017950100130545F09760010048
:10898000E780A07197D7FF1F23A2B71797D7FF1FC4
:108990002380A71797D7FF1FA38C971597D7FF1F83
:1089A0002389671597D7FF1FA38787ECB7E700E0F8
:1089B0003707400023A0E71801000100B7860040F8
:1089C0006FF04FA2B7E700E03707400023A0E71899
:1089D00001000100B786004015BD97D6FF1F83C672
:1089E00086250547639CE60429472381E70209475A
:1089F0002383E7022385E70297D7FF1FA38C070E87
:108A000097D7FF1FA3890722B7870040A3810700DC
:108A100017D7FF1FA302070E05472383E700B640C1
:108A2000264496440649F259625AD25A425BB25BD6
:108A3000225C925C025DF24D616182802947238154
:108A4000E70209472383E7022385E7022387E7023A
:108A50002389E70255B717D7FF1FA30EF7E06FE092
:108A60001FFF854717D7FF1F2306F7EE17D7FF1FF6
:108A70002304F7FA17D7FF1F2302F70617D7FF1FA4
:108A8000230FF7046FE0BFFE854717D7FF1F2303AF
:108A9000F7EC17D7FF1F2301F7F817D7FF1F230F96
:108AA000F70217D7FF1F230CF70217D7FF1FA303E7
:108AB00007EA17D7FF1FA30107F617D7FF1FA30F5A
:108AC000070097D7FF1FA38C07008280411106C6BD
:108AD00097000000E78080FBB787004023800700F5
:108AE000130740FC2386E7001307C004A386E700B2
:108AF00017D7FF1F130707DA2398E70017D7FF1FC1
:108B0000130747DD239AE70017D7FF1F1307C7E8AE
:108B1000239CE70017D7FF1F130747F4239EE700A6
:108B200029472381E70209472383E7022385E702D8
:108B30002387E7022389E702A3810700930600F851
:108B4000A380D700930690022380D700FD5623838D
:108B5000D7002381E7009306000537E700E0230BE9
:108B6000D740B70640002320D71003C7170013676C
:108B70001700A380E700B24097D7FF1F239E07F698
:108B800041018280411106C697000000E78000F095
:108B9000B787004023800700130700FC2386E70007
:108BA0003147A386E70017D7FF1F1307A7CE2398E7
:108BB000E70017D7FF1F1307E7D1239AE70017D75E
:108BC000FF1F130767DD239CE70029472381E70286
:108BD00009472383E7022385E702A3810700930661
:108BE00000F8A380D700930690022380D700FD569B
:108BF0002383D7002381E7009306000537E700E0D1
:108C0000230BD740B70640002320D71003C7170017
:108C100013671700A380E700B24097D7FF1F239D7B
:108C200007EC41018280F1679387072017D7FF1F68
:108C3000232EF7EA854717D7FF1F231BF7EAA14723
:108C400017D7FF1F2307F7EA97D7FF1FA38307EA6A
:108C500097D7FF1F238007EA97D7FF1F238E07C0F0
:108C600097D7FF1FA38907C0814717D5FF1F13059B
:108C7000E5C0FD5517D6FF1F130606C12947B306E9
:108C8000F5002380B600B306F600238006008507B2
:108C9000E397E7FE97D7FF1FA38507E497D7FF1F4A
:108CA000A38307E497D7FF1F238E07E297D7FF1F01
:108CB000238907E297D7FF1F238807E297D7FF1F73
:108CC000A38207E297D7FF1F238F07E0814717D6BC
:108CD000FF1F130626F34147B306F6002380060064
:108CE0008507E39BE7FE828017D7FF1F0347A7F4A2
:108CF00085476316F700170300006700E3E81703D2
:108D000000006700E3DC411122C406C617D7FF1F2D
:108D1000034767F285472E8613F4F50FAA8563177C
:108D2000F70417D5FF1F130525CB97600100E780D7
:108D3000602B97D7FF1F238107CEB787004023847E
:108D40008702B7E600E03706400023A0C6180100FE
:108D5000010003C7A7021377C70F2385E702B240BC
:108D6000224423A0C61001454101828017D5FF1F70
:108D7000130545BA97600100E780C02697D7FF1F0B
:108D8000238A07BCB787004023828702B7E600E04A
:108D90003706400023A0C6180100010003C7670280
:108DA0001377C70F2383E7025DBF411106C6970003
:108DB0000000E78080E7B240410117030000670030
:108DC000E3F2411106C697F0FFFFE78080BF97D717
:108DD000FF1F83C737B8A1CB97D5FF1F83C5A5B7A2
:108DE00089C917D5FF1F130525B797E0FFFFE78057
:108DF000605297D7FF1FA38F07B497D7FF1F238B0E
:108E000007CE37E700E0B70640002320D71801005F
:108E10000100378600408347660293F7370F23032C
:108E2000F6022320D710B2404101828041C9D9C542
:108E300097D7FF1F83C747CCD1C3011122CC4AC8A3
:108E40004EC656C25AC006CE26CA52C42E89AA8918
:108E50000144930A0004371B030063772403B3071C
:108E60008940C207C183BE8463F4FA0093040004FE
:108E7000C204C180130A1BD497D7FF1F83C787ADD5
:108E80009DE37D1A631C0A00F2406244D2444249C9
:108E9000B249224A924A024B0561828097F0FFFF55
:108EA000E78020B2D1BF338589002694A68542048D
:108EB00097000000E78060E5418045B7828097D742
:108EC000FF1F9387A7E918429C4383D645000345BB
:108ED000070083C5C700035646006396A50083D5E7
:108EE000E700638DD502011106CE2386A7002397E4
:108EF000D700B705CF00DC4B9385757D05077D1640
:108F00002EC2230001003AC42316C1002317D1004A
:108F100099C30A858297F24005618280828041115F
:108F200022C417A4FF1F1304A44D5C4C06C691CBAA
:108F3000C84B01C9B7E70400BC5782975C4C23AA11
:108F40000700B240224441018280DC4DDC4B81CFDE
:108F5000B7E70400904503A38705914517D5FF1F88
:108F6000034505E002838280B7E7040003A30705F9
:108F7000A14517D5FF1F0345A5DE02836D713C088F
:108F80003EC6B707E500232291103EC8AA843C08DC
:108F90003285232611103ECA23248110232021115B
:108FA0002E8997300000E780605A2A849795010047
:108FB00093854590177501001305856E9760010034
:108FC000E780A00DA285179501001305659B9760AA
:108FD0000100E780800C294597600100E780C01000
:108FE000B705CB009385757D680097100000E7807A
:108FF000E05FA285680097300000E7808047014766
:1090000081467000CA85268597200000E78060832E
:1090100005CD2A84979501009385C58917750100B0
:109020001305056897600100E7802007A285179562
:1090300001001305A59597600100E780000629450A
:1090400097600100E780400A8320C110032481104B
:1090500083244110032901105161828097D7FF1F9B
:109060009387C7CF18429C43797122D406D6034810
:10907000070083C807012A8483D6450003554600AC
:109080006396080183D82701638DD80223880701DE
:1090900005072399D7003708CC00DC4B1308787DEF
:1090A0003ACC1307F5FF42CA23080100231EE10052
:1090B000231FD10099C7080832C62EC482973246B2
:1090C000A245228597000000E78080EBB250225431
:1090D0004561828079713146977501009385054D10
:1090E000280006D697600100E780C0EF97A7FF1F12
:1090F00083D70731231B0100231C0100231D01001E
:10910000231E0100231F010099E3C167FD17231AE5
:10911000F10097A7FF1F83D7C72E91EB97D7FF1FAB
:109120009387C7C39C439C43DC4783D7070097A61C
:10913000FF1F9386E62C231BF100D84E83D74600F1
:10914000231CF1005C4B91CB97A7FF1F83C7B72B64
:1091500081EB97000000E780C0DCB250456182805F
:10916000FD1717A6FF1FA300F62A0356070183C7A2
:1091700006014C472800230FF10097300000E780DC
:10918000602C97D7FF1F938767BD9C430147978645
:1091900001009386A67B884330004C08971000009E
:1091A000E780206A5DD975B799C9B7E7040003A3C2
:1091B0000705A14517D5FF1F034585BA02838280A5
:1091C0005C4EDC4BB9CFB1CD411122C41775010003
:1091D0001305054D2E84978501009385E57206C61B
:1091E00097600100E78060EBA285178501001305F9
:1091F000E57397600100E78040EA29459760010028
:10920000E78080EEB7E704002244B24003A387055D
:1092100017D5FF1F0345C5B413064006914541010C
:1092200002838280411122C417A4FF1F1304041B70
:109230001C4C06C689C7DC4399C34C488297584CDE
:10924000B7E70400BC57484B82975C4CB2402244BD
:1092500023AA07004101828017A7FF1F1307071ADF
:10926000834707009306F00B850793F7F70F63E931
:10927000F60097A6FF1F2383F61803450700828098
:10928000930700F8FDB78357450099E37D55828029
:10929000011122CC17A4FF1F130484165C4C4AC88A
:1092A0004EC6DC4B52C406CE26CA56C2B2892E8A9E
:1092B0002A898DC7B7E70400FC5F829797D7FF1F05
:1092C0009387C7A79C431307301FB307F540715519
:1092D0006375F70697000000E780A0C49307D00DE0
:1092E0007D5563EC3705B7E4040093878900B858CF
:1092F000832AC401139507014181029723AAAA007A
:10930000484C584921E7978501009385E55D17751D
:1093100001001305E53897600100E78000D8178544
:1093200001001305656997600100E78000D72945B2
:1093300097600100E78040DB5D55F2406244D24413
:109340004249B249224A924A056182801387490004
:10935000B705CF002319E5009385757D310597107A
:109360000000E780A028484C83456900310597300C
:109370000000E7800010484C4E86D28531059730BA
:109380000000E780200C7146CA8517A5FF1F130552
:10939000250797600100E780E0C4FC5C8297032604
:1093A000C90097D7FF1F23ABA79811CABC4C8545AE
:1093B00017D5FF1F0345C59A82970145BDBF97008A
:1093C0000000E78060D1D5BF411106C622C426C285
:1093D00017D4FF1F1304C49897000000E78060B4FF
:1093E000B7E40400FC4C034504008545829703451F
:1093F0000400224403A3C405B2409244A1454101A4
:109400000283411126C297D4FF1F938424959C4068
:1094100006C622C44AC0D5C3DC43C5C35CC1230011
:10942000B5002A849785010093854547177501008B
:109430001305052797600100E78020C6294597603E
:109440000100E78060CA9C4023A4070023A2070014
:1094500097A7FF1F938787F8DC4FDC4B91C72955EF
:1094600097000000E78040DC97A7FF1F938747F92C
:10947000DC4FDC4B89C797000000E78020F537E917
:1094800004008327C905894517D5FF1F0345458D6E
:1094900082978327C905914517D5FF1F0345458C42
:1094A00082979C4003A3470163090300228522445D
:1094B000B2409244024941010283B24022449244A4
:1094C0000249410182800111328506CE22CC26CA92
:1094D0002E8497300000E7806007AA8497850100FA
:1094E0009385053F177501001305851B97600100E3
:1094F000E780A0BA03078400035664008355440044
:10950000A686178501001305E54497600100E780F2
:10951000C0B8294597600100E78000BD97A7FF1FED
:1095200083C727EC639D9700014597000000E78003
:10953000A0CF81450A8597000000E780C0ECF2408B
:109540006244D244056182806D71232481102326F8
:1095500011102322911093F745002E84638707147E
:109560003C083EC0B707E5003EC23C083EC4231796
:1095700001002318010023190100231A0100231BF5
:10958000010097A7FF1F83D767E599E3C167FD1720
:109590002316F10097A7FF1F83D767E491EB97C7C6
:1095A000FF1F9387A77B9C439C43DC4783D707001F
:1095B00017A7FF1F130787E22317F100544F8357A4
:1095C00047002318F100DC4AA1E797850100938545
:1095D0006534177501001305A50C97600100E7803D
:1095E000C0AB178501001305A54397600100E78014
:1095F000C0AA294597600100E78000AF13454400E9
:109600008320C11003248110832441105161828082
:1096100097A7FF1F83C7F7DC2555D9C3FD1717A6EA
:10962000FF1FA300F6DC03D6060183470701CC46E3
:109630000A85230BF10097300000E780A0E097C770
:10964000FF1F9387A7719C4317A7FF1F130707D915
:10965000978601009386062D88430A866C00971032
:109660000000E780001EAA8451D9978501009385E8
:10967000652A177501001305A50297600100E780B0
:10968000C0A1A685178501001305453A9760010022
:10969000E780A0A0294597600100E780E0A4268527
:1096A00097000000E78040B891BF93F725009DC761
:1096B000B7E70400BC4741468145280882972555F5
:1096C00097000000E78040B628089305F00F970048
:1096D0000000E78040D3134524001DB793F7150021
:1096E00081CB97000000E780209F1345140009BF3D
:1096F00093F78500014589D717A7FF1F0347B7D008
:1097000097A7FF1F9387C7CF0DC3D84F584B11CFD3
:1097100037E70400384F9047854517C5FF1F0345BD
:109720002564029713458400E1BD97F0FFFFE780B1
:10973000407FCDBF5C4D411106C688C317C7FF1FD0
:10974000232EF760B7E7040083A70708170500007A
:109750001305C5DF8297B24097C7FF1F2382A7601A
:1097600001454101828001113335A000A307A1000A
:10977000B7E7040083A7471706CE1306F100854517
:10978000130550308297F24005618280828041113A
:1097900022C406C697B7FF1F83C717A8054489EFE1
:1097A00097C7FF1F83C787E7014499E717B4FF1FD7
:1097B000034484A613441400228597000000E78028
:1097C000C0FA178501001305252D09E4178501004E
:1097D0001305852D2244B240410117630100670043
:1097E000C38B797122D4A30F010037E404008327CF
:1097F000841726D24AD006D6AA842E891305503063
:109800009305F10132C6829732468347F1019315E1
:109810000601C18185CB01452EC697000000E78077
:10982000C0F483274417B2454A86268582970545AA
:1098300097000000E78060F3B2502254925402591E
:1098400045618280832744174A8626858297EDB733
:1098500041119397050122C406C626C2C1872E84F2
:1098600063D40702B7E40400FC5417A5FF1F0345A7
:1098700025BC829719C1BC5482972165218DB240C5
:10988000224492444101828093F715008DC7B7E7C7
:10989000040083A7471A17A6FF1F130666B897C5CB
:1098A000FF1F9385A54C17A5FF1F034565B8829739
:1098B00013451400E9B793F725000145E9D397C78D
:1098C000FF1F83C7274C85E7B7E7040003A8871A63
:1098D0001307401F97A7FF1F83C787B5814613064D
:1098E0004006994517C5FF1F035545490298134582
:1098F000240071B797C7FF1F83D747486398A70213
:1099000017C7FF1F231DB74617C7FF1F231AC746D8
:1099100017C7FF1F2317D7462E861785010013058B
:10992000251FBE85175301006700237717850100A7
:109930001305851F176301006700038E0357450059
:1099400097C7FF1F83D787436318F702C167F917CB
:1099500017C7FF1F2324F74297C7FF1F23A2074201
:1099600097C7FF1F238A074097C7FF1F238C074015
:10997000170300006700E3E1178501001305C51A0E
:1099800017630100670043897D15954763E2A71CB3
:10999000178701001307C70E0A053A951C410111EC
:1099A00022CC06CEBA972E84828717850100130534
:1099B000251897600100E7802086A1A203C7250033
:1099C00099476311F7022E8597000000E78040F762
:1099D0008345640017850100130585169750010023
:1099E000E780A06B97B7FF1F2388078217850100C8
:1099F0001305C5167DBF03C7250095476319F702F8
:109A0000C16717C7FF1F03576737F91703D5A500AD
:109A10006309F702B7E7040083A7C7178297178582
:109A200001001305A51497500100E780E07E8547EB
:109A300017A7FF1F2302F77E178501001305851561
:109A40008DBF97C7FF1F239BA73283D7E50097C61B
:109A5000FF1F2396F63283D7050197C6FF1F239178
:109A6000F63283D7250197C6FF1F239CF63097C790
:109A7000FF1F23830730631BE502B7E70400BC4FD9
:109A8000096613060690894517A5FF1F0345459AE9
:109A900082970356E4008355A4001785010013053F
:109AA000250E97500100E780405F51B79307700F74
:109AB0002316F100B7E7040083A7870D17A6FF1F41
:109AC000034606976C0082974DF9854717C7FF1F1D
:109AD0002304F72A5DB7178501001305650CD1BD76
:109AE00083C5250091476392F50217850100130590
:109AF000A50C97500100E780207297000000E780D6
:109B000040C9F24062440561828099476392F50240
:109B1000228597000000E780A0E283456400178556
:109B200001001305E50197500100E7800057D1BF00
:109B30009547639AF50083471400E1F31785010008
:109B40001305C509BDB5178501001305A509E1BFBA
:109B500082803757315F97A7FF1F9387A78E130720
:109B600077D598C39356C50017870100130707F7E9
:109B7000BA9683C5060093568500BD8ABA9603C679
:109B8000060093564500BD8A3D89BA962A9783C63A
:109B9000060003470700238407002383D700A3831D
:109BA000E7002382B700A382C70097A7FF1F938710
:109BB000678A2383B700A383C7002384D700A384C5
:109BC000E7008280411106C697000000E780A0F8F8
:109BD000B7E7040083A7871417A6FF1F130686861E
:109BE000D54501458297B2404D4697A5FF1F938505
:109BF0006586130570304101170300006700A3BE9E
:109C000061712324811A37E4040083270408232682
:109C1000111A2322911A2320211B232E31191705F3
:109C20000000130525C3829717A9FF1F1309498058
:109C3000994785442300A900231CF1009785010062
:109C40009385C5E89307400617750100130545A5E0
:109C5000231CF1082308910097C9FF1F938969AC61
:109C600097500100E780604383D509001785010004
:109C70001305C5E497500100E7802042294597501D
:109C80000100E780604603D5090097000000E780E7
:109C900080EC8327441710088545130550308297C0
:109CA000832744171796FF1F1306C67ACD45130561
:109CB00070308297832744171796FF1F1306867705
:109CC000B5451305603082978327441730088945CE
:109CD00013051031829783274417300989451305EE
:109CE00020318297832744159305000A0D458297FA
:109CF000832744159305000A11458297A305910017
:109D00002306910002CD23080100230C01008327C4
:109D10008416300991451305704082978327841675
:109D20001306B100854513050040829783278416EA
:109D300070008545130510408297832784163008EC
:109D40008545130520408297832784161008854592
:109D5000130550408297832704157D5582978327EA
:109D600044137D5582977D5597A0FFFFE780E091D2
:109D70008327440C82979790FFFFE780406D8327ED
:109D800084141796FF1F1306E66BD545014582978D
:109D900089471306700F814528092306F100978033
:109DA000FFFFE780C0368D4713060008814528086D
:109DB000230CF1089780FFFFE78060359147230C63
:109DC000F100976701009387277F984383C7470077
:109DD0003AC8230AF10097C0FFFFE780E07A7000DD
:109DE0008545054597A0FFFFE78040913009930521
:109DF000700F094597A0FFFFE7804090300893055A
:109E000000080D4597A0FFFFE780408F100895459B
:109E1000114597A0FFFFE780608EC16717C7FF1F3E
:109E20001307C7F5F9171CC3232207001795FF1F57
:109E30001305C55F97A0FFFFE780208B8327C41D14
:109E400017C5FF1F130505F282973C48034509001B
:109E5000854582978320C11A0324811A8324411ADD
:109E60000329011A8329C1195D618280C16717C85E
:109E7000FF1F0358A8F0F9176301F8083DCDB5CDD1
:109E8000011126CAB7E4040083A7841222CC2E86CF
:109E90002315B10006CE2A8401478146ED4542854F
:109EA00082972AC611ED17850100130565C49750E6
:109EB0000100E7806036F2406244D244056182804E
:109EC000FC440356A100A28582972C0017C5FF1FF2
:109ED0000355C5EA97A0FFFFE780E08D69DD178590
:109EE0000100130525C297500100E780E03283A7E7
:109EF000C412ED45280082977DBF82800DC585473D
:109F00001797FF1FA30DF7529797FF1F238A07523A
:109F100035469795FF1F9385E5511305603017036C
:109F200000006700438C9797FF1FA38A0750E9BF83
:109F300097C7FF1F83C707E5A9EFC16717C7FF1FB3
:109F40000357C7E3F9176306F7044111854722C495
:109F500017C7FF1F2308F7E237E404007C4C06C64E
:109F600089451795FF1F0345A54C82970323841A43
:109F70002244B2409797FF1F83C7874B17C5FF1F27
:109F80000355C5DF1307401F8146314699454101FE
:109F9000028382806D7123248110232611102322D5
:109FA0009110328401CD8947630AF5028320C110E4
:109FB00003248110832441105161828017850100A0
:109FC000130505C3AE8497500100E780E024A28505
:109FD000268597B0FFFFE7802063C9BFB7E704007D
:109FE000FC472800829717850100130525C197506B
:109FF0000100E78060228347810039C41307000B0A
:10A000006380E7021387A7051377F70F8D4663ED8B
:10A01000E602A285280097C0FFFFE780A0D679B7A7
:10A020008547E3F587F8834591001775010013050F
:10A030006598B335B00097A7FF1F2387B7069750E1
:10A040000100E78080059DB703479100A207B9662C
:10A05000D98F1387E6556384E70C636DF7042D678A
:10A060001307B755638FE708636AF700296713077B
:10A07000A755638FE708A2852800A1BF31671307A2
:10A08000C7556388E70635671307D755E395E7FE9D
:10A090008947E3FD87F097000000E780A0E993057A
:10A0A000E4FFC205C1811305A1009790FFFFE7807F
:10A0B0002013EDBD3D671306F7556389C706636D31
:10A0C000F6009386E665E398D7FAA285280097C044
:10A0D000FFFFE7804010D9BD9306F766638DD70474
:10A0E0001307F777E399E7F897C0FFFFE780603B36
:10A0F00075BD0146A285280097C0FFFFE78020F4C8
:10A1000075B5A285280097C0FFFFE780600179BD83
:10A11000A285280097C0FFFFE780C00041BDA2854F
:10A12000280097C0FFFFE780000249B597C0FFFFF6
:10A13000E7808013A5BD97C0FFFFE7802019BDB55C
:10A14000C16717C5FF1F035565C3F9176307F500FE
:10A15000B7E7040003A3C7170283828017F3FFFF4A
:10A16000670023631783FFFFE702C3F52A840845CE
:10A170002E89B28919C900C1971500009385A5865B
:10A18000610597300100E780600481447D5A971093
:10A190000000E780E03963C7A40481449710000001
:10A1A000E780003A63C8A40497C7FF1F9387C7BD21
:10A1B0009C43DC47B307F94091872302F400638393
:10A1C00009048327C900B307F4409587A302F4006C
:10A1D0001C4C89C79C4799C3228582971783FFFF30
:10A1E000670083F15C44139714008504BA972390A9
:10A1F000470171BF1C48139714008504BA97239038
:10A20000070069BF832789000547B307F440958796
:10A21000A302F40083570400638EE7028DC309474D
:10A220006384E7040D47E395E7FA97870100938776
:10A23000A7EF1CCC97870100938707F011A8978799
:10A2400001009387E7B51CCC97870100938747B639
:10A250005CC8BDBF97870100938787A11CCC9787F7
:10A2600001009387E7A1EDB797870100938787F0F7
:10A270001CCC978701009387E7F0D9BF95E517833A
:10A28000FFFFE702C3E50046184483479400758347
:10A290009D8B6317F70097100000E78060B448C4F7
:10A2A0001783FFFF6700E3E582801783FFFFE70264
:10A2B00063E113893500C16442094111AA8901444F
:10A2C000F11413590901054A2EC697100000E780C2
:10A2D0002026B2456348A400014541011783FFFFD2
:10A2E000670083E183A7090013171400BA9783D787
:10A2F00007006388B7006394970063742A0105041C
:10A30000E1B70545D9BF1783FFFFE702C3DAAA8982
:10A310002E89328BB6843A8ABE8A97A00000E780E5
:10A3200000FE71C9268597200000E780C00C8D478C
:10A3300063E7A7007D551783FFFF670043DB83DBDF
:10A34000440097100000E780A0242A8497100000A2
:10A35000E78040259307740031443305850263CDBF
:10A36000A70297100000E780A02297100000E78066
:10A3700020222A8497100000E780C02293077400EF
:10A3800031443305850263C3A70497100000E780BA
:10A3900020209307450029A897100000E78080201F
:10A3A000330585021307F0179307C017E35FA7FA79
:10A3B0002D55E3C277F963040B02D6865286A68533
:10A3C0004A8597200100E78000BDB5B797100000CF
:10A3D000E780401D330585029307C5FFD1BF832762
:10A3E00049001385C90083D5270097000000E78046
:10A3F00000EC61F581B769553DBF97C7FF1F2397F3
:10A40000A79897C7FF1F93872798904381470C46CB
:10A410003307F500420741836393B70082805446B7
:10A42000139847008507C2962390E600D5B797C7D3
:10A43000FF1F938767959C4303C58700828017C5DC
:10A44000FF1F0355A59482801783FFFFE70223C9EE
:10A45000C1671387D7FF630BE502636AA700F11793
:10A460006300F50201451783FFFF670083C9138767
:10A47000E7FF6302E502FD171D8D13351500E5B7F3
:10A4800097500000E780A0297D15C5BF97500000B8
:10A49000E78020FED5BF97500000E78040FCEDB775
:10A4A0001783FFFFE702A3C34111AA8401442EC60C
:10A4B00097100000E780C008B2456348A40001453A
:10A4C00041011783FFFF6700C3C39C4813151400A5
:10A4D0003E9583570500E385B7FE0504C9BF0348D1
:10A4E0005500814693F7F60F63E5070181473E85E6
:10A4F0008280584593975600BA9703D72700631672
:10A50000B70003D70700E304C7FE8506E1BF834613
:10A51000450001479377F70F63E4D700814711A8FF
:10A520001C45131657000507B29703D60700E3131F
:10A53000B6FE3E8582801783FFFFE702A3B893171C
:10A540000501C18797CAFF1F938A0A84635BF008DD
:10A5500083A70A00C0479C4703570400198D420592
:10A5600041816368F500014422851783FFFF67007E
:10A57000A3B812052A94CDBFDC4713944900014AC1
:10A580003E94834744006341FA02014A83475400E2
:10A590006349FA028509C20993D9090183A70A0010
:10A5A0009847E3EBE9FCC1B71C4413195A00A68590
:10A5B0003E994A8597000000E780C0EE05E1050A54
:10A5C000C9B75C4413195A00A6853E994A8597007D
:10A5D0000000E78020ED19E1050A4DBFE30C09FA00
:10A5E00061B7AA8481495DBF1783FFFFE70223AFEC
:10A5F0001C452A8481E79307C5001CC51C4423120F
:10A6000004001CC09307F00F63EDB70093F5F50F3E
:10A61000228597200000E780C0E51783FFFF6700D1
:10A6200043AE93940501C167C18063F9F500A68527
:10A63000228597200000E780E0E8C5B7C18193F547
:10A64000F50F228597200000E780A0E2A6852285ED
:10A6500097200000E780E0E3C9B797B7FF1F938713
:10A66000A772884382801C4599C797B7FF1F23AD07
:10A67000A770014582807D55828097B7FF1F938721
:10A68000A770984383474500484792073E958280CC
:10A690001783FFFFE702A3A4617100451C183EC6A3
:10A6A000B70780013EC81C183ECA8357440002CE3B
:10A6B00002D002CC231EF100834784002A8902D2F3
:10A6C0002301F1023C083ED402D697000000E78047
:10A6D00000FB835705002316F10297500000E78026
:10A6E00040C72307A1025C4003556400F18313F7C0
:10A6F00017008347F10252055181F99BD98FA307B7
:10A70000F10297100100E780607839CDAA840355E3
:10A71000050097A00000E78060BF83D704002AD21D
:10A720006800231CF10083D72400231DF1001C487E
:10A7300003D647008C4397200000E780A0D08347D2
:10A74000B400CA86177601001306064C8117A305CC
:10A75000F4006C00481097200100E780C0835D6121
:10A760001783FFFF6700E3992155D5BF1C45B1CF83
:10A7700003C5A700894613576500630BD7028D46B2
:10A78000630ED70285466300D702130740063305E0
:10A79000E50203C7B700418B15CB83C7B700BD8B5C
:10A7A0003355F54082801375F5031307803EC5B716
:10A7B00009671375F50313070771D1BF3727090020
:10A7C0001375F5031307077CD9B7014582801783FA
:10A7D000FFFFE702C39003A98500630C09048347C8
:10A7E000B900AE8493F7070E85C30345990093051E
:10A7F00020030D810505B305B50288446105973036
:10A800000100E780C0AC35A02E8597000000E780EE
:10A8100020F62A8419CD97000000E780605C83252C
:10A82000C900B307B54063FA87002E94B305A4406E
:10A83000E9F51783FFFF6700C38C85457DBF17834C
:10A84000FFFFE702C3892A8403D50500011132C640
:10A8500036C43AC22EC002CA02CC02CE97A0000073
:10A86000E780C0AA82452ACA22852ECC9700000024
:10A87000E780E0E003570500231EE1009750000049
:10A88000E78020ADA24632469247230FA1003687CB
:10A890004C08B2862285014697000000E780E0A6BA
:10A8A00005611783FFFF6700C3851783FFFFE7027A
:10A8B000038361711C183EC6B70780013EC81C188F
:10A8C0003ECA3C0800453ED4AA8402CC02CE02D047
:10A8D00002D202D697000000E78060DA83570500B5
:10A8E00035592316F10297500000E78080A6230710
:10A8F000A10209C48357440081EB21594A855D6157
:10A900001773FFFF6700E37F035564005205518111
:10A9100097100100E78080572A8965D18347B400EA
:10A9200093F7070E99C71305840197300100E7805C
:10A93000409C83574400231EF10083478400230179
:10A94000F1025C4003550900D98313F707088347D8
:10A950001102231CA10093F7F707D98FA300F1027E
:10A9600083572900231DF1005C40F18313F7170082
:10A970008347F102F99BD98FA307F10297A000004A
:10A98000E780C0982AD235D983479400680013978E
:10A9900057008347B400FD8BD98FA305F4001C48F2
:10A9A00003D647008C4397200000E780A0A9A68724
:10A9B0001777010013074725740005464C102685BC
:10A9C00097000000E78060942A890DD98347B4007E
:10A9D000A685FD8BA305F40097000000E78060DFEB
:10A9E00031BF1773FFFFE702836F832485FE2A843C
:10A9F0004111268597000000E78080D7834734FF08
:10AA000093F7070E8DCB2AC6268597000000E780B6
:10AA100060C809CD834734FFB245FD8BA309F4FE1E
:10AA200091C5228597300100E780608A4101177344
:10AA3000FFFF6700036D7DD98327C4FF26858297BA
:10AA400075F5834734FF93F7070E91C7228597303A
:10AA50000100E780008A032584FE97000000E7805C
:10AA600000E5E9B71773FFFFE70263649C414111FA
:10AA70002A8903C7070089472E849356670063809D
:10AA8000F6040D466388C6049307F0076304F702D3
:10AA90002E8597200000E78060ABAA848149C16BB6
:10AAA000130C490097B7FF1F9387072E9C439847C5
:10AAB00063E4E90441011773FFFF6700036303D7F1
:10AAC00045008547E3F8E7FE2E8597200000E780E4
:10AAD00040ADE1B703D74500E3FEE7FC2E859720A4
:10AAE0000000E780A0A6AA84228597200000E780C6
:10AAF00000A8C204C98C5DB7DC470355A900139AAE
:10AB000049003E9A93170501C187635DF0008357A2
:10AB10000A006397A70263E774038327CA00034D03
:10AB20005A002DA0A1672167A98F1307F7EFE374DF
:10AB3000F7FE6397090097000000E780209161FD10
:10AB400085098DB783278A00034D4A00835DA900DC
:10AB500003576900216A138BC7003AC6814A33CA7A
:10AB60004D01631E5D0197B7FF1F938767229C43CA
:10AB7000E1DBA2866286814526858297D1B7A167EF
:10AB80009387F7EF930C4BFF63F24703B2455A8567
:10AB900097F0FFFFE780A0710DC103278B001047DE
:10ABA00009CE10436382C4023107D5BFEE856685A6
:10ABB00097000000E780008F71F993861A0093FADE
:10ABC000F60F130B0B0271BF835644005C43E3E99D
:10ABD000F6F622853AC697200000E7802081A1671B
:10ABE0009387D7042A8A035D4400324763E89700BD
:10ABF0008347D90093E707F8A306F9001C47668549
:10AC00002286E2858297C1670844FD17337AFA00ED
:10AC1000529508C02312A40125B797B7FF1F938749
:10AC2000A7169843814715C31447814763FFD50092
:10AC3000939745004C47BE9519C903C755008147F6
:10AC40006375E600DC451606B2973E85828003C731
:10AC500045008147E37BE6FE16069C45F5B7177372
:10AC6000FFFFE7022346AA892E8A814497BAFF1F75
:10AC7000938A8A1183A70A00984763E6E400177352
:10AC8000FFFF67006347DC471394440001493E948B
:10AC900013BB140083474400634BF900014913BB05
:10ACA000140083475400634FF9008504E1B708445A
:10ACB000931759005287DA860146A2853E958299FC
:10ACC0000509C9BF4844931759005287DA860546DB
:10ACD000A2853E9582990509E9B71773FFFFE70240
:10ACE0000340814517F5FFFF1305054897B7FF1F80
:10ACF000239E070897000000E780A0F61773FFFF68
:10AD00006700234097B7FF1F938707089C4395C3AD
:10AD10001773FFFFE702A33C814517F5FFFF1305FB
:10AD2000A54497000000E780C0F31773FFFF67009A
:10AD3000433D82801773FFFFE702C33837E4040006
:10AD40008327841241112315E100AE893289368AA6
:10AD50003A8681460147ED45AA8482972AC621C9D1
:10AD60000356A100D28597400100E780A0278327E2
:10AD7000C413CE8526858297058905C98327440D8E
:10AD80002314210101462C00268582972A8401C9BB
:10AD9000B7E7040083A7C712ED45280082972285F4
:10ADA00041011773FFFF670023354944D5B7655448
:10ADB000FDB75C41FD175CC182801773FFFFE7029E
:10ADC0000332B7E70400FC5F829795473305F5022D
:10ADD00081450D811773FFFF6700A3321773FFFFD3
:10ADE000E702E32FB7E70400FC5F8297954733053E
:10ADF000F5020D811773FFFF6700A3301773FFFF84
:10AE0000E702E32DB7E7040083A7870B035505008E
:10AE100082971773FFFF6700C32E1773FFFFE702C8
:10AE2000032C035505003287AE861786FF1F035695
:10AE3000866897B5FF1F9385E5F597000000E780CA
:10AE4000A0EF1773FFFF6700C32B1773FFFFE70225
:10AE50000329B7E7040083A7C71782971773FFFF7B
:10AE60006700232A1773FFFFE7026327B7E7040091
:10AE700083A7871397B5FF1F9385C5F18297014577
:10AE80001773FFFF6700E3271773FFFFE702232510
:10AE9000B7E7040083A7C71F81451785FF1F035528
:10AEA000855D82971773FFFF6700A3251773FFFF68
:10AEB000E702E322B7E7040083A7871397B5FF1FD4
:10AEC000938545EE829701451773FFFF6700632363
:10AED0001773FFFFE702A320B7E7040083A7C71F8C
:10AEE00081451785FF1F0355055F82971773FFFF85
:10AEF000670023211773FFFFE702631E2E859780EB
:10AF00000000E780C0B297800000E780C0EF1773B1
:10AF1000FFFF6700031F1773FFFFE702431C9780C3
:10AF20000000E780C0F91773FFFF6700831D5C49CD
:10AF3000E1175CC95CC583572501A1072319F500FA
:10AF400083570501A1072318F5008280F1473305D7
:10AF5000F50297B7FF1F9387E7E69C433E958280F3
:10AF60008D476315F60803D74600854763F0E70869
:10AF70001773FFFFE702A316368536842E899710D4
:10AF80000000E780A05C29C98357440093140501A1
:10AF9000C18063E39704228597100000E780005B7F
:10AFA000FD14231294009307A0026300F502930797
:10AFB000B0026307F50293079002631FF500228534
:10AFC00097000100E780A08801A80146CA85228574
:10AFD00097A00000E78040B31773FFFF670063127C
:10AFE000228597100000E7806007FDB7828097B642
:10AFF000FF1F938666DD9C42014599CF9843D4425A
:10B0000017B6FF1F2322E6DC6396D70097B6FF1F13
:10B0100023AEE6DA1385C7FE82801773FFFFE702CF
:10B02000030C97000000E780A04B714433058502B4
:10B03000914597900000E78000EC11E56555177386
:10B04000FFFF6700030C97B7FF1F23ABA7D697003E
:10B050000000E780E04833058502914597900000A5
:10B06000E78060E961DD97B7FF1F23ADA7D49700A4
:10B070000000E780E04697B7FF1F239DA7D2970007
:10B080000000E780E04597B7FF1F2396A7D2977788
:10B0900001009387A7BC17B7FF1F2321F7D297079B
:10B0A0000000938707E917B7FF1F2327F7D0014553
:10B0B00079B71773FFFFE7028302AA8517B5FF1F51
:10B0C000130545CF97100000E780605F1773FFFFFF
:10B0D000670023031773FFFFE70263009700000078
:10B0E000E78060FD97100000E780E05E97B7FF1FE4
:10B0F000938787CD9C4391CF1387C7FE19CB83D508
:10B10000C7FF17B5FF1F1305A5CC97200100E780E7
:10B11000001C1773FFFF6700C3FE1773FFFFE702F2
:10B1200003FC97000000E780C0EC09CD8347850051
:10B130002A8493F7070499EB0355E5009700000074
:10B14000E78080F91773FFFF6700A3FB8347C50003
:10B150009304450117B9FF1F130909C785E3832726
:10B1600009005CC997B7FF1F23A097C68327490032
:10B17000F1FB97B7FF1F23AB97C4E9B7FD17230671
:10B18000F500610597800000E780A0D9830784005F
:10B1900063CB07048347840093E707F82304F40094
:10B1A000B7E704009C5F82974205A9474181337548
:10B1B000F5028347840093F707FCC98F2304F4004A
:10B1C0008347D4003E951C402318A40089CF9843A0
:10B1D00019CB8347C4005040814585073305F502EC
:10B1E000420541810297832709005CC897B7FF1F7A
:10B1F00023AC97BC8327490089E797B7FF1F23A794
:10B2000097BC8347C4009DDF8355040117B5FF1F1A
:10B21000130505BC97200100E780600B25B7177365
:10B22000FFFFE702C3EB97B7FF1F9387A7DF9C479A
:10B2300001448583858B85E3AE84B2853A86971079
:10B240000000E780204F2A8419C597100000E7808E
:10B250006045829408CC22851773FFFF670063EA7C
:10B260001773FFFFE70203E641112E8932C6AA8950
:10B2700097000000E780C031324713060502CA86F6
:10B28000970500009385C5CC17B5FF1F130585B240
:10B2900097000000E780E0F82A8425C99304C500E0
:10B2A00097000000E780E0411946AA85268597109F
:10B2B0000000E78020198545268597100000E7806B
:10B2C000001517750100130525974E958345050058
:10B2D000268597100000E780C0195C4831468145FB
:10B2E000A1075CC85CC483572401E1172319F4004B
:10B2F00083570401E1172318F4001C4C3E85977016
:10B30000FFFFE780C0E0A3042501228541011773F8
:10B31000FFFF670063DE1773FFFFE70243DC4111A5
:10B32000AA842EC632C497100000E780003A004D70
:10B33000B2452246834784000CC050C093F7F70300
:10B3400093E707042304F4002318040026859710CC
:10B350000000E780203583479400A9462317A40006
:10B3600013D7370005073307D7029D8B85072306C0
:10B37000F400A306E40083C70401D8488507230F1F
:10B38000F7FE17B7FF1F130727A45843232A04000B
:10B390009307440129E317B7FF1F2329F7A217B723
:10B3A000FF1F2323F7A217B4FF1F130464A22285F3
:10B3B00097200100E780E0E31C44858B5D8D19E553
:10B3C0008145228597200100E78060F041011773D5
:10B3D000FFFF670003D31CC317B7FF1F2328F79E87
:10B3E000D9B71773FFFFE70283CF97050000938556
:10B3F00065B7014597000000E78000B0014517736D
:10B40000FFFF670003D01773FFFFE70243CD9700EC
:10B410000000E78080B01773FFFF670083CE83478B
:10B42000C500A5E31773FFFFE70263CB2A8403552A
:10B43000E50097000000E78000C821C18347840031
:10B4400093F7F7FB2304F4001C4091C7DC4381C74A
:10B450004C400145829797000000E78080B917B5FE
:10B46000FF1F1305E59697200100E78080E803554C
:10B47000E40097000000E78020C61773FFFF670015
:10B4800043C882801773FFFFE70263C597B7FF1FAA
:10B490009387879397050000938565C817B5FF1FAD
:10B4A0001305059323A0070023A20700972001009E
:10B4B000E780C0D11773FFFF6700A3C41C4D91CF75
:10B4C000DC4381CF1773FFFFE70263C183450700A9
:10B4D00082971773FFFF6700C3C2828097B7FF1F71
:10B4E000938747919C4303C50700828097B7FF1F4E
:10B4F000938747909C4303C51700828097B7FF1F2F
:10B500009387478F9C4303C52700828097B7FF1F0F
:10B510009387478E9C4303C54700828097B7FF1FE0
:10B520009387478D9C4303C53700828097B7FF1FE1
:10B530009387478C9C4303C55700828097B7FF1FB2
:10B540009387478B9C4303C56700828097B7FF1F93
:10B550009387478A9C4303C57700828097B7FF1F74
:10B56000938747899C4303C58700828097B7FF1F55
:10B57000938747889C4303C59700828097B7FF1F36
:10B58000938747879C4303C5A700828097B7FF1F17
:10B59000938747869C4303C5B70011E11D45828010
:10B5A00097B7FF1F938707859C4303C5C700828019
:10B5B00097B7FF1F938707849C4303C5D7008280FA
:10B5C00097B7FF1F938707839C4303C5E7008280DB
:10B5D00097B7FF1F938707829C4303D5070182809B
:10B5E00097B7FF1F938707819C4303C5270182807C
:10B5F00097B7FF1F938707809C4303D5470182803D
:10B6000097A7FF1F9387077F9C4303D5670182801D
:10B6100097A7FF1F9387077E9C4303D587018280EE
:10B6200097A7FF1F9387077D9C4303C5A7018280CF
:10B6300097A7FF1F9387077C9C4303C5B7018280B0
:10B6400097A7FF1F9387077B9C4303C5C701828091
:10B6500097A7FF1F9387077A9C4303C5D701828072
:10B6600097A7FF1F938707799C438857828097A7E6
:10B67000FF1F938727789C4303D5C702828097A733
:10B68000FF1F938727779C4303D5E70219E1130532
:10B69000800C828097A7FF1F9387C7759C4303C5C3
:10B6A0000703828097A7FF1F9387C7749C43C85BDB
:10B6B000828097A7FF1F938767738843828097A72D
:10B6C000FF1F9387E7728843828019E17D5582804E
:10B6D000F5DE984265DFFDD917B7FF1F1307879482
:10B6E0001847AA877155058B631D072403C50700FA
:10B6F0001547E37DA7FC03C737001305F0057D1749
:10B700001377F70FE364E5FC03C35700E30003FC82
:10B7100083C86700E38C08FA03C7770049457917A7
:10B720001377F70FE364E5FA03C7A7001148130581
:10B73000F7FF1375F50FE36BA8F803CE97000D48DC
:10B740001305FEFF1375F50FE362A8F803C8B700F1
:10B750006309080065181378F80F1305600DE36797
:10B7600005F703C5C700794879151375F50FE36F21
:10B77000A8F403C8D7000D457D181378F80FE367C8
:10B7800005F503D80701930E4017511842081358C6
:10B790000801E3ED0EF303C8E7007D181378F80FF6
:10B7A000E36605F303C827017D181378F80FE36FEC
:10B7B00005F103C88700C54E75181378F80FE3E745
:10B7C0000EF103D86701856E938EBEE06D184208B6
:10B7D00013580801E3EC0EEF03D847016D18420837
:10B7E00013580801E3E40EEF03D8870179184208E3
:10B7F00013580801E36C05ED03C8A7017D18137801
:10B80000F80FE36505ED03C5B7011D487D151375F8
:10B81000F50FE36DA8EA03C5D701714879151375D3
:10B82000F50FE365A8EA03D5E7011308E00F7D15DE
:10B8300042054181E36CA8E803C507024948791530
:10B840001375F50FE364A8E8C85301C937C834007D
:10B850005915130858BFE36BA8E603A8870237C53C
:10B860003400130555BF5918E36205E717A5FF1FFC
:10B870002320C55803C6050117A5FF1F232CF55625
:10B880000545E375C5E403D82501D04933760603A1
:10B89000E31E06E203C61501E30A06E217A6FF1F30
:10B8A0002326B65483C5270001466387A50003C637
:10B8B0001700F1453306B60283C707039305C0029C
:10B8C00072971A071307C70516031A979608469723
:10B8D000B387B70241553E9732974207418363626F
:10B8E000E8061763FFFFE702837F36859780000035
:10B8F000E780806B97000100E780004B2A8497A0C7
:10B900000000E780605D2A9497F00000E7804029FE
:10B910002A9497900000E78080842A9497F0FFFF94
:10B92000E780E06F2A9497400000E78000972A9410
:10B9300097700000E780809F22951763FFFF6700E4
:10B94000437C82801763FFFFE70263794111A307FD
:10B95000A10097A00000E78080C89305F1001705BB
:10B9600000001305E5B597F0FFFFE780802F014544
:10B9700041011763FFFF6700C3781763FFFFE7020A
:10B98000837317A4FF1F1304E46903288400795903
:10B990009368180097A4FF1F23AA1469137818004E
:10B9A00063100802BA84BE89368B328A2E89AA8A2D
:10B9B00097F0FFFFE780E0A77D15269519E531593F
:10B9C0004A851763FFFF6700837297F0FFFFE780E8
:10B9D00040A67D152695A167E353F5FE97B7FF1F97
:10B9E0009387479B98433E8C814B01CB014597F051
:10B9F0000000E7800047933B15004A85DA865686AB
:10BA0000D28597900000E780A0502A8911CD1C4470
:10BA1000F99B17A7FF1F232BF76083270C00CDD3BB
:10BA2000E3800BFA829769BF268597A7FF1F23AD96
:10BA3000075E97F0FFFFE780809C4146CE8517A503
:10BA4000FF1F1305A56797300100E780A05997D025
:10BA50000000E780209C0325040B97D00000E780BE
:10BA6000E09F054597D00000E780E0A605459700D8
:10BA70000000E78060EDA9B797A7FF1F9387875A5B
:10BA80009C47858BEDC71763FFFFE702436517A54A
:10BA9000FF1F1305E56097A7FF1F23A5075897A76A
:10BAA000FF1F23A3075897A7FF1F23A1075897201D
:10BAB0000100E780008497500000E780C0F89710ED
:10BAC0000100E780804F97100100E780805597A71D
:10BAD000FF1F9387A7539C4391C70545978000009C
:10BAE000E780202397A7FF1F9387073C9C4399C7B4
:10BAF00041657D1597700000E78020A597F0000054
:10BB0000E780C04097D00000E780609297A7FF1FB2
:10BB1000938747669C43139717016356070097F076
:10BB20000000E780E0AF97A7FF1F23A9075897A75A
:10BB3000FF1F23A7075897A7FF1F23A5075897A7FD
:10BB4000FF1F23A3075897000000E780008C970091
:10BB50000000E780A07597F0FFFFE780401897F09E
:10BB60000000E78020D91763FFFF670083598280B8
:10BB700097A7FF1F9387074B8843828097A7FF1FD4
:10BB80009387474AC8438280B7E7B000938707503E
:10BB900063E1A70297A7FF1F9387C748D843FD57C4
:10BBA0006367E50097A7FF1F23A0A74881473E854D
:10BBB0008280B957EDBF1763FFFFE70243529780BA
:10BBC0000000E780A07497800000E780007717638B
:10BBD000FFFF670003531763FFFFE702A34E2A84AA
:10BBE0009304140201112E85B289A685214636C61A
:10BBF0003A8997300100E780803C0DE9B246380869
:10BC00002686CE851305940497500000E780A04057
:10BC100021462C084A8597300100E780403A1335C9
:10BC2000150005611763FFFF6700034D0145D5BF90
:10BC30001763FFFFE702A34A9305450617A5FF1FF9
:10BC40001305851B97100100E78060681763FFFFED
:10BC50006700234B1763FFFFE702634841112EC6BD
:10BC600097F0FFFFE780C017B24588C14101176315
:10BC7000FFFF670003491763FFFFE702A344AA849D
:10BC80002E8497800000E780406BAA898545228535
:10BC900097000000E780E07D83C7E40113899408E2
:10BCA00099E313890403CE85228597000000E7807D
:10BCB000407C214693051902228597000000E78009
:10BCC000607897A7FF1F9387E7358C4322859710ED
:10BCD0000000E780C0822146938584022285970078
:10BCE0000000E78020761763FFFF6700E3401763DB
:10BCF000FFFFE702433C397197F00000E78020B472
:10BD00009305400661E997800000E780405F630289
:10BD1000051497A7FF1F83C7E70F13B7170097A650
:10BD2000FF1F2389E60E014499CFC16417A9FF1FA5
:10BD30001309492F9309400EFD1497000000E78076
:10BD400020836342A40A97F0FFFFE78060094169FE
:10BD5000B7290900096AFD7A2A8B81447D199389E4
:10BD6000F97B130A0A71938A8AC797000000E7805B
:10BD7000208063D7A4041304400EB387840217A75E
:10BD8000FF1F1307272A0324070B3E948357C40180
:10BD90006382270B18403307EB4063EAE9008347CF
:10BDA00044008507B3874703D6976365F7080146C4
:10BDB0008145094597F0FFFFE780C04AAA8B29E536
:10BDC00097400000E780C08285476317F5068965C4
:10BDD0009385057117A5FF1F130505029710010034
:10BDE000E780E04E95A0B30734030327090BBA9709
:10BDF00003D7C7016308970003C75700A382070052
:10BE00002382E700050415BF9305C500228597002E
:10BE10000000E78080E65E852286976501009385B5
:10BE2000E5E297F0FFFFE780404F5E859710000046
:10BE3000E780608A850415BF97A7FF1F9387871E39
:10BE40009C478D83858BC1F721611763FFFF6700D6
:10BE5000032A01468545094502D002D202D402D602
:10BE600097F0FFFFE7800040AA8479DD97F000009B
:10BE7000E780209C1389C4002A8481454A85970065
:10BE80000000E780005F0C4041464A8597000000B3
:10BE9000E780405B832944006385090C4E8502D806
:10BEA00002DA02DC02DE97300100E78020382ACE79
:10BEB000141005462C0808184ECC97500000E78057
:10BEC000200A1375F50F51ED8355840093E5250085
:10BED0004A8597000000E780E05E11460C104A8515
:10BEE00097000000E78000560146976501009385A2
:10BEF00065D6268597F0FFFFE780204226859700CC
:10BF00000000E780407D5C40A1D3014685450D459A
:10BF100097F0FFFFE7800035AA841DD548401389BC
:10BF2000C40097300100E78060302AC64A85970038
:10BF30000000E780404C3246636FC5004C404A85A4
:10BF400097000000E780005001468145268597F064
:10BF5000FFFFE780803C268597000000E780A07700
:10BF6000E5B583558400ADB71763FFFFE7022317DC
:10BF700097A7FF1F9387070B9C471DC193E7870077
:10BF800017A5FF1F130545E717A7FF1F2320F70A73
:10BF900097100100E78080311763FFFF6700631689
:10BFA000DD9B17A7FF1F2323F70897300000E780CA
:10BFB00020647DF117A5FF1F130505E4971001000C
:10BFC000E7802033D1BF1763FFFFE702C30E41694B
:10BFD000AA892E8AB28A368BBA8B814417ACFF1F8E
:10BFE000130C4C04930C400E7D1997F0FFFFE78073
:10BFF000205863C4A40001443DA0338494038327E4
:10C000000C0B3E948357C401638627055A87D68656
:10C010005286CE851305040397000000E780E0BB3D
:10C0200001C923800B0022851763FFFF6700230CE3
:10C030008347F40185C35A87D6865286CE85130579
:10C04000940897000000E78040B909C58547238020
:10C05000FB00D1BF850451BF835745006380071E95
:10C060001763FFFFE702030601112A84970000000F
:10C07000E780C04D09C985476309F5060561176367
:10C08000FFFF6700630797E00000E780407B7DF5D6
:10C09000835744004947ED9BE392E7FEC145228563
:10C0A00097000000E7804033AA84228597000000B3
:10C0B000E780204F0357440002CE91472A89631A34
:10C0C000F700228597000000E780A0513C082ACCA9
:10C0D0003ECE97E00000E780C0755C55C5D374087C
:10C0E0004A86A6850545829751BF03574400D1472C
:10C0F000E3F6E7F8032A0400C169014997AAFF1F84
:10C10000938A4AF2130B400EFD1997F0FFFFE78068
:10C110002046634FA90E2285032A040097000000E1
:10C12000E780C042A1452A89228597000000E78068
:10C13000A02AAA84228597000000E780804A144044
:10C140002A86AA8978082685CA8597000000E78094
:10C15000C0E7AA8405D503C7F40189476315F70032
:10C160008347C10181DF5546D2851385640097302E
:10C170000100E78020E7014597800000E780001973
:10C1800001C583D7C401A5E797A7FF1F938787E958
:10C190009C4793551900858913D73700058B01CF2C
:10C1A0008983858B6399B70001452EC697000000EF
:10C1B000E780C0DBB2454E8597800000E780A01E77
:10C1C0000346C1012A8493751900268597900000C3
:10C1D000E780203935C1268597800000E780201848
:10C1E000268511C0014597800000E780404B9730BD
:10C1F0000000E780E03F8547E312F5E883C754007D
:10C200001307F00FE38CE7E68507A382F400BDB5C2
:10C21000B304690383A70A0BBE9483D7C401638B5D
:10C2200037015546D2851385640097300100E780B9
:10C2300000D955DD0509D1BD5DD86DB78280176382
:10C24000FFFFE70223E897800000E780400B05C16D
:10C25000C164014417A9FF1F1309C9DC9309400EEB
:10C26000FD1497F0FFFFE780A030634EA40017A5F0
:10C27000FF1F130565B897100100E78020031763BF
:10C28000FFFF670063E7330534038327090B3E95FF
:10C290008357C5016388970023120500978000002B
:10C2A000E780E00B050475BF97A7FF1F938787D72B
:10C2B0009C478D83858B8DE31763FFFFE70223E2A5
:10C2C00017A5FF1F130545B397100100E780600213
:10C2D0001763FFFF6700E3E282801763FFFFE70257
:10C2E00003E0970500009385C5A017A5FF1F130560
:10C2F000A5B097100100E78060ED1763FFFF6700AE
:10C3000043E01763FFFFE70283DD8841B7E70400DE
:10C31000BC5B050542054181829709C5854723001D
:10C32000F50005051763FFFF6700A3DD83C7F5FF71
:10C330002E858507A38FF5FE828083C7F5FFFD1745
:10C3400093F7F70FA38FF5FE99EF1763FFFFE7024F
:10C3500003D9B7E70400BC571385F5FF829717632D
:10C36000FFFF670003DA82801C41035745008D8F71
:10C37000BA951CC12312B5003E85828093D78500F3
:10C38000A2051441DD8D835745001387E6FF18C1D0
:10C3900089072312F50013D685004111238FB6FEBD
:10C3A000A38FC6FE4101828018419307F7FF1CC18D
:10C3B0008357450085072312F500A30FB7FE82803F
:10C3C000835745008D8F2312F5001C41BE950CC18B
:10C3D0002E858280AA8703D7470008410D8FAA9532
:10C3E0002392E7008CC38280184108453305A7409B
:10C3F000828083574500035765001D8F1C41084507
:10C400003385A7403305A74082801763FFFFE7020B
:10C4100003CD41112EC62A8497000000E780A0FDBD
:10C42000B2456373B50001A0835744000840BE9530
:10C430002312B4003E9541011763FFFF670063CCF0
:10C440001763FFFFE702A3C941112E84B28532C6EC
:10C4500097000000E780A0FB3246A28597300100DC
:10C46000E78040B841011763FFFF670083C9176386
:10C47000FFFFE702C3C62E84854597000000E780D2
:10C4800000F9230085001763FFFF670083C7176368
:10C49000FFFFE702C3C441112317B100894597008C
:10C4A0000000E780C0F68347E1002300F5008347E2
:10C4B000F100A300F50041011763FFFF670063C4AB
:10C4C0001763FFFFE702A3C193D78500A2054111BF
:10C4D000DD8D2317B100894597000000E78020F328
:10C4E0008347E1002300F5008347F100A300F50036
:10C4F00041011763FFFF6700C3C01763FFFFE70237
:10C5000003BE1397850193D78501C166938606F014
:10C51000D98F13D78500758FD98FA2053707FF00F4
:10C52000F98D4111DD8D2EC6914597000000E78001
:10C5300000EE6C00114697300100E780A0AA41018F
:10C540001763FFFF6700E3BB1763FFFFE70223B931
:10C550001C41854503C4070097000000E78080E682
:10C5600022851763FFFF6700C3B91763FFFFE70268
:10C5700003B71C414111894503C7070083C7170052
:10C580002307E100A307F10097000000E78080E3A4
:10C590000355E10041011763FFFF670083B617638E
:10C5A000FFFFE702C3B31C414111894503C70700E0
:10C5B00083C717002307E100A307F10097000000DD
:10C5C000E78040E08357E100410113D58700A207CF
:10C5D0005D8D420541811763FFFF670083B21763DA
:10C5E000FFFFE702C3AF0C4141112A8411466800E6
:10C5F00097300100E780009F914522859700000059
:10C60000E78040DCB247C166938606F01397870146
:10C6100013D58701598D13D78700758F598DA207C0
:10C620003707FF00F98F5D8D41011763FFFF67003A
:10C6300043AD1C45BE950CC18280AE87944391E604
:10C64000584101EF0CC15CC1828003C757001367DA
:10C650001700A382E700B687D5B70CC3EDB7AA874A
:10C66000084119CD1841D44398C36313D500D8C3EA
:10C670002A87034657009376160081E62320070099
:10C680008280944381CA8C4203A847008CC3639381
:10C690000601CCC3799A14C3A302C7003687D1BF61
:10C6A0001C45DC471D8DB777DBB6938777DB0985A3
:10C6B0003305F502420541818280F147B385F502D9
:10C6C00048452E9582808347450085072302F50063
:10C6D00082801763FFFFE70283A02A8409E41763BF
:10C6E000FFFF670003A283474400F5DBFD1793F7C4
:10C6F000F70F2302F400E5F71C4403D727000507D2
:10C700002391E700DC4399C3228582974C4889CD69
:10C7100083475400898B99E71C4422859C479C439E
:10C720009C478297232A04000040232004007DB701
:10C730001763FFFFE702A39A8357250041112EC616
:10C7400081EB0144228541011763FFFF6700639B72
:10C75000035705008147F146E305F7FEB385D7028D
:10C76000404585072E948345440008C4F5F5B2473B
:10C77000AA8481E7232A040009A81C456C002285AD
:10C780009C439C43829748C84DDD85472312F400A3
:10C79000B24723200400231804002319F4005C4846
:10C7A0005CC483D72400FD172391F40061BF176395
:10C7B000FFFFE702C3929797FF1F9387E7658843C0
:10C7C0002326050023240500410597100100E7807A
:10C7D00040B21763FFFF6700C3921763FFFFE702D2
:10C7E00003901794FF1F130424631C40411199CF39
:10C7F0009C472300B5002AC65CC197000000E78073
:10C8000040FB1C40DC4399C33245829741011763CA
:10C81000FFFF6700038F0347450029E3584DAA87B0
:10C820007D551DCF1763FFFFE702638B1CC3DC47F9
:10C830009796FF1F23A2E65EF1561305070123908A
:10C84000D700970500009385050297100100E78047
:10C85000E09701451763FFFF6700A38A7D5582803B
:10C8600082801763FFFFE7028387011161468145DC
:10C8700028009760FFFFE78080899797FF1F9387C5
:10C88000A7599C4328009305F00FDC473EC697004C
:10C890000000E780C0F405611763FFFF670063864F
:10C8A0009797FF1F938747579C43D847A167938764
:10C8B000C702631EF70A397106DE22DC26DA800021
:10C8C0004AD84ED652D456D23285B2849700000050
:10C8D000E780C0C7AA89268597000000E78020C9A5
:10C8E0002318A4FC268597000000E78040C8231980
:10C8F000A4FC268597000000E78060C783D744002A
:10C900000A8A231AA4FC858393F7F70F230EF4FCFD
:10C910008607BD0793F7073F3301F1408A8A014933
:10C920008347C4FD6367F902CE85130584FC232C7D
:10C9300054FD97000000E78080EA5281130104FC57
:10C94000F2506254D2544259B259225A925A216139
:10C950008280268597000000E78060C19317190048
:10C96000D69705092390A7001379F90F55BF828048
:10C970009797FF1F9387474A9C43D847A1679387A0
:10C98000A702631AF70A397106DE22DC26DA800074
:10C990004AD84ED652D456D23285B284970000007F
:10C9A000E780C0BAAA89268597000000E78020BCEE
:10C9B000FD572318A4FC26852319F4FC97000000DA
:10C9C000E780E0BA83D744000A8A231AA4FC85834F
:10C9D00093F7F70F230EF4FC8607BD0793F7073F85
:10C9E0003301F1408A8A01498347C4FD6367F90234
:10C9F000CE85130584FC232C54FD97000000E780AE
:10CA000000DE5281130104FCF2506254D2544259A8
:10CA1000B259225A925A21618280268597000000DD
:10CA2000E780E0B493171900D69705092390A70073
:10CA30001379F90F55BF82809797FF1F9387C73DE2
:10CA40009C43D847A16789076310F70A397106DE4E
:10CA500022DC26DA80004AD84ED652D456D232850D
:10CA6000328997000000E78060AEAA894A85970066
:10CA70000000E780C0AF835749000A8A2318A4FC4E
:10CA8000858393F7F70F230CF4FC8607BD0793F714
:10CA9000073F3301F1408A8A8144834784FD63E77D
:10CAA000F402CE85130584FC232A54FD9700000070
:10CAB000E780E0D25281130104FCF2506254D25458
:10CAC0004259B259225A925A216182804A8597006E
:10CAD0000000E780C0A993971400D697850423909F
:10CAE000A70093F4F40F55BF82809797FF1F938799
:10CAF000A7329C43D847A1679387E704631EF70AD0
:10CB0000397106DE22DC26DA80004AD84ED652D4AD
:10CB100056D23285B28497000000E78020A3AA890C
:10CB2000268597000000E78080A42318A4FC2685B2
:10CB300097000000E780A0A3231AA4FC2685970095
:10CB40000000E780C0A283D744000A8A2319A4FC0E
:10CB5000858393F7F70F230EF4FC8607BD0793F741
:10CB6000073F3301F1408A8A01498347C4FD636767
:10CB7000F902CE85130584FC232C54FD9700000098
:10CB8000E780E0C55281130104FCF2506254D25494
:10CB90004259B259225A925A2161828026859700C1
:10CBA0000000E780C09C93171900D69705092390D1
:10CBB000A7001379F90F55BF82809797FF1F9387BE
:10CBC000A7259C43D847A1679387C704631AF70A30
:10CBD000397106DE22DC26DA80004AD84ED652D4DD
:10CBE00056D23285B28497000000E7802096AA8949
:10CBF000268597000000E7808097FD572318A4FC46
:10CC00002685231AF4FC97000000E780409683D71E
:10CC100044000A8A2319A4FC858393F7F70F230E97
:10CC2000F4FC8607BD0793F7073F3301F1408A8A7A
:10CC300001498347C4FD6367F902CE85130584FC6F
:10CC4000232C54FD97000000E78060B95281130146
:10CC500004FCF2506254D2544259B259225A925AA8
:10CC600021618280268597000000E780409093171D
:10CC70001900D69705092390A7001379F90F55BF1E
:10CC800082809797FF1F938727199C43D847A167F6
:10CC9000DD076317F7041753FFFFE7024344797179
:10CCA0003285328497000000E780408A2AC62285B8
:10CCB00097000000E780A08B2311A1022285970036
:10CCC0000000E780A088B2452300A1022808970051
:10CCD0000000E780C0B045611753FFFF6700634263
:10CCE00082809797FF1F938727139C43D847A1679C
:10CCF000938787046317F7041753FFFFE702233E68
:10CD000079713285328497000000E78020842AC63A
:10CD1000228597000000E78080852311A1022285EB
:10CD200097000000E7808082B2452300A102280816
:10CD300097000000E780A0AA45611753FFFF670036
:10CD4000433C82809797FF1F9387070D9C43D847EA
:10CD5000A1679387A7046312F7021753FFFFE70247
:10CD6000033801112800814597000000E78020A7C3
:10CD700005611753FFFF6700C33882809797FF1F35
:10CD8000938787099C43D847A16793875702631904
:10CD9000F7021753FFFFE70283340111328597F042
:10CDA000FFFFE780A07A2308A100814528009700B3
:10CDB0000000E780C0A205611753FFFF67006334DE
:10CDC00082809797FF1F938727059C43D847A167C9
:10CDD0009387E702631BF7041753FFFFE702233033
:10CDE00001113285328497F0FFFFE7804078AA84F2
:10CDF000228597F0FFFFE7808077854709E9228544
:10CE000097F0FFFFE78080744205B337A000280049
:10CE10008145231891003ECA97000000E780209CBE
:10CE200005611753FFFF6700C32D82809797FF1F8F
:10CE3000938787FE9C43D84799476313F708175396
:10CE4000FFFFE702C32979713285328497F0FFFF33
:10CE5000E780C06F2AC6228597F0FFFFE780207128
:10CE60002310A102228597F0FFFFE780206E2301A7
:10CE7000A102228597F0FFFFE780406DA301A10288
:10CE8000228597F0FFFFE780606C2302A1022285D4
:10CE900097F0FFFFE780806B2313A102228597F0B4
:10CEA000FFFFE780A06AB2452314A102280897007B
:10CEB0000000E780C09245611753FFFF67006324BD
:10CEC00082809797FF1F938727F59C43D847A167D8
:10CED0009387C7036313F7081753FFFFE702232065
:10CEE00079713285328497F0FFFFE78020662AC689
:10CEF000228597F0FFFFE78080672310A10222853B
:10CF000097F0FFFFE780A0662311A102228597F02A
:10CF1000FFFFE780A0632302A102228597F0FFFFB5
:10CF2000E780C062A302A102228597F0FFFFE7809D
:10CF3000E0612303A102228597F0FFFFE7800061F3
:10CF4000B245A303A102280897000000E7802089CA
:10CF500045611753FFFF6700C31A82801753FFFF15
:10CF6000E702E31701112A8497F0FFFFE780005ED4
:10CF7000AA84228597F0FFFFE780605F228597F003
:10CF8000FFFFE780C05E035744008D4763F7E7006B
:10CF9000228597F0FFFFE780805D228597F0FFFFF5
:10CFA000E780E05C2800A68597000000E7802083EA
:10CFB00005611753FFFF6700C3149797FF1F9387FF
:10CFC000A7E59C43D847A167FD07631FF7001753E8
:10CFD000FFFFE702C310328597000000E78040F8AA
:10CFE0001753FFFF6700E31182809797FF1F938716
:10CFF000A7E29C43D847A167E5076315F7081753D5
:10D00000FFFFE702C30D79713285328497F0FFFF8D
:10D01000E780C0532AC6228597F0FFFFE78020559E
:10D02000228597F0FFFFE78080542310A10222851C
:10D0300097F0FFFFE780A053520551812311A10211
:10D0400022852302010297F0FFFFE7802050A30210
:10D05000A102228597F0FFFFE780404F2303A10242
:10D06000228597F0FFFFE780604EB245A303A1023F
:10D07000280897F0FFFFE780807645611753FFFF90
:10D080006700230882809797FF1F9387E7D89C4308
:10D09000D847A1679387E703631FF7001753FFFF84
:10D0A000E702E303328597000000E78060EB175347
:10D0B000FFFF6700030582809797FF1F9387C7D5FF
:10D0C0009C43D847A16793874704631EF702175311
:10D0D000FFFFE702C30079713285328497F0FFFFCA
:10D0E000E780C0462AC6228597F0FFFFE7802048E8
:10D0F000B245280897F0FFFFE780606E456117533F
:10D10000FFFF6700030082809797FF1F9387C7D0B8
:10D110009C43D847A167938787026310F70417538E
:10D12000FFFFE702C3FB79713285328497F0FFFF7E
:10D13000E780C0412AC6228597F0FFFFE7800041C3
:10D14000B2452300A102280897F0FFFFE78020697D
:10D1500045611753FFFF6700C3FA82801753FFFF33
:10D16000E702E3F7011197F0FFFFE780203EAA8571
:10D17000280097F0FFFFE780806605611753FFFFE7
:10D18000670023F89797FF1F938707C99C43D847E9
:10D19000A167D107631FF7001753FFFFE70223F4CE
:10D1A000328597000000E780A0FB1753FFFF670060
:10D1B00043F582809797FF1F938707C69C43D84704
:10D1C000A167C507631FF7001753FFFFE70223F1AD
:10D1D000328597000000E780A0F81753FFFF670033
:10D1E00043F282809797FF1F938707C39C43D847DA
:10D1F000A167B907631FF7001753FFFFE70223EE8C
:10D20000328597000000E780A0F51753FFFF670005
:10D2100043EF82809797FF1F938707C09C43D847AF
:10D22000A167AD07631FF7001753FFFFE70223EB6A
:10D23000328597000000E780A0F21753FFFF6700D8
:10D2400043EC82809797FF1F938707BD9C43D84785
:10D2500089476318F7021753FFFFE70243E80111FC
:10D26000328532C897F0FFFFE780402EAA8528005C
:10D2700097F0FFFFE780A05605611753FFFF670097
:10D2800043E882809797FF1F938707B99C43D8474D
:10D29000A1678D076311F7041753FFFFE70223E42B
:10D2A00001113285328497F0FFFFE780202A1306B0
:10D2B0006100AA844C00228597300000E78000239B
:10D2C0002800A68597F0FFFFE7806051056117539E
:10D2D000FFFF670003E382809797FF1F938707B4E0
:10D2E0009C4381CFDC4391CB1753FFFFE70223DF41
:10D2F00082971753FFFF6700C3E082801753FFFF39
:10D30000E702E3DD79713C08AE843ED2A165B70740
:10D310000A002A843ED448103C08DD053ED636C4B7
:10D3200032C63AC297D0FFFFE780402C1247481020
:10D33000BA8597F0FFFFE780C01332464810B285E8
:10D3400097F0FFFFE780E014A2464810B68597F0FB
:10D35000FFFFE7800012501001478146A685228515
:10D3600097D0FFFFE780E04D45611753FFFF67004F
:10D3700043D91753FFFFE70283D601117C0003292D
:10D38000C501AE843ECAA165B70707002A843ECC1A
:10D3900048087C00C5053ECE97D0FFFFE7800025FA
:10D3A0008345D900480897F0FFFFE780800C5008BC
:10D3B00001478146A685228597D0FFFFE780604818
:10D3C00005611753FFFF6700C3D31753FFFFE70241
:10D3D00003D183C7950093F7F707A384F50097005F
:10D3E0000000E78040F91753FFFF670083D1175310
:10D3F000FFFFE702C3CE79713C08AE843ED2A1653F
:10D40000B70709002A843ED448103C089385450498
:10D410003ED632C636C497D0FFFFE780201DA24615
:10D420004810B68597F0FFFFE780A0043246481009
:10D43000B28597F0FFFFE780C00550100147814695
:10D44000A685228597D0FFFFE780A03F456117534F
:10D45000FFFF670003CB1753FFFFE70243C883C7F3
:10D46000950041112A8493F7F707A384F5003285CC
:10D470002EC697F0FFFFE780800F85672AC4637090
:10D48000F50297700000E78060E82246B24509ED9A
:10D4900011478146228597000000E78060E6410140
:10D4A0001753FFFF6700E3C501478346F501DDB76A
:10D4B0001753FFFFE70203C101113C003ECAB70743
:10D4C0000A003ECC3C003ECE83C79500AA89328537
:10D4D00093F7F707A384F5002E8497F0FFFFE7800A
:10D4E00000098567637DF504A165AA849385850499
:10D4F000480897D0FFFFE780600F268597700000EF
:10D50000E780C0E02A8929E19145480897F0FFFFAC
:10D51000E78020F6A685480897F0FFFFE78060F7D0
:10D52000CA85480897F0FFFFE780A0F401478146CD
:10D530005008A2854E8597D0FFFFE78080300561B7
:10D540001753FFFF670043BB8145480897F0FFFF73
:10D55000E78020F20349090275BF1753FFFFE70276
:10D5600063B679711C103ECAB7070F003ECC404D20
:10D570001C10AA84AE894808994532C636893ECE29
:10D5800097D0FFFFE780800632464808B28597F0C3
:10D59000FFFFE78000EE630C0902A545480897F0FD
:10D5A000FFFFE780C0E62546CA8597200100E78097
:10D5B00060A3500801478146CE85268597D0FFFF9E
:10D5C000E780202845611753FFFF6700E3B28355CA
:10D5D000C402480897F0FFFFE780A0EB0355E40280
:10D5E000814505C5854785456301F502C167FD177E
:10D5F0009305F00F630BF5007D1597700000E78031
:10D60000608D9305150093F5F50F480897F0FFFF1F
:10D61000E78020E683450403480897F0FFFFE78092
:10D6200040E583451403480897F0FFFFE78060E476
:10D6300083552403480897F0FFFFE78080E5835572
:10D640004403480897F0FFFFE780A0E49DB7175315
:10D65000FFFFE702C3A883C795008146014693F701
:10D66000F707A384F50097000000E78040EF175309
:10D67000FFFF670003A91753FFFFE70243A6797175
:10D680003E841C103ECA2E89B7070F00A1653ECC10
:10D69000FD051C10AA84480842C03AC23ECE36C4DA
:10D6A00032C697D0FFFFE78060F432464808B28563
:10D6B00097F0FFFFE780E0DBA2464808B68597F0C9
:10D6C000FFFFE78000DD12474808BA8597F0FFFFAB
:10D6D000E78020DC0248630C08029145480897F077
:10D6E000FFFFE780C0D21146A28597200100E780A6
:10D6F000608F500801478146CA85268597D0FFFF75
:10D70000E780201445611753FFFF6700839F894519
:10D71000480897F0FFFFE78080CF8347040023008D
:10D72000F50083471400A300F500E1B71753FFFF8E
:10D73000E702439983C7950001112A8A93F7F707F7
:10D74000A384F5003285AE8432C697F0FFFFE780F0
:10D7500000E232462A89328597F0FFFFE78000DF3A
:10D7600085676373F902AA894A8597700000E7808C
:10D77000E0B92A8419ED114781464A86A68552856B
:10D7800097000000E780C0B705611753FFFF6700EF
:10D79000A3969387E9FF93F7F70F0547E366F7FE34
:10D7A0008347F50195EB8947E380F9FE8346F40151
:10D7B000528501474A86A68597000000E78040B45D
:10D7C000A167D90748083ECC230A010002CE970082
:10D7D0000000E780A0B04DBF639EE7008947639ECD
:10D7E000F90093071020231FF50097700000E780D1
:10D7F00000B76DBF0947E39BE7FA8D47E398F9FA55
:10D80000228597700000E780C0DE9787FF1F93870F
:10D81000E77F9C4399E79787FF1F9387E7689C43BF
:10D8200099C703D5040097800000E780E0CD231F4F
:10D83000040022855DBF1753FFFFE702438A0111F1
:10D840003C003ECAB7070B003ECC3C003ECE83C72F
:10D8500095002A89328593F7F707A384F500AE84F3
:10D8600097F0FFFFE780A0D093170501C187635AA7
:10D87000F006A1652A849385E502480897D0FFFF4A
:10D88000E780C0D6A285480897F0FFFFE78060C018
:10D890009787FF1F938747619C43A9EB01449375CA
:10D8A000F40F480897F0FFFFE780A0BC9355844031
:10D8B00093F5F50F480897F0FFFFE78080BB93557D
:10D8C000044193F5F50F480897F0FFFFE78060BA31
:10D8D000014781465008A6854A8597D0FFFFE7801B
:10D8E00040F605611753FFFF6700A3814165854638
:10D8F0000546A2857D1597500000E780A0BC59DD44
:10D90000510597000100E780C08E130440063344A0
:10D91000850271B71743FFFFE702637C0111B70768
:10D9200006003EC683C7950021642A8993F7F7074E
:10D93000A384F500AE8428009305A4040AC40AC891
:10D9400097D0FFFFE78080CA300001478146A68557
:10D950004A8597D0FFFFE780C0EE97E0FFFFE780A2
:10D96000E01113049404480822CC230A010002CEDB
:10D9700097000000E780809605611743FFFF67006E
:10D9800043781743FFFFE702E373C1642A89014428
:10D990009789FF1F93890969130A8002FD1497E094
:10D9A000FFFFE780E0BD6347A40001451743FFFF89
:10D9B00067008374B307440303A7C90ABA9703D760
:10D9C00007006306970083D72700638427010504B7
:10D9D000F9B70545E1BF1743FFFFE702A36E2A8AA7
:10D9E0002E8999C123A0050081498144978AFF1F90
:10D9F000938A0A43614B97E0FFFFE780A0BE63C7AD
:10DA0000A4004E851743FFFF6700036F3384640350
:10DA100083A70A003E948357040099E76304090032
:10DA2000232089008504C1BF4146D28513054400E7
:10DA300097100100E780A05875F5A289E5B7174354
:10DA4000FFFFE702236839717C083ED4B7070A005C
:10DA50003ED67C083ED883C795002A8A328593F744
:10DA6000F707A384F5002E8932C697F0FFFFE78001
:10DA700000B085676373F5083246AA84328597F053
:10DA8000FFFFE780A0AC8547AA8963E8A706A165E8
:10DA900093858504281097D0FFFFE78020B5268561
:10DAA00097700000E78080862A8429ED9145281030
:10DAB00097F0FFFFE780E09BA685281097F0FFFF17
:10DAC000E780209DCE85281097F0FFFFE780609AC1
:10DAD000014781463010CA85528597D0FFFFE78005
:10DAE00040D6A1679387770448183EDC230A0102D9
:10DAF00002DE97F0FFFFE780607E21611743FFFFA2
:10DB00006700835F8145281097F0FFFFE7806096EC
:10DB1000A685281097F0FFFFE780A0979797FF1F33
:10DB2000938707879C4381CB22856389090097D01F
:10DB30000000E78080238345040271B797D000007E
:10DB4000E7800022CDBF1743FFFFE702A35783C73B
:10DB500095004111AA8993F7F707A384F500328550
:10DB6000AE84328A97F0FFFFE78060A08567637F0D
:10DB7000F5022A8997600000E78040792A8491465F
:10DB800031C58347F50105476387E70291C70D4714
:10DB90006366F704AD461DA89305050303250A0037
:10DBA000414697100100E78080410DE9410117438C
:10DBB000FFFF670063549305950803250A0041465B
:10DBC00097100100E780A03F814669F54A86A68547
:10DBD0004E8597000000E780C081C9BF83250A00F9
:10DBE0001305940897700000E780E02819C1C1462A
:10DBF000F1BF9787FF1F938767419C4399E79787FA
:10DC0000FF1F9387672A9C4399C72285978000004E
:10DC1000E780608969FD8547A30FF400228597B0EE
:10DC20000000E780A083228597600000E7802073D2
:10DC30004E8581464A86A68597F0FFFFE780607B88
:10DC4000A1679387570448003EC42302010002C61F
:10DC500097F0FFFFE780806891BF1743FFFFE7025F
:10DC6000834583C795004111AA8993F7F707A384D9
:10DC7000F50032852E89B28A97F0FFFFE780208F6A
:10DC800085676374F50EAA8497600000E7800068DA
:10DC90002A840DED416B014A978BFF1F938B8B38C4
:10DCA000130C400E7D1B19A833048A0383A70B0BAA
:10DCB0003E948357C40163836705050A97E0FFFF1D
:10DCC000E780008BE342AAFE95460DA08357C5016D
:10DCD000639697029305050303A50A004146971032
:10DCE0000100E780C02D994611E181462686CA854C
:10DCF0004E8597F0FFFFE780C06F85A883A50A00D7
:10DD00001305040397700000E780E016C14679FD13
:10DD10002285231E940097A00000E78020742285AE
:10DD200097600000E780A0639787FF1F938747668F
:10DD30009C43A9C323000402228597D00000E780FA
:10DD400080EF4E8581462686CA8597F0FFFFE780E3
:10DD5000406AA1679387070448003EC4230201007C
:10DD600002C697F0FFFFE780605741011743FFFFAE
:10DD70006700E33789472300F402E1B7397106DE13
:10DD800022DC4AD8800052D456D25AD026DA4ED657
:10DD90005ECE2E8A32892A8B97D0FFFFE780407AA9
:10DDA0000605710541998A8A3301A140232224FC8A
:10DDB000231404FC97D0FFFFE780807883479A0004
:10DDC0000605350593F7F7072315A4FCA304FA000D
:10DDD0004A85232624FC97E0FFFFE78040799317CC
:10DDE0000501C1876340F0025681130104FCF25023
:10DDF0006254D2544259B259225A925A025BF24B9F
:10DE000021618280AA844A8597E0FFFFE78020761F
:10DE1000AA894A8597E0FFFFE7806075A165938531
:10DE2000C5022A89130544FC97C0FFFFE780007CE8
:10DE3000268597C0FFFFE7804070854511C94A8657
:10DE4000CE8597C0FFFFE780C069AA8B21E989458D
:10DE5000130544FC97E0FFFFE780A061A68513054A
:10DE600044FC97E0FFFFE780C062CE85130544FCC9
:10DE700097E0FFFFE780E061CA85130544FC97E067
:10DE8000FFFFE780006101478146130644FCD2850D
:10DE90005A8597D0FFFFE780C09AB9B7814513052F
:10DEA00044FC97E0FFFFE780C05CA685130544FCB7
:10DEB00097E0FFFFE780E05DCE85130544FC97E027
:10DEC000FFFFE780005DCA85130544FC97E0FFFF74
:10DED000E780205C814497D0FFFFE7806066E3D451
:10DEE000A4FA83A70B0113971400BA9783D50700F0
:10DEF00099C5130544FC97E0FFFFE780805985042E
:10DF0000D9BF797106D622D44AD000184ECE52CC51
:10DF100056CA26D25AC8AE893289AA8A97D0FFFF3C
:10DF2000E78000620605690541990A8A3301A1402C
:10DF3000232A24FC231C04FC97D0FFFFE7804060C9
:10DF400083C7990006052D0593F7F707231DA4FC49
:10DF5000A384F9004A85232E24FC97E0FFFFE78085
:10DF6000006193170501C187634FF00052811301CF
:10DF700004FDB250225492540259F249624AD24AE4
:10DF8000424B45618280AA844A8597E0FFFFE78083
:10DF9000005EA1659385A5022A89130544FD97C0FB
:10DFA000FFFFE780A064268597C0FFFFE780E05869
:10DFB000854509C9CA8597C0FFFFE78080552A8B30
:10DFC00029E18945130544FD97E0FFFFE780604A9A
:10DFD000A685130544FD97E0FFFFE780804BCA85C7
:10DFE000130544FD97E0FFFFE780A04A0147814603
:10DFF000130644FDCE85568597D0FFFFE7806084E9
:10E00000B5B78145130544FD97E0FFFFE780604603
:10E01000A685130544FD97E0FFFFE7808047CA858A
:10E02000130544FD97E0FFFFE780A046814497D0A9
:10E03000FFFFE780E050E3DBA4FA83270B0113978F
:10E040001400BA9783D5070099C5130544FD97E0DE
:10E05000FFFFE78000448504D9BF1743FFFFE702B5
:10E06000030883474500404DD5EFFD575DC4834607
:10E07000940009476363D70A0346B400854663EEFC
:10E08000C6088306E40063CA06085C45F956239077
:10E09000D7009787FF1F83C7E7D899E3A304E4005D
:10E0A0009787FF1F938747E09C4381E78947A30633
:10E0B000F4009787FF1F9387A72D9C4381E789472B
:10E0C0002306F4009705000093854506AA841305EE
:10E0D000040197F00000E780600FFD57231AF40257
:10E0E00081471CDC01489787FF1F23A987D29787A8
:10E0F000FF1F9387E7D2232E040304C0804397D0E9
:10E10000FFFFE780204E61463306C5028145228528
:10E110009740FFFFE780A0FF81473E851743FFFF41
:10E12000670023FEFD57D5BF1743FFFFE70223FB20
:10E130002A840355450297600000E780201D19E5F9
:10E14000231E04001743FFFF6700A3FB8357E4016E
:10E15000F5DB930504FF17450100130565E997E01A
:10E160000000E7802014F9BF1743FFFFE70223F701
:10E170002E89A16541119385E5032A8436C432C6F0
:10E18000BE843AC297C0FFFFE7804046124722850F
:10E19000BA8597E0FFFFE780C02D32462285B28521
:10E1A00097E0FFFFE780E02EA2462285B68597E044
:10E1B000FFFFE780002E630309029145228597E067
:10E1C000FFFFE780C0241146A68597100100E78075
:10E1D00060E141011743FFFF6700A3F289452285F3
:10E1E00097E0FFFFE780A02283C704002300F5002B
:10E1F00083C71400A300F500E9BF1743FFFFE70240
:10E2000003EE83C79500444D054793F7F707A384B2
:10E21000F5001C42411183C707006367F7062E848F
:10E220002A89B1C003C7D400630FF7021787FF1F05
:10E23000130787C7184305C3A386F40097A00000FF
:10E24000E780804983C7D40099E741657D159740F1
:10E250000000E780802F83D72403918B89C797E044
:10E260000000E78000134A85A28597F0FFFFE78052
:10E270008010A167C10748003EC42302010002C606
:10E2800097F0FFFFE780800541011743FFFF67001C
:10E2900043E71743FFFFE70283E403D745008D47B9
:10E2A000AA8441112E8432892E8563E3E70297E028
:10E2B000FFFFE780C02BAA8523000900268597C0B1
:10E2C000FFFFE780002541011743FFFF670063E37D
:10E2D00097E0FFFFE780A0292AC6228597E0FFFF8D
:10E2E000E780E028B24585472A862300F900268585
:10E2F00097C0FFFFE780E01EF9B7397106DE22DC28
:10E3000026DA80004ED652D456D24AD85AD05ECEA3
:10E31000AE89B284AA8A97D0FFFFE7806021060504
:10E320001305250241990A8A3301A140232224FCC6
:10E33000231404FC97D0FFFFE780801F83C7990058
:10E3400006054D0593F7F7072315A4FCA384F900F0
:10E350002685232624FC97E0FFFFE78040219317C2
:10E360000501C1876340F0025281130104FCF250A1
:10E370006254D2544259B259225A925A025BF24B19
:10E3800021618280AA8B03AB040097C0FFFFE78066
:10E39000C01A51E583D7440001498544F11793B76A
:10E3A0001700A301F4FC834734FCA165C9C793851A
:10E3B000E504130544FC97C0FFFFE7802023A685F2
:10E3C000130544FC97E0FFFFE780A00ADE851305F4
:10E3D00044FC97E0FFFFE780C00B834734FC114605
:10E3E00091E30946DA85130544FC97E0FFFFE780D7
:10E3F00060058144630A0900416B7D1B97D0FFFFD4
:10E40000E780001363CCA40201478146130644FC55
:10E41000CE85568597C0FFFFE780A042B1B7A6859D
:10E42000130634FC97000000E780E0E69334150003
:10E430002A8986048DBF9385C504A5BF8327C9009B
:10E4400013971400BA9783D50700638865011305F5
:10E4500044FC97E0FFFFE780C003850445B71743FE
:10E46000FFFFE70243C579711C103EC4B7070F00D8
:10E470003EC61C103EC883C79500AA8A328593F712
:10E48000F707A384F500AE89328497E0FFFFE780A9
:10E49000000E93170501C187635AF0062A8A228568
:10E4A00097E0FFFFE780A00C2A895285032B040028
:10E4B00097C0FFFFE780600839ED8357440081442F
:10E4C0000544F11793B71700A303F10083457100CA
:10E4D000DA872287CA865286280097000000E780E4
:10E4E000E0C8014781463000CE85568597C0FFFFC2
:10E4F000E7802035A1679387D70348083ECC230ADD
:10E50000810026CE97F0FFFFE78040DD456117438D
:10E51000FFFF6700C3BDA2851306710097000000CE
:10E52000E78060D7AA84094455D13544E30055FB00
:10E530004A8597F0FFFFE78000450D4441D901442B
:10E5400097D0FFFFE780C0FE634DA400C16B01447C
:10E55000FD1B97D0FFFFE780A0FD634EA40015448C
:10E56000B5B7DC4413171400BA9783D70700638349
:10E5700027030504F1B7D84493171400BA9703D7BB
:10E580000700631B770123902701268597A00000D1
:10E59000E780C0DA01441DBF050465BF1743FFFFD4
:10E5A000E70243B283C7950041112A8A93F7F70720
:10E5B000A384F50032852E89328497E0FFFFE7803F
:10E5C00000FB93170501C1876353F006AA892285D2
:10E5D00097E0FFFFE780A0F92311A1004E85832A71
:10E5E000040097C0FFFFE78040F539E583574400FA
:10E5F00085440144F11793B71700A300F1000348C5
:10E60000110003572100D6875285CE862686CA85FB
:10E6100097F0FFFFE7806006A167F10748003EC45E
:10E620002302910022C697F0FFFFE78020CB410133
:10E630001743FFFF670043ACA28513061100970044
:10E640000000E78040C52A84894455D983572100BA
:10E6500011678544BA97C2071167C1831307F7EFA3
:10E66000E36FF7F89787FF1F9387479A9C4381CB07
:10E6700085451305210097500000E780607483559D
:10E6800021002285814497C0FFFFE780A0E125D9C2
:10E6900023100500228597A00000E78080CC85B775
:10E6A0001743FFFFE70223A183C7950041112A8B7F
:10E6B00093F7F707A384F50032852E8A328497E01A
:10E6C000FFFFE780C0EA93170501C1876351F00699
:10E6D000AA8A228597E0FFFFE78060E92A895685AC
:10E6E000832B040097C0FFFFE78020E531E58357C7
:10E6F000440081440544F11793B71700A301F100CA
:10E7000003483100DE875A854A87D6862286D2851D
:10E7100097F0FFFFE78060F6A167ED0748003EC471
:10E720002302810026C697F0FFFFE78020BB41014E
:10E730001743FFFF6700A39BA285130631009700D4
:10E740000000E78040B5AA8409445DD99167CA9763
:10E75000C2071167C1831307F7EF0544E362F7FAB5
:10E76000CA8597C0FFFFE780E0D3014451F9814992
:10E7700097D0FFFFE780C0DC63DBA9009848939740
:10E780001900BA9703D7070005EF2390270197D008
:10E79000FFFFE780E0DA1544E384A9F6268597A019
:10E7A0000000E78000BC9787FF1F938727869C4364
:10E7B0000144B9D74A8597500000E780005889B7CF
:10E7C00085097DB71743FFFFE702C38F79713E8448
:10E7D0007C083EC82E8AB7071400A1653ECAE5052D
:10E7E0007C08AA89080836C4428932C6BA8AC68417
:10E7F0003ECC97C0FFFFE78060DFCA85080897E03E
:10E80000FFFFE78000C732460808B28597E0FFFFA8
:10E81000E78020C8A246630A09049D45080897E0DE
:10E82000FFFFE780C0BE1D4681459740FFFFE780A0
:10E83000008E63890A089145080897E0FFFFE7808A
:10E8400000BD1146A68597000100E780A079100859
:10E8500001478146D2854E8597C0FFFFE78060FE65
:10E8600045611743FFFF67002389B685080897E0D5
:10E87000FFFFE78000C21C400808D8439355C7013A
:10E88000858912075183B205D98D97E0FFFFE78094
:10E8900040C01C40080883C5870097E0FFFFE78061
:10E8A00040BD1C40080883C5A70097E0FFFFE78034
:10E8B00040BC1C40080883C5970097E0FFFFE78035
:10E8C00040BB85BF8945080897E0FFFFE78020B47B
:10E8D00083C704002300F50083C71400A300F500DC
:10E8E000BDB71733FFFFE702E37D83C795004111F2
:10E8F000AA8993F7F707A384F5003285AE843284A2
:10E9000097E0FFFFE780A0C693170501C187635D0D
:10E91000F0042A89032A040097C0FFFFE780E0C1C2
:10E9200019E9835744000548F11793B71700A30767
:10E93000F100814631A81306F100A285970000007E
:10E94000E78060951DC51C459DC783D647000148DB
:10E950000347F10093078500D2884A86A6854E8535
:10E9600097000000E78040E641011733FFFF670092
:10E97000A37809487DBF1D486DBF1733FFFFE7022D
:10E98000637465715C083EC4B7077B013EC65C08D2
:10E990003EC883C795002A8A328593F7F707A38478
:10E9A000F500AE8997E0FFFFE78040BA8357E100AA
:10E9B000E1C78945280097C0FFFFE78020C3814554
:10E9C000280097E0FFFFE780C0AA97C0FFFFE7801D
:10E9D00000C99787FF1F9387A79B9C431774FF1F4E
:10E9E00003444444AA843334800099C3136424004C
:10E9F0009777FF1F9387474B9C4399C31364440049
:10EA00009777FF1F938787609C4399C313648400A3
:10EA100083D504002800014997E0FFFFE78060A745
:10EA200083D52400280097E0FFFFE78080A683D5E8
:10EA30004400280097E0FFFFE780A0A597D0FFFFE4
:10EA4000E78000AB93150501C181280097E0FFFF27
:10EA5000E78020A4A285280097E0FFFFE78060A35D
:10EA60009C446360F902014781463000CE8552859F
:10EA700097C0FFFFE780E0DC59611733FFFF6700B5
:10EA8000A367DC441314490028003E9497E0FFFF7D
:10EA9000E7806096834744000347540089070607D0
:10EAA000BA978607E36AF5FC835524002800814A5B
:10EAB00097E0FFFFE780E09D83454400280097E052
:10EAC000FFFFE780009B83455400280097E0FFFF8D
:10EAD000E780209A8347440063C9FA00814A83474C
:10EAE000540063C1FA020509A5BF1C4413975A00DC
:10EAF0002800BA9783D50700850A97E0FFFFE780D3
:10EB00004099C9BF032BC40093975A0028003E9B2D
:10EB100083552B00850A97E0FFFFE7808097835598
:10EB20000B00280097E0FFFFE780A0964DBF17334A
:10EB3000FFFFE702C35A5C4993E717005CC997A03F
:10EB40000000E78060B51733FFFF6700835B173372
:10EB5000FFFFE702C3582E84814597F0FFFFE7804F
:10EB6000C0E705C583570500FD172310F50009C44C
:10EB7000835725002310F40097000000E78060FB16
:10EB800001451733FFFF6700C35731457DD8231078
:10EB90000400C5BF1733FFFFE702C35283C79500C8
:10EBA00041112A8A93F7F707A384F50032852E894D
:10EBB000328497E0FFFFE780809B93170501C187B0
:10EBC0006356F006AA89C145228597E0FFFFE780DA
:10EBD000A0802A8B4E85832A040097C0FFFFE78020
:10EBE000C09531E983574400231101000544F11712
:10EBF00093B71700A300F1008144034811000357A5
:10EC00002100D6875285CE862286CA8597F0FFFFDF
:10EC1000E780A0A6A1679387170248003EC423029D
:10EC2000810026C697E0FFFFE780406B4101173364
:10EC3000FFFF6700634C13061100A28597F0FFFFEA
:10EC4000E7806065AA8409E523110100094475B7CE
:10EC5000930521005A8597000000E78080EF8357D5
:10EC600021002A84D9DB9777FF1F9387273A9C439B
:10EC700081CB85451305210097500000E7804014A3
:10EC8000835521002685314497C0FFFFE7808081AE
:10EC90002DD523100500268597900000E780606C35
:10ECA0000144A1BF1733FFFFE702634341112E89DF
:10ECB0006C00AA8402C697F0FFFFE78000D20DC166
:10ECC0000357050005072310E50097000000E780C3
:10ECD00040E681473E8541011733FFFF67006342ED
:10ECE0003247954765DBCA85268597300000E78067
:10ECF000800CC147E34005FE32448547414623105E
:10ED0000F40083570900A685130544002311F4007D
:10ED100097000100E780002D228545BF1733FFFFD4
:10ED2000E702433A83C795004111AA8A93F7F70790
:10ED3000A384F5003285AE89328497E0FFFFE78037
:10ED4000008393170501C1876356F0062A8AC145DF
:10ED5000228597D0FFFFE7802068AA845285032B85
:10ED6000040097B0FFFFE780407D31E983574400FE
:10ED7000231101008544F11793B71700A300F10098
:10ED800001440348110003572100DA875685D286D3
:10ED90002686CE8597F0FFFFE780208EA1679387B8
:10EDA000070248003EC42302910022C697E0FFFFFD
:10EDB000E780C05241011733FFFF6700E333A285AC
:10EDC0001306110097F0FFFFE780E04C2A8409E565
:10EDD00023110100894475B726859305210097000A
:10EDE0000000E78060ECAA8449FD8355210022855C
:10EDF00097B0FFFFE780006B49F5014997C0FFFF1F
:10EE0000E7800074635DA900184893171900BA974A
:10EE100003D707000DEF035721002390E70097C0A9
:10EE2000FFFFE780E071630625039777FF1F938755
:10EE3000E71D9C4399C70355210097500000E780C8
:10EE4000C0EF228597900000E780A0511DBF050903
:10EE500075B795443DB705C19307F00F630FF500F3
:10EE6000C547630CF5009307F5FF05453315F5001D
:10EE70004205418182800145828041657D15828005
:10EE8000B9E91733FFFFE702832503450603328400
:10EE900097000000E78060FC9305803EB305B50253
:10EEA000C205C18181CD0357E402854763F8E700BD
:10EEB0001305040197E00000E78060418357E402F6
:10EEC00041677D176385E700FD172317F4021733A9
:10EED000FFFF6700032382801733FFFFE702A31DB4
:10EEE000004283C79500444D0349140093F7F70788
:10EEF000A384F50083470400220911673369F900F0
:10EF0000A167B347F90041112A8BAE8A63ECE70E83
:10EF1000834724001307C00EB91793F7F70F6373E5
:10EF2000F71003473400C14763EEE70E8347440000
:10EF30001307E00793C707086371F70C8349840040
:10EF400083477400A209B3E9F900856763F7F90AFA
:10EF5000034A6400834754004E85220A336AFA004C
:10EF600097500000E780803A61C123962403834BC9
:10EF70003400137AFA00239A340323887403239904
:10EF8000440393890401631C090023A60402239807
:10EF900004024E8597E00000E780A0353DA00349BC
:10EFA00024004A8597000000E78020EB2397A40205
:10EFB000834744004E85A388F402E38D0BFCE30BEA
:10EFC00009FC97E00000E780602E97900000E78042
:10EFD000407281460146D6855A8597E0FFFFE7805B
:10EFE0000058A167938797033EC42302010048009D
:10EFF00002C697E0FFFFE780602E41011733FFFF55
:10F000006700E30E8544A2862686D6855A8597E05A
:10F01000FFFFE780C054A167938797033EC4230294
:10F020009100F1B7BD44C5B79144F1BF1733FFFF5D
:10F03000E702430901111C08404D3EC2B7070F000B
:10F040003EC41C083EC62A89AE8997C0FFFFE780F0
:10F0500000D7585C1C5C6346B70E6394E50063E21E
:10F06000A70E3385A740B3B7A700B305B740130673
:10F07000803E81469D8D97000100E780C0B69314C5
:10F080000501C180A1659385C503480097B0FFFFC6
:10F09000E780C0558145480097D0FFFFE780603D7D
:10F0A00083550404480097D0FFFFE780803E8355D6
:10F0B0002404480097D0FFFFE780A03D814589CC1C
:10F0C000C167FD179305F00F6388F40026859750FC
:10F0D0000000E78020E0AA85480097D0FFFFE78086
:10F0E000403903554404814501CDC167FD1793059F
:10F0F000F00F6307F50097500000E780A0DDAA85B8
:10F10000480097D0FFFFE780C0368345640448007D
:10F1100097D0FFFFE780E03583457404480097D01F
:10F12000FFFFE7800035500001478146CE854A85C4
:10F1300097B0FFFFE780E07005611733FFFF6700BE
:10F14000A3FB814481B71733FFFFE70243F983C76D
:10F15000950093F7F707A384F50097000000E78078
:10F1600020ED1733FFFF6700C3F91733FFFFE702F6
:10F1700063F583C795004111404D93F7F707A384CA
:10F18000F5002A8A3285B284AE8997D0FFFFE780E6
:10F19000003E2A8B268597D0FFFFE780403D2A89D5
:10F1A000268597D0FFFFE780603A93170B0163CA6B
:10F1B0000702E177CA97C207C183116763E3E702D9
:10F1C00093070910C207C1831307B00F637BF700D1
:10F1D00093170901C187AA8A634AF000C54763FEF5
:10F1E000570141011733FFFF670003F197B0FFFF9D
:10F1F000E7802025E31725FFD5B763080B026306D8
:10F200000902814463890A02B7077F00231064055D
:10F21000231124057CC0568597000000E780E0C3D9
:10F220009304803EB304950239A0B7077F002320E2
:10F2300004047CC081440355240497E00000E78067
:10F24000E0A2A1C497C0FFFFE78060B7269593D7DF
:10F25000F44133379500AE97BA9708DC5CDCCE8575
:10F26000528597000000E780A0DC99E02322040487
:10F27000A1679387B70348003EC42302010002C67A
:10F2800097E0FFFFE7808005A9BF814701481CDCAC
:10F29000232E0403E9B71733FFFFE70243E497C0C7
:10F2A000FFFFE7802034E1473305F5029145975091
:10F2B0000000E78040C4E55711C59777FF1F23A1E1
:10F2C000A7B681473E851733FFFF670083E31733F7
:10F2D000FFFFE702C3E09777FF1F938727B48043C0
:10F2E0003DC0835704046390A70683572404639C9E
:10F2F000B7043689B28497C0FFFFE78040AC5C5CFE
:10F3000063C3B7046395B7001C5C63EEA702834731
:10F31000640463F3F400A6872303F40483477404AE
:10F3200063F39700A687A303F4048357440441675B
:10F330007D176385E70085072312F4043C4481C7E9
:10F34000CA85268582971733FFFF670083DB97778F
:10F35000FF1F9387A7AC9C43014599C303C5870052
:10F3600082801733FFFFE70283D70111B707070039
:10F370003EC683C79500584D0AC493F7F7070AC8DD
:10F38000A384F5002A89AE8411CB1C4283C70700F1
:10F390002304F70097900000E78000342164930570
:10F3A0005402280097B0FFFFE78040249700000038
:10F3B000E78020FAAA85280097D0FFFFE780600B3E
:10F3C000300001478146A6854A8597B0FFFFE78058
:10F3D000404713044402480822CC230A010002CE0D
:10F3E00097E0FFFFE78080EF05611733FFFF6700BD
:10F3F00043D11733FFFFE70283CE01117C003ECAE1
:10F40000B70707003ECC7C003ECE83C795002E8414
:10F41000AA8493F7F707A384F500A16593855502A5
:10F42000480897B0FFFFE780601C97000000E78066
:10F4300040F2AA85480897D0FFFFE7808003500874
:10F4400001478146A285268597B0FFFFE780603F90
:10F4500005611733FFFF6700C3CA9777FF1F9387C4
:10F46000E79B9C43094599C303C597008280977722
:10F47000FF1F9387A79A9C43094599C303C5D700EB
:10F4800082809777FF1F938767999C43014599C3B3
:10F4900003C5A70082801733FFFFE702A3C2011153
:10F4A000B70708003EC683C79500404D0AC493F7CE
:10F4B000F7070AC8A384F5002A89AE8429C4144238
:10F4C000854703C7060063E0E70A834794000946BF
:10F4D00081496380C702B307F740A304E400B3394E
:10F4E000F00083C716002305F40097900000E78022
:10F4F000A01E03572403058B19C76386090097D004
:10F500000000E78000E9216493058402280097B099
:10F51000FFFFE780A00D97000000E78040F4AA8578
:10F52000280097D0FFFFE780C0F497000000E78035
:10F5300080F5AA85280097D0FFFFE78080F3014778
:10F5400081463000A6854A8597B0FFFFE780602F8F
:10F5500013047402480822CC230A010002CE97E06B
:10F56000FFFFE780A0D705611733FFFF6700C3B82F
:10F570001733FFFFE702A3B601117C003ECAB707AD
:10F5800008003ECC7C003ECE83C795002E84AA8422
:10F5900093F7F707A384F500A165938585024808D2
:10F5A00097B0FFFFE780800497000000E78020EB22
:10F5B000AA85480897D0FFFFE780A0EB97000000DE
:10F5C000E78060ECAA85480897D0FFFFE78060EAF3
:10F5D000500801478146A285268597B0FFFFE78046
:10F5E000402605611733FFFF6700A3B19777FF1F20
:10F5F0009387C7829C43014599C303C5B7008280A6
:10F600001733FFFFE702A3AD0111B70707003EC69E
:10F6100083C79500404D0AC493F7F7070AC8A3842F
:10F62000F5002A89AE8405C81C42054783C7070038
:10F630006368F7060347B400630FF700A305F400FF
:10F6400097900000E78040098347B400B9CF97D076
:10F65000FFFFE78000BF21649305B400280097B046
:10F66000FFFFE780A0F897000000E78060F8AA8518
:10F67000280097D0FFFFE780C0DF014781463000B8
:10F68000A6854A8597B0FFFFE780A01B290448089C
:10F6900022CC230A010002CE97E0FFFFE78000C4DE
:10F6A00005611733FFFF6700C3A597D0FFFFE78011
:10F6B000E0BF55B71733FFFFE70263A201117C00DB
:10F6C0003ECAB70707003ECC7C003ECE83C79500FC
:10F6D0002E84AA8493F7F707A384F500A165AD05EE
:10F6E000480897B0FFFFE78060F097000000E780D0
:10F6F00020F0AA85480897D0FFFFE78080D7500800
:10F7000001478146A285268597B0FFFFE7806013F9
:10F7100005611733FFFF6700C39E9767FF1F93873D
:10F72000E76F9C43094599C303C5C700828017331F
:10F73000FFFFE702C39A01117C00AE843ECAA165B7
:10F74000B70707002A843ECCD1057C0048083ECE8E
:10F7500097B0FFFFE78080E997000000E78020FC7A
:10F76000AA85480897D0FFFFE780A0D0500801473E
:10F770008146A685228597B0FFFFE780800C056152
:10F780001733FFFF6700E3971733FFFFE702239567
:10F7900083C7950093F7F707A384F500970000004F
:10F7A000E78020F91733FFFF6700A3951733FFFFAA
:10F7B000E702439183C795000329C501411193F7DF
:10F7C000F707A384F5001C4283C90700854763E659
:10F7D00037079777FF1F9387A7BB9C432E84AA8484
:10F7E00085CF97000000E78080F389476306F50224
:10F7F000630409028347C900638037032306390184
:10F8000097900000E78040ED83572903898B89C7D3
:10F8100097D00000E780E0B72685A285970000001A
:10F82000E78020F1A167CD0748003EC42302010014
:10F8300002C697E0FFFFE78060AA41011733FFFF90
:10F840006700838B9767FF1F9387475D9C431D4528
:10F8500099C303C5E70082801733FFFFE7022388BF
:10F860000111B70707003EC683C79500584D0AC46B
:10F8700093F7F7070AC8A384F5002A89AE8415C751
:10F880001C4283C7070093968701E18663C406067E
:10F8900085466381D7068346E7006388F600230721
:10F8A000F70097900000E78020E321649305E400CF
:10F8B000280097B0FFFFE78060D397000000E78043
:10F8C000A0F8AA85280097D0FFFFE78080BA0147FB
:10F8D00081463000A6854A8597B0FFFFE78060F635
:10F8E0003504480822CC230A010002CE97E0FFFF2E
:10F8F000E780C09E05611733FFFF670083801723F1
:10F90000FFFFE702C37D01117C003ECAB707070075
:10F910003ECC7C003ECE83C795002E84AA8493F70C
:10F92000F707A384F500A165B905480897B0FFFF64
:10F93000E780C0CB97000000E78000F1AA85480867
:10F9400097D0FFFFE780E0B2500801478146A285CB
:10F95000268597B0FFFFE780C0EE05611723FFFF04
:10F960006700237A1723FFFFE702C375AA840144C7
:10F970001769FF1F1309C94AE14997C0FFFFE780D4
:10F9800060C66344A400014519A8330534038327E6
:10F9900009003E95835725006397970011051723AB
:10F9A000FFFF670063750504C9BF032E8500630A66
:10F9B0000E121763FF1F1303636503230300631510
:10F9C000030029436390061203234E0163150300CD
:10F9D0001D43639907101723FFFFE702C36DC68914
:10F9E000428A3E89BA8AB684328BAE8B2A84B5E1CC
:10F9F00003554E0019E501431A851723FFFF6700E1
:10FA0000036FA167A98F116763FBE70097000000F0
:10FA1000E78080F5814597F0FFFFE7808013084479
:10FA2000B70700E05841F98F18455CC1B707001FC0
:10FA3000F98F1CC55C4991C7610597E00000E7801C
:10FA4000408BE38A09FA228597900000E78060C620
:10FA50005DB7328597C00000E78040430D4349DD24
:10FA60001C44116703D54700A167A98F63FBE7001A
:10FA700097000000E78040EF814597F0FFFFE780A7
:10FA8000400D0323840093164B01D1828347B300BA
:10FA9000035663008588FD8BA305F300FD777D8EFB
:10FAA000558EFD76FD16B204F18E83274301C58E77
:10FAB000231273012313D3002304530123052301CD
:10FAC000A3044301BDDF228597B0FFFFE78040CA52
:10FAD000AA850844B5D1610597D00000E780207F52
:10FAE0008DB71D431A8582801723FFFFE702835DD0
:10FAF0000569AA84AE89328A0144FD5A7D1997C0EE
:10FB0000FFFFE780E0A26347A40001451723FFFF42
:10FB10006700835ED84493171400BA9703D7070091
:10FB2000631F37032390570163070A0026859790C8
:10FB30000000E780A0809C449DC383D76700B3F793
:10FB40002701639E3701D2880148814701478146DA
:10FB500001468145268597000000E78040E50504C1
:10FB600079BF1723FFFFE702E35579711C103EC4EC
:10FB7000B7070F003EC61C103EC883C79500AA8A6F
:10FB8000328593F7F707A384F5002E89328497D046
:10FB9000FFFFE780C09D93170501C187635AF006F8
:10FBA000AA89228597D0FFFFE780609C2A8A4E852C
:10FBB000032B040097B0FFFFE780209839ED8357AF
:10FBC000440081440544F11793B71700A303F100E3
:10FBD00083457100DA872287D2864E86280097E017
:10FBE000FFFFE780A058014781463000CA8556854F
:10FBF00097B0FFFFE780E0C4A1679387F703480849
:10FC00003ECC230A810026CE97D0FFFFE780006D0F
:10FC100045611723FFFF6700234EA285130671007D
:10FC200097E0FFFFE7802067AA84094455D15285F9
:10FC300097E0FFFFE78020D50D4459D90546D285CE
:10FC4000268597000000E78060EA2A8451B71723D1
:10FC5000FFFFE702C3488355070003462700411111
:10FC60002A842E8532C62EC497E0FFFFE780A0D1FC
:10FC700001C93246A245228597000000E78000E7CF
:10FC800041011723FFFF6700C3471723FFFFE70268
:10FC9000834283C795004111AA8A93F7F707A3848B
:10FCA000F5003285AE89328497D0FFFFE780208C43
:10FCB00093170501C1876357F00AC1452A8A228537
:10FCC00097C0FFFFE78040712A8D228597D0FFFF04
:10FCD000E780E0892A89228597D0FFFFE7800087A7
:10FCE000930705F893F7F70F1307E007AA8B637BD9
:10FCF000F706228597D0FFFFE78040852A8C228572
:10FD000097D0FFFFE7808084AA8C5285032B0400E4
:10FD100097B0FFFFE780608239E9835744002311E1
:10FD200001008144F11793B71700A300F1000544C7
:10FD30000347110083562100938784005685DA8893
:10FD400022885286CE8597F0FFFFE780E0A7A16763
:10FD5000E90748003EC42302810026C697D0FFFF72
:10FD6000E780C05741011723FFFF670043381306A0
:10FD70001100A28597E0FFFFE780E051AA8409E522
:10FD80002311010009446DB7930521006A8597F09E
:10FD9000FFFFE78060F12A8441FD835521009356DF
:10FDA000C9001316490185486688E2875E87858AFF
:10FDB0005182268597000000E78060BF2A848DBFAE
:10FDC0001723FFFFE702232F83C7950041112A8BDA
:10FDD00093F7F707A384F5003285AE89328497C084
:10FDE000FFFFE780C07893170501C1876352F00ACF
:10FDF0002A8A228597C0FFFFE7806077AA8A22853A
:10FE000097C0FFFFE780A0762A89228597C0FFFF71
:10FE1000E780C073930705F893F7F70F1307E00720
:10FE20002A8C6377F706228597C0FFFFE780007270
:10FE3000AA8C228597C0FFFFE78040712A8D5285EA
:10FE4000832B040097A0FFFFE780206F39E58357DD
:10FE5000440085440144F11793B71700A301F10052
:10FE600003473100930784005A85DE882688D686AA
:10FE70005286CE8597F0FFFFE78000958D474800BA
:10FE80003EC42302910022C697D0FFFFE7800045C1
:10FE900041011723FFFF67008325A2851306310068
:10FEA00097E0FFFFE780203F2A84894455D9935685
:10FEB000C9001316490185486A88E6876287858AE2
:10FEC0005182D68597000000E78060AEAA8449BFC2
:10FED0001723FFFFE702031F2A8981440144617A47
:10FEE000916A176BFF1F130B6B1297B0FFFFE78030
:10FEF000206563C7A40022851723FFFF6700C31F87
:10FF00008327090093991400CE9703D50700330780
:10FF10004501420741836364570305C103270B0072
:10FF200019C785453E8597400000E78060E9832733
:10FF300009000504CE972390070085047DB797003C
:10FF40000000E78060A2832709000504CE97239074
:10FF5000070065D5814597F0FFFFE78080BFF1BFBF
:10FF60001723FFFFE702031683C7950041112A8A72
:10FF700093F7F707A384F50032852E89328497C062
:10FF8000FFFFE780C05E93170501C187635AF00445
:10FF9000AA89832A040097A0FFFFE780005A31E571
:10FFA0008357440085440144F11793B71700A30118
:10FFB000F10003483100D68752850147CE86268658
:10FFC000CA8597D0FFFFE780406BA167F50748001F
:10FFD0003EC42302910022C697D0FFFFE780003085
:10FFE00041011723FFFF67002311A285130631008B
:10FFF00097E0FFFFE780202A2A8489445DD997672C
:020000040001F9
:10000000FF1F9387A7009C4381CF044997B0FFFF50
:10001000E7800053AA85268597400000E78040DAF4
:100020001305040197000000E780C0EA228597804D
:100030000000E78000338144ADBF1723FFFFE702D4
:10004000830783C795004111AA8A93F7F707A38412
:10005000F5003285AE8932842311010097C0FFFF7D
:10006000E780E05093170501C1876354F0062A8AA0
:10007000C145228597C0FFFFE7800036AA8B5285D5
:10008000032B040097A0FFFFE780204B21E9835753
:10009000440085440144F11793B71700A300F10011
:1000A0000348110003572100DA875685D286268639
:1000B000CE8597D0FFFFE780405CA167938727023A
:1000C00048003EC42302910022C697D0FFFFE7807C
:1000D000E02041011723FFFF67006301A28513069B
:1000E000110097E0FFFFE780001B2A8489444DD967
:1000F0009767FF1F938787F198433E8901CF044993
:1001000097B0FFFFE780C043AA852685974000008F
:10011000E78000CB1305040197000000E78080DB37
:1001200097B0FFFFE780C04195443DD9930521007A
:100130005E8597F0FFFFE78020B7AA8435F11C4861
:100140000357210022852390E70097800000E78075
:10015000402183270900A9D70355210097400000BB
:10016000E780A0BD35BF1723FFFFE702C3F483C7B5
:1001700095004111AA8A93F7F707A384F500328509
:10018000AE89328497C0FFFFE780603E9317050178
:10019000C1876351F0062A8A228597C0FFFFE78056
:1001A000003D2A895285032B040097A0FFFFE780BA
:1001B000C03831E58357440085440144F11793B7B3
:1001C0001700A301F10003483100DA8756854A87FA
:1001D000D2862686CE8597D0FFFFE780004AA167AA
:1001E000F90748003EC42302910022C697D0FFFFC2
:1001F000E780C00E41011723FFFF670043EFA28590
:100200001306310097E0FFFFE780E0082A84894465
:100210005DD99167CA97C2071167C1831307F7EFCA
:100220008544E362F7FA9767FF1F938727DE9843B9
:10023000BE8B01CF044997B0FFFFE7806030AA85ED
:10024000268597400000E780A0B7130504019700BA
:100250000000E78020C897B0FFFFE780602E95443C
:100260003DD11C48228581442390270197800000BE
:10027000E780200F83A70B00B9D74A85974000007D
:10028000E780A0AB89B71723FFFFE70243E52A8485
:100290004105B28497000000E780C0C311C52285E4
:1002A00097800000E780E00B81460146A685228505
:1002B00097800000E780C04E1C4C89C7DC4799C37B
:1002C000228582971723FFFF6700A3E39767FF1F2D
:1002D0009387C7B49C43014599C313850701828066
:1002E0009767FF1F938787B3884382801723FFFF99
:1002F000E702E3DE9317C600DD8DC2054111C1811F
:100300002A8432C697C0FFFFE780A01832462285B4
:1003100011829375F60F97C0FFFFE78080154101AA
:100320001723FFFF6700E3DD1723FFFFE70283D9F1
:1003300079713C083ED2B7070C003ED43C083ED64B
:1003400083C79500AE842A8993F7F707A384F50045
:10035000A16593853504481097A0FFFFE780002929
:10036000C165FD150144176AFF1F130AAACB930A42
:10037000400EAE892E8B2EC697B0FFFFE780401F40
:100380004205931704014181C183B24563E9A70285
:10039000C167FD176387F500481097C0FFFFE7802E
:1003A000400F501001478146A6854A8597A0FFFF60
:1003B000E780204945611723FFFF6700E3D3330738
:1003C000540383270A0BBA9703D6C701630A360181
:1003D000638A3501481097000000E78060F1DA85F4
:1003E000050451BFB285EDBF1723FFFFE702A3CC81
:1003F00079717C083EC8B70711003ECA7C083ECC24
:1004000083C79500AA89328593F7F707A384F5007F
:100410002E8997C0FFFFE780801585676378F50414
:10042000A165AA848905080897A0FFFFE780001C42
:10043000268597400000E78060ED133415000A041C
:10044000A285080897C0FFFFE780A002A6850808DC
:1004500097C0FFFFE780E00325CC014781461008E5
:10046000CA854E8597A0FFFFE780A03D4561172311
:10047000FFFF6700C3C7B30754030327CA0ABA972D
:1004800003D70700631C970003D627006380650528
:10049000080897000000E780A0E5DE8505042EC669
:1004A00097B0FFFFE780C00D42059317040141811B
:1004B000C183B245E3E1A7FCC167FD17E38FF5F8FF
:1004C000080897C0FFFFE780C0FC41BFB285F9B7BD
:1004D000C165FD150144176AFF1F130AAAB4930AE8
:1004E00080022E8BAE8B65BF1723FFFFE70223BF71
:1004F00018418347170083460700A207D58FD2070C
:10050000D1832390F50083472700034717008D45CB
:10051000A207D98F91832310F60097C0FFFFE780D1
:1005200060EA1723FFFF6700C3BD1723FFFFE70241
:1005300063B9C16401441769FF1F1309A9AE930988
:100540008002FD1497B0FFFFE78080036347A4009B
:1005500001451723FFFF670023BA330534038327C0
:10056000C90A3E9583570500E38597FE0504D9BF68
:100570001723FFFFE70203B52A8AAE89B284B68A41
:1005800097400000E78080D819E591473E85172302
:10059000FFFF670063B62A894E8597C00000E78099
:1005A000E08E2A84638E0A048D476DD103570500BF
:1005B000C547E31D47FD0347F9018546AD47E317EE
:1005C000D7FC8347450081CF4146A6855D0597F05E
:1005D0000000E780C09E814755D9AD4745BF13094C
:1005E00065012302E500CA85268597100000E78093
:1005F000606231C1A547E38B0AF82302040079B792
:1006000005C183570500E39247F94146A6851905C0
:1006100097F00000E780A09A81472DD99947BDB790
:100620004E8597000000E78080F02A84954739DDE9
:10063000130955004DBF4146A685231044012311DF
:1006400034011305190097F00000E780A099228576
:1006500097800000E780A0EA81470DBF1723FFFFC6
:10066000E702E3A779717C003ECCB7070A003ECED3
:100670007C003ED083C79500B2842E8493F7F707A1
:10068000A384F5001306A1002A892C002685970073
:100690000000E780A0E5A16528088D0597A0FFFF71
:1006A000E780C0F490408355A10003558100854642
:1006B00097000000E78000ECAA84AA85280897C06C
:1006C000FFFFE78000DB0356A10083558100280867
:1006D00097000000E780C0C1300801478146A2852D
:1006E0004A8597A0FFFFE780C015854748103ED494
:1006F0002302910202D697D0FFFFE78020BE45611A
:100700001723FFFF6700E39F1723FFFFE702239DE7
:1007100079717C003ECCB7070A003ECE7C003ED00B
:1007200083C79500B2842E8493F7F707A384F5005E
:100730001306A1002A892C00268597000000E78077
:10074000E0DAA16528088D0597A0FFFFE78000EAA1
:1007500090408355A1000355810081469700000019
:10076000E78040E1AA84AA85280897C0FFFFE780B8
:1007700040D00356A100835581002808970000004F
:10078000E78000B7300801478146A2854A8597A0D7
:10079000FFFFE780000B48102302910202D402D62B
:1007A00097D0FFFFE78080B345611723FFFF670005
:1007B00043951723FFFFE702839297000000E7802D
:1007C00060DB1723FFFF6700C3939757FF1F9387D3
:1007D0002765884382801723FFFFE70243908357F2
:1007E00025004111AE842A842307B10017F5FFFFCD
:1007F000130525466C002316F10097A0FFFFE78044
:10080000404691C4228597800000E780E0D6FD57DE
:100810002310F4001306200281451305540097208D
:10082000FFFFE780C08E41011723FFFF6700638D44
:100830001723FFFFE702038979717C003ECCB707DD
:100840000A003ECE7C003ED083C79500AA89AE84C4
:1008500093F7F7073285A384F5001306A1002C0057
:1008600097000000E78080C803558100114497403D
:100870000000E780A0A915C50355A100014497B069
:100880000000E780A06011CD035705008357810069
:1008900045446318F700854597000000E780E0F3C2
:1008A0000144216993053900280897A0FFFFE780DC
:1008B000E0D3A285280897C0FFFFE78080BB0356DE
:1008C000A10083558100280897000000E78040A21E
:1008D000300801478146A6854E8597A0FFFFE78037
:1008E00040F648104AD42302810202D697D0FFFF77
:1008F000E780C09E45611713FFFF6700E37F171372
:10090000FFFFE702237C9757FF1F938727512A8415
:1009100088432E8915C5035745038357C4016311C6
:10092000F7022326050223180502410597D000008F
:10093000E780209C6306090097800000E78060DB69
:1009400081449759FF1F9389E96D130A800297B07C
:10095000FFFFE780E0C263C4A4049757FF1F93879B
:10096000A7549C4399C70355C40197200000E78012
:10097000C0BD63070900228597800000E780C0A002
:100980001306400E814522859710FFFFE7802078EF
:10099000FD57231EF4001713FFFF6700E37533852F
:1009A000440383A7C90A3E95035705008357C40132
:1009B0006317F700CA8597000000E78000E285040E
:1009C00079B71713FFFFE702E36F83C79500411163
:1009D000AA8993F7F707A384F5003285AE8497C000
:1009E000FFFFE780C0B885676378F5042A899740E0
:1009F0000000E780A091014401CD83D70400314479
:100A000063882701854597000000E78080EF014457
:100A10004E85A2864A86A68597D0FFFFE780609D17
:100A2000A1679387170448003EC42302810002C6D1
:100A300097D0FFFFE780808A41011713FFFF67000F
:100A4000A36B1713FFFFE702E3679757FF1F938717
:100A5000E73C804329C4014597C00000E78000219E
:100A600081470148C1641CDC232E040323200404B5
:100A70001759FF1F1309095B01449309400EFD1428
:100A800097B0FFFFE780C0AE634FA400814517F524
:100A9000FFFF1305857F97A0FFFFE780801C1713DA
:100AA000FFFF67006365330534038327090B3E9519
:100AB0008357C50163879700854597000000E7804D
:100AC00040E4050475BF9357050113D78700A38041
:100AD000F50093170501C183A1832380E5002381DD
:100AE000F500A381A50082801713FFFFE702235FB3
:100AF0002300050083C71500A300F50083C7250068
:100B00002301F50083C73500A301F50083C7450025
:100B10002302F50083C75500A302F50083C76500D3
:100B200093059500A30305002303F50023040500A6
:100B3000328597000000E78040F91713FFFF670038
:100B4000435C1713FFFFE702E3574111E9540DCD52
:100B500085CD93F9C5FF2E842A89AA84338AA900FA
:100B6000B7EA040063189A020D88854411CCB7E7F0
:100B700004009C5F82972AC622866C0033053901E7
:100B800097E00000E7800046268541011713FFFF2C
:100B90006700835683A78A03910482979317050100
:100BA000C183A183A38EF4FE93570501238FF4FE26
:100BB000A183238EA4FEA38FF4FE6DB763E6D50256
:100BC0001713FFFFE702A351B28741113686BE8596
:100BD00036C697E00000E780E040B2464101368526
:100BE0001713FFFF6700E3518146368582808387B4
:100BF00005001387F5003D05FD8793F777088346C9
:100C000007007D158606B58FA300F5006307B700C2
:100C10007D17834717009D83DDB782801713FFFF81
:100C2000E702E34BB7E7040083A7070932872A8668
:100C30003A858297133515001713FFFF6700634C41
:100C400015C181478DC11713FFFFE7024349414694
:100C500097E00000E780003985473E851713FFFFC6
:100C60006700234A81473E8582801DCD1713FFFF11
:100C7000E702E346414681452A849710FFFFE7805B
:100C8000004941468145130504039710FFFFE780A3
:100C900000480147C1672322040438C87CC80545C1
:100CA0001713FFFF6700E3450145828081473DCD73
:100CB000B5CD1713FFFFE7028342B2842E891306D6
:100CC000800581452A849710FFFFE7804044CA854C
:100CD00024C4268597000000E780C0F64146814580
:100CE00022859710FFFFE78080423044A28522854D
:100CF00097000000E780C0F293040401A2852685D6
:100D000097000000E780E0EEA68513050402970037
:100D10000000E78000EE228597000000E78020F5C4
:100D200085473E851713FFFF6700A33D3E85828000
:100D30001713FFFFE70203394111E9540DCD85CDAB
:100D400093F9C5FF2E842A89AA84338AA900B7EAB9
:100D50000400639844030D88814411CCB7E7040074
:100D60009C5F82972AC622866C003305390197E082
:100D70000000E7802027268541011713FFFF670049
:100D8000A33783A78A039104829793170501C18330
:100D9000A183A38EF4FE93570501238FF4FEA18354
:100DA000238EA4FEA38FF4FE6DB765CD1713FFFF4E
:100DB000E7024331B28411E605451713FFFF6700D0
:100DC000A3332A842E890145EDD93C487848B3E6FF
:100DD000E700E5D69386F7FFB3B7F6007D17032A41
:100DE0004404BA9734C87CC863050A06C149130590
:100DF0000A03B38949412295637D3601B2862E8666
:100E0000A68597000000E780A0DB7C40BE9464C00C
:100E100065B7CE862E86CE8597000000E78040DA43
:100E2000C114D2944E9923220404A287930604018C
:100E300003C7070003C607038507318FA38FE7FEAB
:100E4000E398F6FE3044A285228597000000E780F3
:100E500020DD2699C1493306994063EC9900A9DC4D
:100E6000A686A6851305040397000000E78040D5F9
:100E700079BF8147B306F4003307F6000347070044
:100E800083C5060085072D8F2380E600E39437FF96
:100E90003044A285228597000000E78060D8C11405
:100EA0005DBF014582800DC11713FFFFE7022323B9
:100EB0001306800581459710FFFFE7804025054513
:100EC0001713FFFF6700E32301458280814749C56F
:100ED000C1C51713FFFFE7028320FC4141462E8462
:100EE000AA846399C70413860501A2878146C14578
:100EF00003C7070003C507038507298F3305D600FD
:100F0000034505008506298FA38FE7FEE392B6FE11
:100F10003044A285268597000000E78060D02285B6
:100F200097000000E78060F885473E851713FFFFB4
:100F30006700231D138507031D8E81452295971099
:100F4000FFFFE780C01C7C40130700F81306040273
:100F5000A2972388E70251BF3E8582801713FFFFC7
:100F6000E702E3176D712E84B284AA8590102800E1
:100F7000368997000000E780A0D309EDD55725A05A
:100F800050400C40280097000000E78040E27DD5EB
:100F9000FD142104F5F42C004A8597000000E78039
:100FA00020F3814761DD3E8551611713FFFF670024
:100FB00043151713FFFFE702831241112EC432C6F7
:100FC0002C00054697000000E78080F941011713C7
:100FD000FFFF670003131713FFFFE7024310011120
:100FE0002A842EC602C802CA02CC02CE97E00000B4
:100FF000E780C023B2462A86A28508089700000031
:10100000E78060FB1375F50F05611713FFFF67009D
:10101000430F1713FFFFE702830C7971B2872A840D
:1010200021462308B10013051101BE853AC436C616
:1010300097E00000E78000FBB246930591013685FA
:1010400097000000E78060A82285141035460C0840
:1010500097000000E78020F62A84224701E9214614
:101060000C103A8597E00000E780C0F722854561C3
:101070001713FFFF6700E3081713FFFFE7022306BC
:101080007171AE84AA850A85328497000000E780DA
:1010900060BB11C90A86A685228597000000E780FB
:1010A00020B8814711E1C5473E854D611713FFFF09
:1010B000670023051713FFFFE70263FF1D712A8AEC
:1010C000B289BE8435468547130511012E8CB68A38
:1010D0003A8BC28C468D2308F10097E00000E78030
:1010E00060F010100C085285231F010097000000CB
:1010F000E780C0F82A843DEDA1476313FD089307FC
:10110000900591E0E5473546E285130511011399F5
:101110000A012308F1001359090197E00000E78054
:1011200060EC1357890093978A00D98F90080C08B8
:101130005285231FF10097000000E78020F42A84E5
:1011400015E9A1E49387FA0091831379F9003EC66B
:10115000631309004149668B8144C14B854DB247F9
:10116000639F970C6A868C0033855C0197E00000D2
:10117000E78040E7228525611713FFFF6700E3F64C
:1011800093079004C9F0A547BDBF834701050947F0
:10119000C14B2308F10083471105A58FA308F10077
:1011A00093872400814463E1FB04014714083386DC
:1011B000E6008C08B386E400BA95DA9683C606008A
:1011C00083C505000507AD8E2300D600E390E7FE3A
:1011D0004147639CE70490080C0852859700000083
:1011E000E780C0E925D181A0B3069B00BA8710082B
:1011F000B305F60090083E9603C5060003460600B8
:1012000085078506298E2380C500E39277FF998F95
:1012100090080C085285BE9497000000E78000E615
:101220008947014749D12A84B1B790083E960346C1
:1012300006001408BE962380C600850759BFB24732
:1012400085046387971481471808B306F700980848
:101250003E973386F90003470700034606008507DB
:10126000318F2380E600E39177FF90080C085285C8
:1012700097000000E78080E05DF53546E2851305C4
:1012800011012308B10197E00000E780A0D5139772
:1012900004014183939784002183D98F10180C088F
:1012A0005285231FF10097000000E78020DD25FD17
:1012B000814710183387F9003E960347070003461D
:1012C0000600B306FB008507318F2380E600E3921A
:1012D00077FF65A81808B306F70098083E9733868D
:1012E000F90003470700034606008507318F238076
:1012F000E600E3E127FFCA87639E770990080C08A0
:10130000528597000000E78060D711FD8147980063
:10131000B306F700900818103E973E960347070063
:10132000034606008507318F2380E600E39177FFAF
:101330003546E285130511012308B10197E000004D
:10134000E78040CA13970401418393978400218367
:10135000D98F10180C085285231FF1009700000048
:10136000E780C0D1E31105EC814710183387F900FD
:101370003E960347070003460600B306FB008507B9
:10138000318F2380E600E3E227FFC109410BC1BB97
:10139000814785B79408BE9683C6060018083E9715
:1013A0002300D700850789BF638006321713FFFF2C
:1013B000E702E3CF59712A84BE89B28B854735464F
:1013C000130511022E8B468C4289BA8A368A230075
:1013D000F10297E00000E780E0C010180C102285B1
:1013E0002317010297000000E78040C96318051227
:1013F000A147631FFC069307900563930900E54727
:101400003546DA851305110293140A012300F1020F
:10141000C18097E00000E780E0BC93178A0013D7F3
:101420008400D98F90080C1022852317F1029700B1
:101430000000E780A0C47DE1639209049307FA00ED
:10144000BD88918391E0C144C207C183DE8C814A8B
:101450003EC6414DB24763E2FA0E6286B3854B0148
:10146000881097E00000E78080B54DC93D557DA00C
:1014700093079004E39609F8A54759B783470105F8
:101480000947C14C2300F10283471105B3C7F90096
:10149000A300F10293872900814963E1FC0481469E
:1014A00018103306D7008C083387D900B6955697A5
:1014B0000347070083C5050085062D8F2300E6003E
:1014C000E390D7FE41476390E70690080C10228511
:1014D00097000000E78080BA35D189A0B3863A0131
:1014E000BA871010B305F60090083E9603C50600B3
:1014F0000346060085078506298E2380C500E392F2
:1015000097FF3387EC4090080C102285BA9997001A
:101510000000E780A0B68947014741D165611713F4
:10152000FFFF670083BC90083E9603460600141038
:10153000BE962380C600850779B7B247850A93997E
:101540000A01939D8A0093D909016391570F85473A
:101550003546DA85130511022300F10293D989007B
:1015600097E00000E78000A8B3ED3D0190000C106B
:1015700022852317B10397000000E78020B059FDB2
:101580008147A68963EA970626860C084A8597E074
:101590000000E78020A581471810B306F700100867
:1015A00098083E973E9603470700034606008507C6
:1015B000318F2380E600E3E197FE639FA905900841
:1015C0000C10228597000000E78040AB21F981478D
:1015D0009810B306F700900818183E973E960347F8
:1015E0000700034606008507318F2380E600E3915C
:1015F000A7FF4109C10CB9BD18089000B306F70058
:101600003E963387FC000347070003460600850724
:10161000318F2380E600B5B798084E97034707003F
:101620001C10CE972380E700850941BF85473546CA
:10163000DA85130511022300F10293D9890097E09E
:101640000000E780209AB3ED3D0190000C10228548
:101650002317B10397000000E78040A2E31005ECD8
:10166000814718089000B306F7003E963387FC00C8
:1016700003470700034606008507318F2380E600F5
:10168000E391A7FF41460C084A8597E00000E780F8
:10169000609581471810B306F700100898083E9728
:1016A0003E9603470700034606008507318F2380D7
:1016B000E600E391A7FF90080C1022859700000038
:1016C000E780C09B1DD599BD7D5582801713FFFF14
:1016D000E702E3A001112A842E8593055100328987
:1016E00002C002C202C402C69304740097F0FFFF56
:1016F000E780A03D1D46A6851305910097E00000F8
:10170000E780408E10088A854A8597000000E780B0
:10171000E09619ED93071400180883C607000346E6
:10172000070085070507B18EA38FD7FEE397F4FE68
:1017300005611713FFFF6700C39C1713FFFFE70244
:1017400063982E848C414111AA89838715003289C0
:10175000914463D30700A1449757FF1F938747C362
:101760009C43A1C7C1CA8D472310F10083C7250040
:101770004A852301F10083C73500A301F10083C727
:1017800045002302F10083C75500A302F10083C77F
:10179000650093059100A30301002303F1002304D6
:1017A000010097F0FFFFE78040320C404A860A852F
:1017B00097F0FFFFE780803303280400835644003E
:1017C000A6881D0881470147E51642868A854E8511
:1017D00097000000E780408E2A8919E5A6852285BA
:1017E00097B0FFFFE780A0C24A8541011713FFFFB2
:1017F000670083904A860A8597F0FFFFE780002FF5
:101800006DB71713FFFFE702E38B2E848C41411164
:10181000AA89838715003289914463D30700A144C4
:101820009757FF1F9387C7B69C43A1C7C1C68D4773
:101830002310F10083C725004A852301F10083C7E7
:101840003500A301F10083C745002302F10083C7DF
:101850005500A302F10083C7650093059100A3031F
:1018600001002303F1002304010097F0FFFFE7804C
:10187000C0250C404A860A8597F0FFFFE7800027C5
:1018800083564400032804008A85858EC2061D08FD
:10189000C1822312D400A68881470147E5164286FB
:1018A0004E8597000000E78060B041011713FFFFED
:1018B000670083844A860A8597F0FFFFE78000234C
:1018C0004DBF1713FFFFE7028381B335B00001114D
:1018D00085052A891315F601336515012308B10022
:1018E0009305110136843AC632C03EC442C297F015
:1018F000FFFFE780801DA2471248425593D687001C
:10190000230BF1009305910193578800A30AD1009E
:10191000A30BF100230C010197F0FFFFE780E01A11
:101920003247024603280400B337E00083564400E0
:101930009207914411C2A1444A85A68842860C08A8
:1019400097F0FFFFE78040772A8919E5A685228571
:1019500097B0FFFFE780A0AB4A8505611703FFFF43
:101960006700237A1703FFFFE702C37501113EC624
:101970008647B335B0008505AA891315F6015D8D3C
:101980002308B1009305110136843A89B28442C418
:1019900046C297F0FFFFE780401322489248164561
:1019A00093578800A30AF1009305910193D788000B
:1019B000230B0101A30BF100230C110197F0FFFF92
:1019C000E780A0103247104083564400B337E00050
:1019D000920703280900914891C0A1480C084E8540
:1019E00097000000E780809CAA8401E983554400A9
:1019F0004A8597B0FFFFE78080A126850561170320
:101A0000FFFF6700636FAA959307F00F17070100A8
:101A1000130787616317B50013C5F7FF1375F50F3B
:101A2000828005058346F5FFB58FBA9783C7070007
:101A3000D5B70357450014419307F00F170601006F
:101A40001306865E3697420741831395060141814E
:101A5000631BE500AD8FB29703C50700130515F3AF
:101A6000133515008280850603C5F6FFA98FB2974E
:101A700083C70700D9BF1703FFFFE7024366B2879A
:101A800036842E86BA86AA853E85BA8497F0FFFFF3
:101A9000E7806052634F0500228597D00000E78001
:101AA000E0782A86A686A285268597F0FFFFE78044
:101AB00080501703FFFF6700C3641703FFFFE702AF
:101AC00063605D712A8BAE8A1705010013054553CB
:101AD0002C00B284368ABA893E8997F0FFFFE780EE
:101AE000C04F2A845DE134104146DA85280097F022
:101AF000FFFFE780404C2A8449E98547A303F100B2
:101B0000A6C2930771002408BEC4A68685470D4669
:101B10002C18281002DC02DED6C0BEC697F0FFFFEC
:101B2000E78000442A8435E183477102A6860D468A
:101B300093F7F7072300FA00C1473EDE2C188947C8
:101B4000281026DCA303F10097F0FFFFE780404157
:101B50002A8405ED4146A6854E8597D00000E78092
:101B600060488D47A6860D462C182810A303F10067
:101B700097F0FFFFE780C03E2A8401E94146A68531
:101B80004A8597D00000E780E04522856161170310
:101B9000FFFF670063561703FFFFE702435497F701
:101BA00000009387E7A1984383C7470079712A898A
:101BB000AE8417050100130525450C083AC4230619
:101BC000F10097F0FFFFE78040412A8405ED1410F3
:101BD0004146CA85080897F0FFFFE780C03D2A8488
:101BE00015E1140815462C00081097F0FFFFE78058
:101BF000803C2A8401E921462C08268597D00000E4
:101C0000E780403E228545611703FFFF6700634F71
:101C10001703FFFFE702A34C97F700009387479A4B
:101C20009C477971AA842E84170501001305453E4F
:101C30000C083EC697F0FFFFE780203A0DE914102C
:101C40004146A685080897F0FFFFE780C03605E10A
:101C5000140811466C00081097F0FFFFE780A035CC
:101C600019E58347F10193F7F7032300F400456179
:101C70001703FFFF6700E3481703FFFFE702234650
:101C80003688A14881470147E54697F0FFFFE78086
:101C9000A0421703FFFF6700C3461703FFFFE702D9
:101CA00003443688A14881470147E54697F0FFFF86
:101CB000E780C06F1703FFFF6700A3441703FFFF10
:101CC000E702E34101112A842E850C0832C697F001
:101CD000FFFFE780803009ED3247970601009386C9
:101CE000A6311008C145228597000000E780E0D8A2
:101CF00005611703FFFF6700C3401703FFFFE702FB
:101D0000033E4111C1472EC032C48A8509463EC2F6
:101D10003EC697F0FFFFE780A02441011703FFFFB5
:101D20006700233E1703FFFFE702633B4111AE86C6
:101D300013061009AA850A8502C002C202C402C69F
:101D400097F0FFFFE780202741011703FFFF67009F
:101D5000433B1703FFFFE7028338328797060100F2
:101D60009386862B2E869305000297000000E7805D
:101D7000C0D01703FFFF6700C3381703FFFFE70258
:101D800003367971C1472ACC2ED032D42C080D46A7
:101D900028003ECE3ED23ED602C402C602C802CAC7
:101DA00097F0FFFFE780C01B45611703FFFF670047
:101DB00043351703FFFFE70283320111AA842E8403
:101DC000170501001305C5258A8597F0FFFFE780F9
:101DD000C02015E514084146A6850A8597F0FFFF47
:101DE000E780601D09ED8347E1010347F101A20788
:101DF000D98FCA07C9836177D98F2310F400056191
:101E00001703FFFF6700E32F15CD1703FFFFE7025E
:101E1000032D9747FF1F9387270590439745FF1F83
:101E20009385C5041745FF1F1305050097D00000D3
:101E3000E78000C51745FF1F130505FF1703FFFFC8
:101E40006700232C1745FF1F130505FE82808DCDEB
:101E50001703FFFFE702A3289747FF1F9387C700D9
:101E6000944301112E840A869745FF1F9385050030
:101E700097D00000E78040C60A85029401450561BD
:101E80001703FFFF6700E3277D5582801703FFFFDD
:101E9000E702E32497D00000E78080D19747FF1F37
:101EA00023A4A7FC17F5FFFF1305E5C997B00000B1
:101EB000E780C0741703FFFF6700A3241747FF1FC5
:101EC0001307C7FC9317150008433E95FD572310D1
:101ED000F50082801703FFFFE70263202A84084091
:101EE00009E51703FFFF6700C3211C4158401CC0D0
:101EF0006313E5005CC08347550023200500F99B70
:101F0000A302F50097A0FFFFE780E07CC9BF17039D
:101F1000FFFFE702231B9747FF1F938727F998438B
:101F20002A8411CB8347350093F7070289C70355ED
:101F30000500894502971305440197B00000E7802A
:101F4000403B835504000355E40097300000E780D0
:101F5000A00C485819C597A0FFFFE780C077232A37
:101F600004021305840397000000E780E0F6814433
:101F7000B1499790FFFFE780E06A63CBA4028347F3
:101F800034002320040493F727FCA301F400004845
:101F90009790FFFFE780006A1316150081452285A0
:101FA0009700FFFFE780A0161703FFFF6700C31429
:101FB000B38734030329040385043E994A859700B7
:101FC0000000E78060F12304090065B7834735000E
:101FD00093F7070299E3014582808357E500E39C6C
:101FE000B7FEC167FD176316F600054582800545FB
:101FF00099A81703FFFFE702830E93170601C18715
:10200000B2842A8401496359F002835705009DCBAD
:1020100001456367F600034584003E953325A6001D
:102020001375F50F0DA01C4813171900BA9783D725
:102030000700E38E97FA05099790FFFFE780805F1E
:10204000E343A9FE01451703FFFF6700830B170356
:10205000FFFFE7022307AE89AA849790FFFFE7807E
:1020600020532A8497D0FFFFE780A02EAA8601473D
:102070001306840197050000938585E41745FF1F2B
:10208000130505E19790FFFFE780A0192A8925C96C
:102090008C441304C50022859E0593F5050897A07E
:1020A000FFFFE780003DCC4083877400E18163DD62
:1020B000070493E50508228597A0FFFFE780603BB2
:1020C0000D4693854400228597A0FFFFE780803767
:1020D00083D50400228597A0FFFFE780A03E83D52B
:1020E0002400228597A0FFFFE780C03D03D649006A
:1020F00083A50900228597A0FFFFE780A0344A85C9
:102100001703FFFF670043FF93F5F5076DB717034C
:10211000FFFFE702C3FC01112A84328532C697A073
:10212000FFFFE780A0289780FFFFE780803183577B
:1021300004001747FF1F1307E7EE3246231BF10089
:10214000930700F8A30DF1001C471843231AA100C0
:102150008983858BB307F740B28548083ECE231CA0
:102160000100230D010097000000E78080EE05616B
:102170001703FFFF6700E3F81703FFFFE70283F48D
:10218000004101453DC49304C40026853289AE89CF
:1021900097A0FFFFE780802595452A8A2685035B67
:1021A000040197A0FFFFE780E021268597A0FFFFAD
:1021B000E780203F8D45AA8A268597A0FFFFE7800C
:1021C0006020268597A0FFFFE780A03D5C48420A7B
:1021D000135A0A01D2975CC423186401814763989B
:1021E0003A0146054D81330625419337160013F514
:1021F000F70F1703FFFF670023F01703FFFFE70246
:1022000083EB89692A8BAE8B328AB68A814401447A
:10221000314CFD199790FFFFE780C04063CDA400CB
:102220009790FFFFE7800043018D33B5AA001703A5
:10223000FFFF6700C3EB3389840383270B003E99BC
:1022400063170A008347890085043E94E1B703566B
:102250000A00DE854A8533F6C90097000000E78052
:10226000E0F16DD10545E1B71703FFFFE70223E772
:1022700001112A847C000355E5003ECAB707070018
:102280003ECC7C003ECE97200000E78020082A89C3
:102290008545480897A0FFFFE780E0399945480841
:1022A00097A0FFFFE780A016AA844A859720000028
:1022B000E780A0082380A4009747FF1F938787D655
:1022C0009C434166130606F09396870113D7870156
:1022D000558F93D68700F18E558FA207B706FF0062
:1022E000F58FD98F11462C00138514003EC497D06A
:1022F0000000E78020CF5008A38204008945228592
:1023000097000000E780E0E019C9AA85130584035F
:1023100097A0FFFFE780A0323C4085073CC00561E5
:102320001703FFFF6700E3DD1703FFFFE70223DB6F
:102330009790FFFFE78000322A8405049790FFFF03
:10234000E78040303305A402F14791453305F5029B
:1023500097200000E78020BA11E565551703FFFFBD
:10236000670023DA9747FF1F23AAA7B29790FFFFC2
:10237000E780402E2A8405049790FFFFE780802C99
:102380003305A4028945060597200000E780A0B622
:1023900069D59747FF1F23ABA7AE9790FFFFE78054
:1023A000602B2A8405049790FFFFE780A02933045F
:1023B000A4029747FF1F239D87AC9790FFFFE780FC
:1023C00060292A849790FFFFE780C02793071400B5
:1023D0003385A7029747FF1F239DA7AA97070100F0
:1023E0009387C7871747FF1F2328F7AA0145BDB763
:1023F0001703FFFFE70203CDAA842E890144974902
:10240000FF1F938929C2130A80069790FFFFE78078
:1024100060236347A40001451703FFFF6700C3CD96
:102420003305440383A709024A86A6853E95970093
:102430000000E780E0B919E10504C1BF0545E9BF27
:102440001703FFFFE70223C7AA8A2E8BB28B368CB5
:102450003A8A814401448149974CFF1F938C8CBC7C
:10246000130D80069790FFFFE780C01D63C9A4008D
:1024700011E085494E851703FFFF670043C7338985
:10248000A40383A70C025E86D6853E994A859700F1
:102490000000E780E0B31DC19790FFFFE780801B3D
:1024A0000544636D4501D2866286DA85130509030A
:1024B00097000000E780A0D411C1854985045DB76D
:1024C0001703FFFFE70203C0C16441112A890144D9
:1024D0009749FF1F938909B5130A8006FD1436C674
:1024E00032C42EC29790FFFFE780C0159245224666
:1024F000B2466348A400014541011703FFFF67008E
:10250000A3BF3305440383A709023E9509C6834749
:102510003500C18B9DC791C68347350093F70702ED
:102520008DC3630699008357E500639C2701035719
:10253000050001CB63E7E50083478500BA97E3CD4B
:10254000F5FA050469BF1703FFFFE702A3B7C164EB
:102550002A8901449749FF1F9389C9AC130A800651
:10256000FD149790FFFFE780E00D6346A40017037A
:10257000FFFF670063B83305440383A709023E9554
:102580008357E500638A97006304990063962701E7
:1025900097000000E780E0970504E1B71703FFFF0D
:1025A000E702E3B089692A8AAE8A328BB68B81440E
:1025B000174CFF1F130C0CA7930C8006314DFD190F
:1025C0009790FFFFE780000863C6A4001703FFFF92
:1025D0006700A3B13389940383270C028355CA0192
:1025E0005A863E994A8597000000E780609E31C177
:1025F000814D15A03384AD038327090303D60B0057
:10260000D68533F6C9003E94228597000000E78006
:10261000E0B609E9850D9790FFFFE780A000E3CBC6
:10262000ADFC01A8228597000000E780E08A230422
:102630000400850471B71703FFFFE702C3A74169D0
:10264000AA8A014A174BFF1F130BCB9D7D19C14B63
:10265000054C9790FFFFE780E0FE6346AA00170352
:10266000FFFF6700C3A893098006B3073A038329D5
:102670000B02BE9983D7E900638E270163842A0188
:10268000639A570103A4890301E84E85970000006F
:10269000E780C0BD050A75BF8357040163997709B8
:1026A0009304C400268597A0FFFFE78020D48545CA
:1026B0002A8D2685835C040197A0FFFFE78080D0E8
:1026C000268597A0FFFFE78060E862056185635972
:1026D00005048D45268597A0FFFFE780A0CE89459C
:1026E000268597A0FFFFE780E0CD8945268597A046
:1026F000FFFFE78020CD8545268597A0FFFFE78077
:10270000A0CD83470500094793F7F707639AE700D1
:102710009945268597A0FFFFE78000CCA30285019D
:102720004848337D2D01231894016A9548C4004020
:10273000A1BF1703FFFFE702839A37E40400832752
:10274000041D82979737FF1F83C7C77A1715FF1F8E
:102750001305C5DDA300F5008327441C829783275A
:10276000841C81461306F00F8145014582971703AB
:10277000FFFF670003991737FF1F1307A767184369
:102780009735FF1F83C505779737FF1F9387077519
:1027900083468703034697036397D5009737FF1F48
:1027A000238AC774828083C587010347A703631701
:1027B000B6009737FF1F238FE772828003C6870119
:1027C0006317C7009737FF1F2386D772828083C69F
:1027D0008701130750026319D70093076002173768
:1027E000FF1F2309F770828083C6870113066002EA
:1027F0006315D60093077002DDB783C7870155BF05
:102800009737FF1F9387876DD44B0947638DE60881
:102810001703FFFFE702A38C1739FF1F130949694C
:102820003E8483470900918B9DCFB7E4040083A7C2
:10283000041D829783A7441C1735FF1F1305C56726
:10284000829783A7841C81461736FF1F0346C668FC
:1028500081450145829721C583470900ED9B1737C4
:10286000FF1F2307F7648347040093F7F70F85CB17
:1028700091471737FF1F232DF76697000000E78069
:1028800080EB97000000E78040EFB7E70400BC4F03
:10289000414691451735FF1F0345C56482971703CD
:1028A000FFFF6700038682801703FFFFE702238391
:1028B0008D4741116306F504C5476308F502854756
:1028C0006310F5029737FF1F2388A762B7E704005C
:1028D000BC4B930500101735FF1F0345A560829779
:1028E00041011703FFFF6700C38185471737FF1FAB
:1028F0002304F760B7E70400BC4B93050020E1BF59
:102900009737FF1F9387875DD44B1147638DE60090
:10291000B7E7040083A7071D8297B7E70400BC4B05
:10292000930500044DBF05491737FF1F2322275D7C
:1029300083C7070032C62E8493F7F70FD5D3B7E4C9
:10294000040083A7041D7D141374F40F8297E376AB
:1029500089FCB245994703C61500E3F0C7FCFC4467
:1029600009061735FF1F130565598297BC48930563
:1029700000081735FF1F0345E556829779BF17F307
:10298000FEFFE702C3751737FF1F130727554047A0
:10299000184B1C409736FF1F23A8F6546316E4001B
:1029A0001737FF1F2324F754130584FE9790FFFF6A
:1029B000E78020A7035564FF9780FFFFE780A06FA3
:1029C00097A0FFFFE78020D117F3FEFF6700637336
:1029D00017F3FEFFE702A3709737FF1F9387075097
:1029E000D84BDC4789C797000000E78080F985470E
:1029F0001737FF1F232EF74E9737FF1F9387873F09
:102A00009C43930500021735FF1F0345A54D83C75F
:102A100087031737FF1F230FF74CB7E70400BC4BA2
:102A2000829717F3FEFF6700C36D9737FF1F23A937
:102A3000A74A828017F3FEFFE702C36837E4040069
:102A40007C4CA1451735FF1F0345C54982977C483B
:102A5000A1451735FF1F0345E5489734FF1F9384B1
:102A6000E4478297DC4489EB97000000E78080D937
:102A700017F3FEFF6700436803D567FF9780FFFFEA
:102A8000E7806063AA896DD1D84891476310F70247
:102A90007C4C91451735FF1F0345C54482977C4800
:102AA00091451735FF1F0345E543829703A9490167
:102AB00003D409018947B7E904001737FF1F232909
:102AC000F74283A7091D21044204829783C784012A
:102AD0001715FF1F130585A561191717FF1FA307FA
:102AE000F7A483A7491C418082979737FF1F23854E
:102AF000074083A7C91C814609469375F40F4A8590
:102B0000829711E99737FF1F83C7474F89C79700FF
:102B1000FF1FE780200EB7E70400BC4F2146A14508
:102B20001735FF1F0345053C829799B717F3FEFF42
:102B3000E702E35A93F7052001112E8481CF970015
:102B40000000E78020E913450420056117F3FEFF2C
:102B50006700235B93F70510A9CF9734FF1F938479
:102B6000E437DC4897000000E78020C11737FF1FDB
:102B700013074728184383C7840103478703631853
:102B8000F700DC4489C797000000E78080DF8547B5
:102B90001737FF1F232EF734B7E70400BC4B93050C
:102BA00000021735FF1F0345E533829713450410D4
:102BB00069BF93F70508BDC79737FF1F83C7173451
:102BC000E91719469735FF1F938565331305D10023
:102BD00093F4F70F1739FF1F0349493297C00000DC
:102BE000E780404093970401C1831737FF1F130705
:102BF0006731231DF100231CF1009737FF1F9387D6
